:020000040000fa
:080000000002040000000000f2
:020000040000fa
:10000800c2080000c2080000fa040000040500004d
:10001800c2080000c2080000c2080000c2080000b0
:10002800c2080000c2080000c2080000848c00005a
:10003800c2080000c2080000c208000094020000c4
:10004800c2080000c2080000c2080000c208000080
:10005800c2080000c2080000c2080000c208000070
:10006800c2080000c2080000c2080000c208000060
:10007800c2080000c2080000c2080000c208000050
:10008800c2080000c2080000c2080000c208000040
:10009800c2080000c208000092030000c208000065
:1000a800c2080000c2080000c2080000c208000020
:1000b800c2080000c2080000c2080000c208000010
:1000c800c2080000c2080000c2080000c208000000
:1000d800c2080000c2080000c2080000c2080000f0
:1000e800c2080000c2080000c2080000c2080000e0
:1000f800c2080000c2080000c2080000c2080000d0
:10010800c2080000c2080000c2080000c2080000bf
:10011800c2080000c2080000c2080000c2080000af
:10012800c2080000c2080000c2080000c20800009f
:10013800c2080000c2080000c2080000c20800008f
:10014800c2080000c2080000c2080000c20800007f
:10015800c2080000c2080000c2080000c20800006f
:10016800c2080000c2080000c2080000c20800005f
:10017800c2080000c2080000c2080000c20800004f
:10018800c2080000c2080000c2080000c20800003f
:10019800c2080000c2080000c2080000c20800002f
:1001a800c2080000c2080000c2080000c20800001f
:1001b800c2080000c2080000c2080000c20800000f
:1001c800c2080000c2080000c2080000c2080000ff
:1001d800c2080000c2080000c2080000c2080000ef
:1001e800c2080000c2080000c2080000c2080000df
:0801f800c2080000c20800006b
:020000040000fa
:10020800c2080000c2080000fa040000040500004b
:10021800c2080000c2080000c2080000c2080000ae
:10022800c2080000c2080000c2080000848c000058
:10023800c2080000c2080000c208000094020000c2
:10024800c2080000c2080000c2080000c20800007e
:10025800c2080000c2080000c2080000c20800006e
:10026800c2080000c2080000c2080000c20800005e
:10027800c2080000c2080000c2080000c20800004e
:10028800c2080000c2080000c2080000c20800003e
:10029800c2080000c208000092030000c208000063
:1002a800c2080000c2080000c2080000c20800001e
:1002b800c2080000c2080000c2080000c20800000e
:1002c800c2080000c2080000c2080000c2080000fe
:1002d800c2080000c2080000c2080000c2080000ee
:1002e800c2080000c2080000c2080000c2080000de
:1002f800c2080000c2080000c2080000c2080000ce
:10030800c2080000c2080000c2080000c2080000bd
:10031800c2080000c2080000c2080000c2080000ad
:10032800c2080000c2080000c2080000c20800009d
:10033800c2080000c2080000c2080000c20800008d
:10034800c2080000c2080000c2080000c20800007d
:10035800c2080000c2080000c2080000c20800006d
:10036800c2080000c2080000c2080000c20800005d
:10037800c2080000c2080000c2080000c20800004d
:10038800c2080000c2080000c2080000c20800003d
:10039800c2080000c2080000c2080000c20800002d
:1003a800c2080000c2080000c2080000c20800001d
:1003b800c2080000c2080000c2080000c20800000d
:1003c800c2080000c2080000c2080000c2080000fd
:1003d800c2080000c2080000c2080000c2080000ed
:1003e800c2080000c2080000c2080000c2080000dd
:0803f800c2080000c208000069
:020000040000fa
:10040000efd020000e7f22000e01880000000000c7
:1004100000012000200288000c000700809c2800ba
:100420000100200011000700000020000000e00093
:100430000200320000000200000000000e05020071
:10044000000000000040da000000fe004440a90067
:10045000602620000000e0000300320000002000c1
:10046000a00188004440a800000006009101880017
:10047000800078000000eb0015003700e2804000ab
:1004800032a0b4009101ba00e280400032a0b40072
:100490009102ba00e280400032a0b4000002eb00fa
:1004a000472bde00f507b200602ce10004003a00a3
:1004b0000059eb008301e900fdff3e000400370016
:1004c0006128e100010032000082eb000400070017
:1004d0001101ba000200e000e8ff3a000000060047
:1004e0003159ba008301e9000c0032002159ba00e9
:1004f0008301e900080032000400e00003003a0034
:10050000e280400032a0b400f5ff370011d9ba00f4
:100510008301e900faff3a008100e800e180400031
:1005200032a0b40000000600841f78000000fa002a
:1005300084e0a90014002000746088000080fa00a4
:100540004f027800004006000000fa008408800096
:100550000440a0000450a10084088800046b23001c
:10056000640888000002eb003408880084e0a900d9
:1005700094e0a80011e1a8000080fa000000060045
:100580000000fa00940880000440a0000450a1007c
:100590009408880004c42900740888000002eb0055
:1005a0005408880013e1a8000080fa00000006004b
:1005b000ca00fa000002eb00040f7800c45f80005c
:1005c000050020004600200007002000860f520092
:1005d000878f5a0051003e0004600100040037007c
:1005e0001600370028003700350037003d0037007f
:1005f000803d2900148d020000000000c469020043
:100600000000000000027800e10f520004003200f8
:10061000a0402900148d0200000000003f003700b8
:100620000040eb00d279020000000000c45f8000af
:100630000402e800c45f880038003700d042290077
:10064000148d02000000000014c0b300631f2000de
:100650000041eb006000b800a0160200000000009e
:100660000042780004407800f6ebb70064bf200039
:1006700014427800e24f42002300320024002000a0
:10068000c45f88002500370064bf20001442780052
:10069000044078001e1802000000000000027800ec
:1006a000e00f52001a00320080472900148d02002a
:1006b0000000000034002000c45f880017003700ed
:1006c000c46902000000000000027800e10f52003f
:1006d00011003a000040eb00226a02000000000016
:1006e0000e00370064bf20001442780004407800f8
:1006f000e21802000000000014002000c45f88001f
:100700000000000005003700000000000300370073
:100710000000000001003700000000000080fa0027
:1007200000000600801f7800849fbe00861f7800ae
:100730000200fa00b4118000044f780087c0a900bd
:1007400004c02000144278000483fb0005802000d0
:10075000850243009e4a78000442e8000440780085
:1007600000ecb700e4bf2000144278000442e80027
:1007700004407800feebb7000080fa004f037800d9
:100780004f02be004f007800004006000200fa0051
:1007900097c0a900e4bf2000144278000482fb0047
:1007a000040f780097c0a8001e02780004007800ab
:1007b0000080fa00000006000400fa00100798000c
:1007c0001e029000040f780084118000660262000f
:1007d000e60f52001e003a000c0037000000000037
:1007e000951180000420200004826200e00f520076
:1007f000fbff3a001e02900014027800a41188004a
:100800001e0290000482e800140798001e02900067
:1008100014027800e00f5200f0ff3a001100370098
:100820000000000095118000042020000482620076
:10083000e00f5200fbff3a001e02780014427800dd
:100840000402fb00a41188001e0fe800010037001d
:10085000000000001e02780014427800e04f5200b1
:10086000efff3a000080fa00000006000a00fa00dc
:100870002007980031079800420798000002eb001b
:10088000040f78003e0290001407980024003700ff
:100890004e0290009e027800848f520002003100c8
:1008a0001e0fe800030037002e02900020003700e2
:1008b000000000002100070000427800e04f5200d5
:1008c000f3ff32000002eb00040f78008411800077
:1008d00066026200e60f520007003a00b511800080
:1008e0003e029000050a78003e0290000482e80073
:1008f0003407980007003700b411800004427800e4
:100900009e029000844a78001e0290000402e800d3
:10091000140798002e0290000402e90024079800b2
:100920002e029000e00f5200e1ff3a002e029000ec
:10093000040078000080fa00000006000000fa00c1
:100940009411800004427800614262000440780003
:100950000080fa00000006000000fa0095118000f7
:10096000041020000482620004f0a7000402ea00e0
:100970000402e9004f22de000442780004407800bf
:100980000080fa00000006000000fa0084118000d8
:1009900066026200e60f520002003a00b4118000c5
:1009a00003003700b5118000f40f200004826200bc
:1009b000040078000080fa00000006000200fa003f
:1009c000000f78008411800066026200e60f52007a
:1009d00003003a001e027800a411880003003700cb
:1009e000f40f20001e026200a41188000080fa00ab
:1009f000000006000000fa000000000000000000f7
:100a00000080fa00004006000000fa00000000002c
:100a1000000000000080fa00004006000400fa0018
:100a2000a201070092010700a6010700e4000700e9
:100a30005a8802000000000024b720005202200063
:100a4000214a290004007800d80b020000000000b1
:100a5000e888020000000000a4020200000000007c
:100a6000c00202000000000001010700a51680007e
:100a70000400220004826200e00f52003d003a00b0
:100a8000e48b0200000000000002be00048fbe00e4
:100a9000452c20000042eb00844a780030003700eb
:100aa000e48b0200000000000002be003e03520082
:100ab000ae835a0004092d0035002000840f530036
:100ac000858f5b00260036006000b800ae7f020014
:100ad0000000000000c0eb00c67f02000000000024
:100ae00000c0eb00c67f0200000000003a80020058
:100af00000000000452c2000f4c0b300844a7800b8
:100b000000000000e48b0200000000000002be00b4
:100b10003e035200ae835a000602be000403be002c
:100b200024aa240045002000840f5300858f5b0019
:100b3000f4ff3400452c20000042eb00844a78008a
:100b400000000000a516800004002200048262005c
:100b5000e00f5200fbff32000000fe0005003700ee
:100b6000a51680000400220004826200e00f5200fb
:100b7000cbff3200c48102000000000001003700fa
:100b800000000000e48b0200000000000003be0033
:100b9000e4588000f55880000403530085835b000f
:100ba00014a1270005002000840f5300858f5b00ef
:100bb00011003600e48b0200000000000002be00bd
:100bc000e4588800f5588800241680000442780014
:100bd000614262000404a200614262000482fb00e0
:100be0006102620026168000e5ff2f008502630087
:100bf00004827200241688000c82020000000000ab
:100c00007484020000000000d8020200000000000e
:100c10009c8c02000000000061000700f456800078
:100c2000055780000659800017598000860f520032
:100c3000878f5a00d2ff3200f4568000055780009b
:100c40000459880015598800f45680000557800023
:100c50000400be00030007007e84020000000000c4
:100c6000c8ff37000c00fa00881f78004007980082
:100c70005107980004c1b300244798000042eb00dc
:100c8000044f7800330037009e4278000582fb0055
:100c9000e802470004824200144278000482fb000c
:100ca000e30247008500780004007800b065020088
:100cb000000000000042eb00144798000f003700ce
:100cc0002e4290000483fb001e4290000482fb0031
:100cd000040247003442900025b7200085024300fb
:100ce000844a78002e4290000442e800244798008d
:100cf0001e4290000442e800144798001e429000f3
:100d00000484fb006302470004007800160c020014
:100d10000000000000027800840f5400e8ff390052
:100d20001e427800e34f52000e0032002e42900027
:100d30008482fb0024b7200084824200e4c2b30016
:100d4000844a78002e4290000442e800244798002c
:100d50001e4fe8001e427800e34f5200caff3600e3
:100d600001003700000000002e429000ff4f5200ab
:100d700006003e002e4290008482fb0024b7200033
:100d8000848242000042eb00844a7800e888020036
:100d9000000000004f0478000080fa000000060008
:100da0000000fa000418800041b12000040078001f
:100db000b0650200000000000080fa00000006009c
:100dc0000000fa00c002a900c022a900c042a90088
:100dd000c062a900c082a900c0a2a900c0c2a90027
:100de000c4e2a900452c20000042eb00844a7800b0
:100df000243a80000480a1000490a10004a0a10076
:100e0000243a88000002eb00441988002c83a900d2
:100e10002ca3a900444e2800041988004440200057
:100e200014198800340021002419880004022000cd
:100e30008419880097c0a800040028008411880045
:100e4000044020009411880034032000c41188005d
:100e5000d7c2a800d3c2a900d782a800d382a90014
:100e60004c7e0200000000000080fa000000060036
:100e70000800fa00881f78000042eb00044f780059
:100e8000320320008000eb00e0ad2000e60b020002
:100e9000000000000acba8000aeba80062002000b6
:100ea000714c2900b0b02000d80b020000000000f7
:100eb000048c2a0055f02000f4568800055788005d
:100ec000f45680000557800094578800a557880085
:100ed000f4ff2f00f50f20001457880025578800d5
:100ee0001457800025578000b4578800c5578800e4
:100ef00094ea2f00151020003457880045578800c9
:100f000094ea2f0015102000545788006557880078
:100f10006022b800745788008557880002012000bd
:100f2000d14c2900a0af2000d80b02000000000027
:100f3000a0af2000ae6802000000000031032000d6
:100f4000e0ad2000ee670200000000000002780023
:100f5000945888001e427800e04f52000200320090
:100f6000e0ad2000260007000e82e80063002000ac
:100f7000040178006000b800d27e0200000000008a
:100f800033032000e2ad20006000200001002000bb
:100f9000d27e0200000000009e0290003403200078
:100fa000848f52000c003a00ae02900094588000ea
:100fb000848f520008003a003e0490003103200064
:100fc000e0ad2000ee6702000000000000027800a3
:100fd000840f5400070032001e427800e04f520098
:100fe00001003200ffff370014c0b300044f780047
:100ff000a3ff37004f0478000080fa0000000600cd
:101000000800fa00300798009458800014079800f0
:101010003e0290003103200004007800ee670200d9
:10102000000000000002780024079800340320002c
:10103000040f78006000b800ae7f020000000000de
:101040000e02780061002000040078000c8002008d
:10105000000000003e0290003103200004007800f0
:101060000c800200000000000080fa000000060072
:101070000000fa00440e200004198800c403200078
:101080001419880094d020002419880054002000ee
:1010900044198800f4fd2f00641988000002eb0059
:1010a000841988000080fa00000006000000fa00a1
:1010b000d2c2a80004f02f00041688000080fa00b5
:1010c000000006000000fa0021e3a8000080fa00fa
:1010d000000006000600fa000518800014188000c1
:1010e00084824200241880008482420034188000e8
:1010f0008482420044188000848242005418800098
:101100008482420064188000848242007418800047
:1011100084824200841880008482420094188000f7
:1011200084824200a418800084824200b4188000a7
:1011300084824200c418800084824200d418800057
:1011400084824200e418800084824200f418800007
:101150000482420005002000048fbe001e02be0073
:10116000452bdd004b22de0004027300cb2ade009b
:10117000240798002e029000040078000080fa00f6
:10118000000006000040da000000fe0000c0da00a7
:10119000000006000a00fa00e20f500022003e00a4
:1011a00084608000e10f5200060032008723200097
:1011b000462320002423200005232000e08f530035
:1011c00004003a008722200046222000242220002a
:1011d00005222000000028001500600003003a00ee
:1011e000800b780007002800958a730005402000d6
:1011f0009482620001003a0014a0a00082027800ec
:1012000006003700940378000710b200fdff32009b
:10121000b103fb00070b78008502e900e08f520064
:10122000f8ff3a000800370034002000b4bf9f00e8
:10123000c0bf9f00d1bf9f00e2bf9f006a805700e0
:10124000d2ff07006fb99700020078000080fa0013
:1012500000000600889fbe008a9fbe008c1f780099
:101260000006eb00e00f5000e08f5800e00f59003f
:10127000e08f590007003d006044b8006055b80099
:101280000000540081805c0002015d0083815d00ec
:101290001c002000e00f5200e08f5a00e00f5b00be
:1012a000e08f5b0007003d006044b8006055b80067
:1012b0000402540085825c0006035d0087835d00a4
:1012c0000c00a20012010700e00f560006003200d9
:1012d0006022b8006033b8000000520081805a00dc
:1012e00002015b0083815b004f0678004f05be0062
:1012f0004f04be0000000600889fbe008a9fbe000b
:101300003004be002005be000404440085844c0067
:1013100006054d0087854d000898be000a90be0066
:101320000440e10005c8e10006d0e10007d8e10073
:1013300002003100680040001008e8004f05be00c0
:101340004f04be00000006001000fa00889fbe0097
:101350008a9fbe000605be000404be003002be0027
:101360002003be00c4b79f00d5b79f00e6b79f001b
:10137000f7b79f000802520089825a000a035b00f7
:101380008b835b0084bf9f0095bf9f00a6bf9f001b
:10139000b7bf9f000498be000698be001100200051
:1013a0004fb29700dfb297006fb39700ffb397007b
:1013b000b2000700010039008000eb001088100027
:1013c0004f05be004f04be000080fa00000006007a
:1013d0001400fa00889fbe008a9fbe008c9fbe004a
:1013e000790007000605be000404be000006eb00fd
:1013f000ccb79f00bcb79f00acb79f009cb79f00c5
:101400008cb79f000d0420004fb39700bfb2970028
:10141000860343002fb29700e00f530004003d0005
:101420009b0007000f004000b3ff070003003700d8
:10143000970007000f004000c3ff0700cfb29700de
:1014400095bf9f00e08f520009003500650007003e
:1014500014002000050020006033b8000000720076
:1014600081807200020173008381730056000700bf
:101470000c06e8008d0f5600e3ff3a001fba9700f4
:10148000e00f520005003d000802be000a03be0046
:1014900000fe2f000f00400097ff07004faa9700a3
:1014a000e00f520008003a000fb497009fb4970075
:1014b0002fb59700bfb59700d8b79f00e9b79f0039
:1014c000fab79f008bbf9f00460007004f06be0083
:1014d0004f05be004f04be000080fa000000060069
:1014e000881f780018002000881f7800b8ff0700c8
:1014f0008f87e9004f04780000000600801feb0092
:10150000b3ff07008f87e90000000600889fbe0038
:101510008a9fbe004100070007003d00440007000d
:10152000180020004900070008003d002f000700b8
:101530000004eb00050037000004eb004300070047
:1015400002003d002900070018002000e4ff07000a
:10155000e00f540001003200410007004f05be00bb
:101560004f04be0000000600889fbe008a9fbe0098
:101570008c1f78002900070005003d002c000700a3
:101580001c0020003d00070007003d00050037005b
:101590000006eb002d00070003003d006044b8008a
:1015a0006055b80013000700d4ff0700e00f560095
:1015b000010032002a0007004f0678004f05be00e8
:1015c0004f04be00000006000100070000000600f6
:1015d00090b79f00a1b79f00b2b79f00c3b79f000d
:1015e0000000060008000700000006006044b80084
:1015f0006055b8000402540085825c0006035d005b
:1016000087835d00000006001fb09700afb0970011
:101610003fb19700cfb1970000000600e00f5000e7
:10162000e08f5800e00f5900e08f590000000600dd
:101630006044b8006055b8000000540081805c0030
:1016400002015d0083815d0000000600e00f520092
:10165000e08f5a00e00f5b00e08f5b0000000600a7
:101660006022b8006033b8000000520081805a0048
:1016700002015b0083815b00000006000820e1009e
:1016800009a8e1000ab0e1000bb8e1000000060083
:101690004f2bde0087037300a7b79f004f23de00a8
:1016a000858242008502730095b79f00ffaa9700cc
:1016b0004f2bde00040242000402730084b79f0037
:1016c0006faa97004f23de008582420085027300d7
:1016d000f5af9f00ccff07004f18de000402420068
:1016e00000027200e4af9f00c7ff07000000400047
:1016f000818048000201490083814900b4ff07004e
:101700000802be000a03be0000fe2f000000060013
:10171000889fbe008a9fbe008c9fbe000404b80054
:101720000506b8008904460060854e000606b8002c
:101730000a054600e0854e000706b8008b05460006
:10174000040eb800890446000a854e00e0854d006d
:10175000050eb8000a0546008b854e00060eb8003f
:101760008b0546000416b8000a0546008b854e001e
:101770000516b8008b054600041eb8008b05460010
:101780000800be000a01be004f06be004f05be00a5
:101790004f04be0000000600020ab900001bb90099
:1017a0000200b800810042008100430000000600f2
:1017b0000002780002003700315a78000201e90087
:1017c000e00f5100fcff3a00000006000002780024
:1017d00002003700015a78000201e900e00f5100d1
:1017e000fcff3a0000000600000278000600370007
:1017f0000201e90031437800065a7800840278003b
:10180000e04f53000600320084027800e00f5100e0
:10181000f7ff3a0002003700805aeb000201e900ae
:10182000e00f5100fcff3a000000060000027800c3
:101830008042eb00b4cf1200fdff3a000080ea00c6
:1018400000004200000006000c00fa00889fbe0065
:1018500000047800f4ff2700d4bf9f008004eb0051
:1018600099bf9f0088bf9f00a8bf9f00240c200045
:10187000b4bf9f0078815700cfb0970070805700a9
:10188000220007000fba9700094a78000fba9700a4
:10189000080052004f04be000080fa00000006005d
:1018a00001002000206888003168880015c0b3005e
:1018b00024d02000054a78000000060024d0200033
:1018c0008042eb0094cf120002003a00100020008a
:1018d000f3ff0700d2e62400631c24002068800088
:1018e00031688000acff070094032300050020004e
:1018f0000002420081824a0024688800356888001e
:101900000500780000f0a100000006002f03b000e1
:10191000889fbe008a9fbe008c9fbe008e1f7800ed
:10192000e0af9f00c1af9f00b2b79f008006eb0001
:101930006e023700cfa897008100e800c1af9f007a
:1019400054c2b300844f500006003a0001027800f0
:101950000006eb0001c3b30000c2b300b7c2b3007e
:10196000070037000000fb00efa897006b0207009c
:10197000e10f40005d0232008d06e8005b02370097
:101980008402780034437800d2c2b300824f5300ff
:101990000900320005003c00804f5300080032006f
:1019a000874f53000c003a0007003700814f530067
:1019b00009003a00060037000c30a000f0ff3700a5
:1019c0000c00a000eeff37000c10a000ecff370069
:1019d0000c20a000eaff370062026600010032001e
:1019e0000c00a10068026600010032000c20a1007a
:1019f0000602fb000403b100e90f52000c003e0098
:101a0000050378000002eb006a22b900b603fb0070
:101a10000703b10004824300860278009603fb00ae
:101a20000703b100e98f5300f7ff360008003700c5
:101a30000002eb00a7c2b300874f530004003a0036
:101a4000bfb1970043027800b3b79f008502e8005a
:101a50000007eb00e6c2b300954f13000a003a00fe
:101a60000ce0a00064435300d54f13000200320085
:101a700005037800080037003fb397004607780059
:101a8000b6b79f008502e80005037800080037001c
:101a90006a70b9000087430086027800b603fb0035
:101aa0000703b100e98f5300f9ff3600f6ff370056
:101ab000b6427800c6af9f00c0c6b30080cf5200c8
:101ac000250032000f003c0036c6b30086cf52001e
:101ad0006e00320004003c00e0cf520008023200e9
:101ae0006b4353000f00370046c6b30086cf520049
:101af000170032006543430086cf520083003a004e
:101b00001300370036c7b30086cf52001f003200e3
:101b100007003c006443530086cf5200140032009b
:101b20000643e80086cf520078003a0013003700e1
:101b300056c7b30086cf520079003200634343009a
:101b400086cf520071003a00a5c79f000d003700f4
:101b5000a5c79f0074003700f00366000501200050
:101b6000010032000500280005067600d0ff37008e
:101b7000a5c79f000c60a0006b003700a5c79f00a1
:101b80000c50a0000c70a00067003700a5c79f0094
:101b9000bfb09700c1027800b1b79f00050478007c
:101ba000e08f520001003a0048cd20000803780081
:101bb0008002eb00010037008502e800e6c37a00ee
:101bc000e0cf5300fcff3a0085047800e00f570097
:101bd00003003200890f5700010031008e047800a5
:101be0000007eb00890f5200010036000907520080
:101bf0006806660014003a0007003700efa8970057
:101c000000022000c5010700e10f40000100320082
:101c10008d06e8000e07e900e00f5700f7ff3a00d5
:101c20000087eb0008003700080278003400fb0052
:101c300004047800efa89700b8010700e10f400006
:101c4000010032008d06e800090278008404e900f2
:101c5000e00f5200f4ff3a00e00f5600a3013200fb
:101c600007003700efa8970000022000ab01070033
:101c7000e10f4000010032008d06e8000e07e90088
:101c8000e00f5700f7ff3a00980137003fb1970087
:101c9000c2027800b2b79f0005007800cf80de0056
:101ca0000101780082017800f0af9f0081b79f00aa
:101cb00092b79f00a3b79f004800de00c80add006e
:101cc00000807200a0c79f00700366000900320008
:101cd000e04f500007003200e14f400005003200a5
:101ce000b0c79f006fdb9700c6c79f002900200088
:101cf00003003700efdb9700b7c79f0019002000f3
:101d000038fc2f000f044400b0ff3700a5c79f0028
:101d100028fc2f000f04440019002000abff3700ff
:101d2000a5c79f000c0cb3008c027800050cb20014
:101d30002b003a00e00f560005003d003fb0970031
:101d40004005be004004be00b0b79f00170037003a
:101d5000f00266000f003200bfb297004501be00de
:101d6000b5b79f00c2a79f00d3a79f0005037800c7
:101d700096029000cfaade00e5a79f00f5a79f007e
:101d80004fa49700dfa497006fa59700ffa59700c9
:101d9000060037003fb0970040047800b0b79f00be
:101da000cfc4de00090578008a057800e00f5400f2
:101db000e08f5c00e00f5d00e08f5d0025003d00de
:101dc0003c00b3006000b8006011b8000804500087
:101dd000898458000a0559008b8559001d00370079
:101de000e00f560005003d00bfb097004105be0062
:101df0004104be00b1b79f0016003700f002660034
:101e00000e003200bfb297004501be00b5b79f007b
:101e100082af9f0093af9f000003eb00a6af9f002f
:101e20008003eb00b7af9f000fac97009fac97000b
:101e30002fad9700bfad9700060037003fb0970069
:101e400040047800b0b79f00090020000a0020007d
:101e50000b002000e00f570007003a001e00200092
:101e6000e00f5400e08f5c00e00f5d00e08f5d004c
:101e7000010032000007eb008c007800010cb2007a
:101e8000f1af9f0005042000858f50002c00320028
:101e900003003c00e08f5000080032003c00370097
:101ea000050820007fa99700850f5100100032001f
:101eb000050c2000850f510035003a00a6c1200016
:101ec00015c0b3003600be003601be000040e10080
:101ed00001c8e10002d0e10003d8e1002b00390085
:101ee0008542e800f4cf5200f6ff3a0027003700a1
:101ef00015c0b30000012000010020006011b800ef
:101f00000040e10001c8e10002d0e10003d8e10097
:101f10001e003900460020000000d0008180d20061
:101f20000281d2008381d2000603e900faff3a0061
:101f30008542e800f0cf5200f1ff3a00130037006d
:101f400015c0b30080002000010020006011b8001f
:101f50000040e10001c8e10002d0e10003d8e10047
:101f60000a003900370020000000d0008180d20034
:101f70000281d2008381d2008703e900faff3a0090
:101f80008542e800f5cf5200f1ff3a00a5c79f0057
:101f90002fc097008002fb008e8f520002003d0090
:101fa000aec79f0003003700850f570001003d00ba
:101fb00005077800e00f520003003200e3026600dc
:101fc000010032000402e9000500240085026600d9
:101fd000050032008e0f5200020034000e02520043
:101fe000010037000002eb002fc197008202fb00c6
:101ff0008001eb00d3af9f00850f52000200340038
:1020000085025200d5af9f00640266002c003200aa
:10201000e202660061026600e08f520006003200b4
:10202000b0022000e00f5200010032000080e80002
:10203000efa8970004003700e00f520006003200be
:10204000efa8970000022000b4000700e10f400055
:10205000010032008d06e8005faa9700e00f5200f1
:102060008d0032000802be000a03be00dfac9700fc
:10207000efa8970000032000c4b79f00d5b79f00ca
:10208000e6b79f00f7b79f00a40007004fb2970084
:10209000dfb297006fb39700ffb39700e10f4000e6
:1020a000010032008d06e8008904e900f0ff3a00e3
:1020b000d9af9f000605be000404be0076003700bd
:1020c000dfaa9700e08f5200180032006802660015
:1020d00016003a000802be000a03be00dfac9700fb
:1020e000efa8970000022000c4b79f00d5b79f005b
:1020f000e6b79f00f7b79f00880007004fb2970030
:10210000dfb297006fb39700ffb39700e10f400075
:10211000010032008d06e8008904e900f0ff3a0072
:10212000d9af9f000605be000404be00e2026600af
:1021300061026600e08f520006003200b00220000b
:10214000e00f5200010032000080e800efa8970085
:1021500004003700e00f52004f003200efa8970054
:10216000000220006d000700e10f40004a0032002d
:102170008d06e800480037000e07e9007fab9700a6
:1021800007042000870f53002d00320003003c009d
:10219000e00f530008003200370037000408200029
:1021a0007fae9700840f560012003200040c20000e
:1021b000840f560030003a004372dd0020c1200039
:1021c000000242005403be004402be000800be00ec
:1021d0000a01be00c2fc0700a40020000500200088
:1021e0006033b800c5fc070004c3b30004424000dc
:1021f0002000370034cc2000bfa29700e08f5200af
:102200000100320024cb2000c272dd000800be00b5
:102210000a01be008502e900050033008301d100f8
:102220000281d3008180d3000080d300f9ff370002
:102230006f00600064407800a0c79f000e00370068
:102240006372b9000800be000a01be0004067800ef
:102250000c06e900050033008301d1000281d300a0
:102260008180d3000080d300f9ff3700674260000f
:102270000443b000a4c79f00afc097000100fb005b
:10228000efa8970025000700e10f4000060032008c
:102290008d06e800040037000c0178000202b2004d
:1022a000b2a79f008cbf9f00e00f5700b2ff3a001b
:1022b0000fbe9700680666000c003200dfa9970089
:1022c000e08f51000900340003067800efa8970062
:1022d0000002200011000700e10f40000100320061
:1022e0008d06e8000c06e900f8ff3a004faa9700b7
:1022f00014407800a0c79f00e04f50008dfd3a00c9
:102300000d0078004f0778004f06be004f05be0055
:102310004f04be002f03b10000000600889fbe00de
:102320000104780038029000e20262008084eb0031
:102330003b003200040378000620b20098029000af
:1023400002003a00e08f520035003a000490a000ed
:102350003404980080047800f90fb200e08f520036
:1023600002003a00a8029000050c7800ea8f5400a1
:1023700005003a000408b20003003a008800780023
:10238000d0002000e5ff070018029000d80290005e
:10239000850f52000b0032000402e800140498007c
:1023a00018027800094a7800040ce80015c0b30050
:1023b00084d02000054a7800ea8f540018003a00c3
:1023c00005003700880078000940780017000700f2
:1023d0008004780012003700380290000410b20028
:1023e0000f00320018019000a800900048009000f3
:1023f00068fb070018029000840f500004003200b0
:10240000380290000403b300340498008084eb0089
:102410000002eb001404980028029000040c7800dd
:10242000090078004f04be00000006000200fa0018
:10243000889fbe00a0ff9f00010478003802900032
:10244000840278000504b200020032000000fb00a4
:1024500035003700e202620005003a000403b300d1
:1024600034049800150498000080eb002e0037001b
:10247000d8049000e08f540006003a0012002000bb
:10248000e68057004800900042fb070019049800be
:1024900023003700a8029000e08f520008003a00a5
:1024a000b5d0200025049800050c780025002000f8
:1024b00055049800150498000430a00034049800d6
:1024c00018019000a80090004800900031fb070020
:1024d000280290008082eb0015049800affa970064
:1024e000054a7800040ce8002ffa9700ea4f5200e2
:1024f0000b003a00380290000410b20008003200cd
:1025000018019000a80090004800900021fb0700ef
:102510000002eb0014049800a8029000050c78005b
:102520002ffa97000400fb004f04be000080fa0061
:0425300000000600a1
:020000040000fa
:1025340045720000726f0000723a0000204d0000e6
:10254400535000004c5f0000527500006e4d0000b7
:102554006f64000062750000733a000020450000bb
:10256400727200006f72000020720000656100004a
:10257400646900006e67000020410000646400008c
:1025840069740000696f00006e6100006c20000037
:10259400416400006472000065730000732c000045
:1025a40020450000727200006f720000636f00002b
:1025b40064650000203d0000202500006400000048
:1025c40045720000726f0000723a0000204d000056
:1025d400535000004c5f0000527500006e4d000027
:1025e4006f64000062750000733a0000205500001b
:1025f4006e73000075700000706f0000727400004c
:102604006564000020500000726f0000746f0000c9
:10261400636f00006c200000436f000064650000dd
:10262400202800002564000029200000666f0000b7
:10263400756e000064200000696e0000204d0000eb
:102644004241000050200000686500006164000001
:102654006572000000450000727200006f72000095
:102664003a2000004d530000504c00005f5200001f
:10267400756e00004d6f0000646200007573000009
:102684003a20000057720000697400006550000091
:102694006f7200007420000066610000696c000025
:1026a400656400002c20000045720000726f000079
:1026b400726300006f640000652000003d2000008c
:1026c4002564000000450000727200006f72000073
:1026d4003a2000004d530000504c00005f520000af
:1026e40065610000644d00006250000064750000e4
:1026f4003a20000042750000666600006572000022
:10270400207400006f6f0000207300006d610000f2
:102714006c6c0000207400006f20000072650000e3
:102724006164000020500000445500000045000092
:10273400727200006f7200003a2000004d530000d6
:10274400504c00005f52000065610000644d0000c1
:1027540062500000647500003a2000004d530000f0
:10276400504c00005f52000065610000645000009e
:10277400616300006b650000742000006661000066
:10278400696c0000656400002c20000045720000a4
:10279400726f0000726300006f6400006520000027
:1027a4003d2000002564000000000000436f00008d
:1027b4006c77000061790000205300006f6c00000a
:1027c40075740000696f00006e730000204d0000f6
:1027d4006f64000062750000732000004d6100000a
:1027e400737400006572000020500000726f0000d6
:1027f400746f0000636f00006c2000004c690000df
:102804006272000061720000790d00000a0000008d
:1028140045720000726f0000722100002055000014
:102824006e610000626c000065200000746f00009f
:10283400206900006e69000074690000616c00008a
:1028440069730000652000004d530000504c0000e7
:102854000d0a0000000d00000a4d00006f64000026
:10286400627500007320000053650000727600005a
:10287400657200002069000073200000616300009d
:102884007469000076650000206f00006e2000006f
:10289400706f0000727400002035000030320000b8
:1028a4002c2000007761000069740000696e00004c
:1028b40067200000666f000072200000636f000054
:1028c4006e6e000065630000746900006f6e0000a6
:1028d40020720000657100007565000073740000cb
:1028e4002e2e00002e0d00000a0000000d0a00002c
:1028f4004d6f0000646200007573000020530000f7
:10290400657200007665000072200000436f0000cd
:102914006e6e000065630000746900006f6e000055
:1029240020610000636300006570000074650000ae
:1029340064210000212100000d0a000000000000b5
:10294400436f00006c77000061790000204d0000a7
:10295400535000004c20000020760000352e00006b
:10296400343200002020000020200000202000003d
:102974002020000020200000202000002020000053
:1029840020200000202000000000000004a300001c
:1029940000000000004d00004348000050420000c9
:1029a4004f41000052440000000000000d0a0000e6
:1029b40044480000435000002f5000006f7700008f
:1029c4006572000020650000766500006e740000ea
:1029d400206f0000636300007572000072650000e0
:1029e4006400000001000000f4010000f401000094
:0c29f40001000000f4010000f4010000ec
:020000040000fa
:102a00000200fa00004f780084c0200014427800d1
:102a10009e4f52002100320084c0200014427800f2
:102a2000e24f42000c00320084c0200014427800c3
:102a30000482fb007e22b90084027800c49c20003e
:102a400004824200e2012000c1a6200004007800b8
:102a5000d80b0200000000001e40780008ecb70010
:102a60001e427800e24f42000e0032009e42780083
:102a70000582fb007e22b90084027800c49c2000fd
:102a800004824200e201200084007800c0a62000f9
:102a9000d80b020000000000030037000000000017
:102aa00001003700000000000080fa00000006006e
:102ab0000000fa0095c020009542780084c02000f4
:102ac0001442780084cf52002f00320094c02000be
:102ad00014427800e24f42001a00320087a0200022
:102ae00094c02000144278000482fb007e22b900ca
:102af00004027800fc024200c49c200004824200d0
:102b00001443780094c02000144278000482fb0033
:102b10007e22b90084027800c49c20000482420016
:102b20001402780085fd2f00848242008402200078
:102b300013c0b300070178008640780005007800d4
:102b40006111070084c0200014427800044078001e
:102b500009ecb70085a820009542780064538000f6
:102b600087fd2f008483430086a02000840220007c
:102b7000854178000701780011c0b3000600780095
:102b80005111070001003700000000000080fa002a
:102b9000000006000c00fa00e45e20001407980014
:102ba00034608000e00f520009003a002863020000
:102bb000000000000002be0084027800f47f2000c4
:102bc0008482620004402000048242003460880055
:102bd000c20320008000eb0000a32000e60b0200ef
:102be000000000000042eb00444798000042eb0068
:102bf000044f78004d0037001e40780080ff07002a
:102c00001e4078000082fb006622b9008402780032
:102c1000444f290004824200944290005547980096
:102c20001e4078000082fb006622b9000402780092
:102c30008482e800444f2900048242009402780014
:102c4000350798001e4078000082fb006622b9001c
:102c500004027800e4024200444f2900048242004a
:102c600094027800450798005e4290000482fb00c1
:102c7000e00f5200010032002b0037001e009000d0
:102c800050079800be0290004e02900084824200dd
:102c90001e02900004824200a402b00014079800b3
:102ca0009e029000e4e12000848f5200fcff3e0071
:102cb0005e40900088eab7005e0290008402b00097
:102cc00064538800655380003e02900004824200f5
:102cd0000402e80074538800755380004e0290008f
:102ce0000482420084538800d400200014548800d9
:102cf000846aa9006eff07009e4278000582fb00ef
:102d00006622b90084027800444f29000482420000
:102d100014427800044078002feab700290b07001e
:102d20001e4fe80001003700ffff37001e42780009
:102d3000e14f5200b0ff36000080fa0000000600ac
:102d40000c00fa00100798002107980062479800cd
:102d500043079800244f98000042eb00044f78008e
:102d60009a0037001e40780025ff070014548000a9
:102d7000ed0f520091003a004dff0700f5a2200030
:102d8000954278002e4a900084cf52008d003a0080
:102d900084212000645188006e429000e04f520070
:102da00008003a004e009000c0508800846aa800d5
:102db00044002000145488004e02900034548800cf
:102dc0007c00370035608000f43f2000848f520083
:102dd000040036003560800084382100848f520062
:102de0000200360004402000346088003460800017
:102df000c45088000402e80034608800ce039000cc
:102e0000b7508800e48b0200000000000002be0002
:102e1000d4538800e5538800848aa8006e4290004d
:102e20000482fb006123b9000082eb008082eb008a
:102e30000602420087824a00360020000700200078
:102e4000860f5200878f5a005a003e00046001002e
:102e50000300370002003700160037002d0037004e
:102e60001e029000ae029000f450880005518800c8
:102e70006e4290000414a2000482fb000402e900e8
:102e80004f22de00044278000482fb0061026200ef
:102e90004222dd0056518000b5ff2f0085026300fd
:102ea00004827200545188000002eb001454880020
:102eb000400037000e82e800940290000e82e80085
:102ec00014027800848242004e0290008482420004
:102ed000c450800004826a00345488001e029000ae
:102ee000ae029000f4508800055188000042eb00cb
:102ef000044078002eeab700d4032000050020002b
:102f00004450880055508800240020001454880044
:102f1000280037001e029000ae02900004027800e4
:102f200084027800254290000483fb003542900023
:102f30000482fb004822dd000602720004037800d0
:102f40001e029000ae0290000402780094437800c4
:102f50008782fb00144290000482fb004822dd00bf
:102f600005027200840243004e02900084824200f7
:102f7000c450800004826a00345488001e0290000d
:102f8000ae02900004027800a200200084007800c5
:102f9000e0a12000d80b0200000000005400200037
:102fa0001454880011c0b30020c0b30039070700d3
:102fb000000000001e4278000800370000000000fa
:102fc00001003700000000001e4fe8001e4278009c
:102fd000e14f520063ff3600e4cfb30004407800b5
:102fe0000080fa00000006000200fa00004f78009e
:102ff0001e427800e14f520002003600140020000b
:103000000b0037001e4078007dfe0700255480002d
:103010000400210004826200e00f5200030032002d
:10302000858aa90014002000010037000002eb008f
:10303000040078000080fa00000006000200fa0098
:10304000004f78001e427800e14f52000200360027
:103050000002eb00080037001e40780068fe070001
:103060001454800067026a0004f0a7000402ea001a
:103070000402e9004f22de00040078000080fa001c
:10308000000006000200fa00004f78001e4278009f
:10309000e14f520048003e001e40780058fe0700f5
:1030a000b4538000c45388001454800005002000ed
:1030b000e600200007002000860f5200878f5a008c
:1030c00037003e0004600100120037000d00370099
:1030d000100037000f003700310037000d003700b7
:1030e0000e0037000d0037002d0037002c00370090
:1030f0002b00370018003700290037002800370060
:1031000024003700265a0200000000002d0a0700a4
:103110002a0037002b0a07002800370011c0b3002f
:1031200010c1b300db060700d4508000e00f52004e
:103130000500320095538000a4508000848f520017
:10314000f6ff3a0001003700000000008400200074
:10315000145488001900370011c0b30010c1b30027
:10316000cc060700d4508000e00f5200050032006a
:1031700095538000a4508000848f5200f6ff3a00df
:103180000100370000000000c40020001454880033
:103190000a003700d40020001454880007003700cc
:1031a0008040eb0040c1b300ba060700050a0700e3
:1031b0000000000001003700000000000080fa005d
:1031c000000006000200fa00004f78001e4278005e
:1031d000e14f520006003e001e40780008fe070046
:1031e000846aa9001e407800a6ff0700010037008e
:1031f000000000000080fa00000006000200fa0053
:10320000004f78001e427800e14f52000200360065
:103210000002eb000b0037001e407800f8fd0700ad
:1032200023fe0700a2002000e1a12000a0a82000aa
:10323000d80b020000000000b4508000a4548800a5
:10324000a4a82000040078000080fa000000060016
:103250000200fa00004f78001e427800e14f520051
:103260000b003e001e407800e5fd070010fe070041
:1032700095538000a4508000848f520005003200d6
:1032800011c0b30000c1b30082060700010037007f
:10329000000000000080fa00000006000400fa00b0
:1032a000204798002e429000e14f52000200360065
:1032b0000002eb001d0037002e409000d0fd0700fb
:1032c00014548000044f78001e427800e74f5200eb
:1032d000050032001e427800eb4f5200020032001f
:1032e0000002eb001100370095538000a4538000ca
:1032f000848f5200090039007553800064538000a8
:1033000084825200a653800094538000040253002c
:10331000048242000402e90004003700a553800043
:1033200094538000048252000402e90004007800f3
:103330000080fa00000006000400fa002047980010
:10334000314798002e429000e14f520002003600b3
:103350000002eb00440037002e409000a8fd07005b
:103360002e409000cdff070000027800040f780087
:103370001e027800e00f520002003a000002eb004b
:10338000390037001e027800e10f520002003a00b7
:103390002e409000aeff070025548000041020004e
:1033a00004826200e00f520009003a007553800069
:1033b00064538000048252000402d1009e0f520028
:1033c000030039002e409000a1ff0700850aa800e5
:1033d000e303470085a820009542780096538000bb
:1033e0001400200013c0b300070178008540780066
:1033f00006007800340f0700945380000402e800b0
:10340000945388009553800074538000848f520039
:103410000200390064538000945388001e02780033
:10342000e10f520003003a002e40900088ff070091
:103430000c00370025548000040220000482620042
:10344000e00f520007003a0084aaa800f28b0200a5
:10345000000000000002be00040278006902420081
:10346000f453880014002000040078000080fa0063
:10347000000006000c00fa00604798004107980021
:10348000520798000002eb00140798006e4290006b
:10349000e14f5200020036000002eb0061003700ed
:1034a0006e40900056fd07006e4090007bff0700c5
:1034b00000027800240798002e029000e00f5200ce
:1034c00004003a006e40900061ff07000002eb002c
:1034d000540037002e029000040f7800ae029000d6
:1034e0005e029000848f5200020036005e0290005f
:1034f000040f78002554800004102000048262002c
:10350000e00f52000a003a007553800064538000b7
:10351000048252008402d1002e029000848f520057
:10352000030039006e40900049ff0700850aa8009b
:10353000945380009e02420074538000848f520096
:1035400016003900755380009453800004825200a5
:1035500014079800ce03900085a8200095427800bb
:10356000965380001e02900013c0b300070178003c
:103570008540780006007800d30e0700ce02900048
:103580001e02900004824200440798001e02900030
:103590001e0f12006453800094538800ce039000e5
:1035a00085a8200095427800965380001e0278007e
:1035b00013c0b3000701780085407800060078004a
:1035c000c10e0700945380001e02420094538800ed
:1035d000ae0290005e029000848f520003003e0015
:1035e0006e4090001aff07000c0037002554800041
:1035f0000402200004826200e00f520007003a003b
:1036000084aaa800f28b0200000000000002be00a5
:103610000402780069024200f45388001e02900000
:103620001e024200040078000080fa00000006003c
:103630000400fa00004f7800110798001e02900065
:1036400004007800160c0200000000000002780060
:10365000040178009e0090001e40780085ff07005e
:10366000000278009e02900004824200040078006c
:103670000080fa00000006000600fa0040479800ab
:103680004e429000e14f5200020036000002eb0073
:103690000c0037004e409000d9fc070075538000a5
:1036a0006453800004825200040fe9004e409000f1
:1036b000fafe070000027800140798001e0290002e
:1036c0001e021200040078000080fa0000000600cc
:1036d0000200fa00004f78001e4078000c0007003e
:1036e00000027800e00f5200070032001e40780010
:1036f000c3fc0700b4538000c453880011c0b3005a
:1037000000c1b300630507000080fa000000060056
:103710000200fa00004f78001e427800e14f52008c
:10372000020036000002eb00120037001e40780055
:10373000b3fc0700b5538000c4538000848f52004f
:1037400004003900b5538000c45380000482520045
:103750000800370085538000c453800084825200e3
:10376000b653800074538000040253000482420068
:103770000402e800040078000080fa00000006005f
:103780000600fa0020479800210798002e4090007c
:10379000dfff070000027800040f78001e027800a7
:1037a000e00f520002003a000002eb002a0037004e
:1037b0002e40900092fc07002e029000e00f520075
:1037c0000a00320085a8200095427800c753800087
:1037d0002e03900014002000854178000701780036
:1037e00011c0b30006007800370e0700c4538000f4
:1037f0000402e800c4538800c5538000845380004d
:10380000848f52000200360074538000c453880035
:103810001e027800e10f520002003a00854aa8001b
:103820000c0037002554800004022000048262004e
:10383000e00f520007003a0084aaa800f28b0200b1
:10384000000000000002be00040278000403b00083
:10385000f453880014002000040078000080fa006f
:10386000000006000a00fa0040479800310798005f
:10387000420798000002eb00040f78004e409000d1
:10388000a3ff070000027800140798001e029000b2
:10389000e00f520002003a000002eb005000370037
:1038a0004e40900056fc0700ce0290001e02900091
:1038b000848f5200020036001e02900044079800d8
:1038c000c55380004e0290008482420084538000e1
:1038d000848f52001900360085538000c453800045
:1038e00004825200040fe8003e029000e00f5200f4
:1038f0000d00320085a8200095427800c753800053
:103900003e0390001e027800854178000701780090
:1039100011c0b30006007800eb0d07003e029000d6
:103920001e024200340798004e0290001e02520010
:103930004407980074538000c45388003e029000ee
:10394000e00f52000a00320085a82000954278005e
:10395000c75380003e0390004e02900085417800de
:103960000701780011c0b30006007800d60d0700eb
:10397000c55380004e02900004824200c453880068
:103980004e0290001e024200440798009e029000e2
:103990004e029000848252004e029000848f5200aa
:1039a00002003e00854aa8000c0037002554800024
:1039b0000402200004826200e00f520007003a0077
:1039c00084aaa800f28b0200000000000002be00e2
:1039d000040278000403b000f45388004e02900003
:1039e000040078000080fa00000006000600fa00db
:1039f000404798004e429000e14f520002003600ce
:103a00000002eb000b0037004e409000fcfb07006b
:103a10008553800074538000048f52004e40900004
:103a20003bff070000027800140798001e02900078
:103a30001e021200040078000080fa000000060058
:103a40000e00fa006047980041079800520798005e
:103a5000630798006e429000e14f520003003e0061
:103a60005e029000e00f520002003a000002eb00fc
:103a7000450037006e409000e1fb07006e4090006b
:103a800023ff07000002780014079800ee02900060
:103a90005e029000848242001e029000848f5200d9
:103aa000040036009e0290006e02900004825200d4
:103ab00054079800c55380006e029000048f4200a6
:103ac000845380009e0f5200050031008553800012
:103ad00074538000048252000482ea001e0f4200e8
:103ae000845380001e0252000402e800240798005c
:103af000de0290002e029000848f52000a003e00e9
:103b000085a82000954278004e0390005e02900048
:103b1000854178001e01780011c0b30006007800ce
:103b2000690d07001700370085a82000954278002e
:103b30004e0390002e029000854178001e0178000f
:103b400011c0b300060078005f0d0700de02900090
:103b50002e0290000482520085a820009542780031
:103b6000775380004e0090002e0390000603400023
:103b7000854178000701780011c0b3000600780085
:103b8000510d07005e029000040078000080fa00ea
:103b9000000006000600fa00204798002107980060
:103ba000ae019000120020008e0078002e409000a0
:103bb000a3ff07001e427800044078000080fa004e
:103bc000000006003e00fa0020779800211f9800b0
:103bd000321f9800431f9800541f9800651f9800db
:103be0002e729000e14f520003003e003e1a9000fa
:103bf000e00f520002003a000002eb0026013700fd
:103c00002e7090007efb07002e709000c0fe070013
:103c100000027800ce1a90000502520014079800a6
:103c20009e0290003e1a9000848f520002003100e4
:103c30000082eb00180137005e1a9000e00f52007e
:103c4000060032009e0290005e1a9000848f52009f
:103c5000020036005e1a900014079800c5538000d9
:103c60004e1a900004824200340798008553800069
:103c70003e029000848f520007003100855380007f
:103c800074538000048252000482ea00be02900055
:103c90000482420034079800be029000050f7800ad
:103ca000855380003e029000048252000402e80026
:103cb000240798004e1a900034079800be1a90000e
:103cc000750798002e1a9000040f98002e1a900085
:103cd00094427800154f98002e1a90000402e800d4
:103ce000241f98000002eb00640798006e1a9000f1
:103cf000e00f52000c0032009e4a900004c6b30050
:103d000084cf5200080036009e4a9000a4c7b3003a
:103d100084cf520004003e009e4a900004ceb300bf
:103d200004c24200144f980004c2b300244f98000c
:103d30002e4a90008482fb002e029000848f520055
:103d4000020036002e029000244f98002e4a900068
:103d50008482fb001e029000848f52000200360015
:103d60001e029000244f98002e4a90000482fb000f
:103d700085a82000954278007203470085417800ad
:103d80001e01780011c0b30006007800ce0c0700b9
:103d90002e4a90000482fb001e0f42002e4a900023
:103da0000482fb00ae0290000482520024079800b7
:103db0002e029000e00f520004003a00745380007d
:103dc000040f78000082eb00240798006e1a900020
:103dd000e00f5200680032000042eb00044f9800f0
:103de000600037000e4a90000482fb000402470086
:103df000a452900004c6b30084cf520011003600d4
:103e00000e4a90000482fb0004024700a452900076
:103e1000a4c7b30084cf52000a003e000e4a9000af
:103e20000483fb000e4a90000482fb00040247005a
:103e3000a452900004ceb30004c2420086024700a0
:103e4000a45298000e4a90000482fb00040247002e
:103e5000a45290001e4a900084cf520023003a00e2
:103e60003e1a90000402e900341f98003e1a9000a8
:103e7000e00f520008003a00be0290007e0290005f
:103e8000848252000e4a90000482fb0004824200a9
:103e90000402e800800037002e1a90009442780057
:103ea000154f98002e1a90000402e800241f980075
:103eb00014002000640798009e4a900004c6b300d6
:103ec00084cf5200240036009e4a9000a4c7b3005d
:103ed00084cf520020003e009e4a900004ceb300e2
:103ee00004c24200144f98001b0037007e0290006d
:103ef000341f98006e029000e00f5200160032004e
:103f00008e0a9000251f98002e1a90009442780087
:103f1000154f98002e1a90000402e800241f980004
:103f20009e4a900004c6b30084cf520008003600b9
:103f30009e4a9000a4c7b30084cf520004003e0004
:103f40009e4a900004ceb30004c24200144f980071
:103f50000002eb00640798000e4a90000442e8005b
:103f6000044f98008e4a90002e4a900084cf520051
:103f70009cff3900370037000042eb00044f9800e7
:103f8000300037000e4a90000482fb000402470014
:103f9000a45290001e4a900084cf520017003a00ad
:103fa0003e1a90000402e900341f98003e1a900067
:103fb000e00f520008003a00be0290007e0290001e
:103fc000848252000e4a90000482fb000482420068
:103fd0000402e800300037002e1a90009442780066
:103fe000154f98002e1a90000402e800241f980034
:103ff00014002000640798000f0037007e02900034
:10400000341f98006e029000e00f52000a00320048
:104010008e0a9000251f98002e1a90009442780076
:10402000154f98002e1a90000402e800241f9800f3
:104030000002eb00640798000e4a90000442e8007a
:10404000044f98008e4a90002e4a900084cf520070
:10405000ccff39002e4a90000482fb009e029000a3
:1040600004825200140798009e0290003e1a9000ad
:10407000848f5200020031000082eb0006003700fe
:104080002e4a90000482fb00be029000048242008f
:104090003407980024ff3700040078000080fa00fd
:1040a000000006000800fa00004f78001147980051
:1040b0001207980023079800340798000e03e800c1
:1040c000be0290002e0290009e019000120020007f
:1040d000860078001e407800bafe070000027800d3
:1040e000040078000080fa00000006000e00fa00cc
:1040f000881f78000042eb00044f78003c02370034
:104100001e4078003efa07000042eb00644798002a
:104110000002eb00140798000002eb00240798004f
:10412000255480000420200004826200e00f520029
:1041300005003a00255480000440200004826200fb
:10414000e00f52000c0032006c3a02000000000048
:1041500000027800e00f52000700320004c1b300f3
:1041600064479800245480004a22de0061426200c5
:104170000482fb00140798002554800004022000ec
:1041800004826200e00f52000a003200f8538000ff
:10419000f28b0200000000000002be000402780062
:1041a00004025400e00f520002003c0004c1b300be
:1041b00064479800255480000404200004826200b3
:1041c000e00f52000a00320008548000f28b020017
:1041d000000000000002be00040278000402540047
:1041e000e00f520002003c0004c1b3006447980095
:1041f00014548000eb0f52000c003a000854800069
:10420000f28b0200000000000002be0004027800f1
:1042100004025400e00f520004003c0014c1b3003b
:1042200064479800c400200014548800145480008f
:10423000e40f520064003a000002eb0044079800cb
:104240005c0037004e0290007422b900040278002e
:10425000f002420004a3200004824200140278000d
:10426000e00f5200570032004e0290007422b90055
:1042700004027800f002420004a3200004824200fd
:104280009402780034548000848f520046003a0033
:1042900007fa07004e0290007422b90084027800e9
:1042a00004a3200004824200a200200084007800c1
:1042b000e0a12000d80b0200000000004e02900098
:1042c0007422b90004027800ea02420004a320002c
:1042d0000482420014027800b45088004e0290001c
:1042e0007422b90004027800ec02420004a320000a
:1042f000048242001402be0061024200e0824a00d1
:10430000845088009550880005518000f45080004a
:1043100084824200b450800084824200c4508000f5
:1043200004826a003454880024c1b30064479800b2
:104330006400200014548800ce029000c4fe2f00b8
:1043400004aab90004027800870220008483430095
:104350004e0290000402e8007422b9008402780042
:1043600004a3200004824200040378004e0290005f
:104370007422b9008402780004a320000482420061
:10438000840278000702780013c0b30006017800a9
:1043900011c0b300050078004b0b07000002eb00d2
:1043a00044538800080037004e0290000402e800e1
:1043b000440798004e029000e20f5200a1ff360021
:1043c00001003700000000006e429000e04f5200f4
:1043d000090032001e02900004f0a7000402ea0067
:1043e0000402e9004f22de00044278008440780095
:1043f0006e40900027020700245480007002620083
:10440000e00f52002d003a0014548000e70f5200d4
:104410006f013a00e48b0200000000000003be00c0
:10442000d4538000e55380000402530085825b0072
:10443000e00f5200e08f5a006701350024548000dd
:1044400067026200e60f52000e003a00245480001a
:104450004322de0061426200644798001e407800fb
:1044600008fb07001e40780006fb07006e42900024
:10447000e04f52005a013a00e40020001454880032
:104480005a0137008af9070021c0b30000c1b30008
:1044900000020700e48b0200000000000003be00e1
:1044a00084962800950020000602420087824a0078
:1044b000d4538800e55388004c013700e48b020098
:1044c000000000000003be00d4538000e5538000cc
:1044d0000402530085825b00e00f5200e08f5a0017
:1044e0004101350072f907001454800005002000d6
:1044f000c600200007002000860f5200878f5a0058
:10450000ef003e00046001000c0037002600370079
:10451000530037005d003700eb003700860037009e
:1045200095003700a9003700b6003700c3003700f8
:10453000c7003700a5003700d30037000c5a02002f
:104540000000000000027800e00f5200e00032009e
:10455000140020001454880054518000640262004a
:10456000e00f520008003200f45080000551800036
:104570000402780011c0b30004007800585a020009
:1045800000000000d9003700f45080000551800081
:104590000402780011c0b30004007800585a0200e9
:1045a00000000000d10037006a02470004007800d4
:1045b0008a5a02000000000000027800e00f52005a
:1045c000c5003200265a02000000000000027800f8
:1045d000e00f5200160032005e029000ee029000e2
:1045e000f4508800055188002400200014548800ed
:1045f00005518000f450800084824200b450800055
:1046000084824200c450800004826a0034548800ce
:104610000042eb00044078002eeab700d4032000eb
:10462000050020004450880055508800af00370036
:10463000e48b0200000000000003be008496280006
:10464000950020000602420087824a00d453880069
:10465000e55388000002eb0014548800a3003700e3
:10466000f28b0200000000000002be00040278008d
:10467000f4538800e0a120009a7c020000000000b2
:1046800034002000145488009800370021a2200034
:10469000e0a120005c7d0200000000000002780024
:1046a000e00f52001d003a00f28b020000000000f3
:1046b0000002be0084027800f4538000048352009c
:1046c000445080005550800004027800840f53004d
:1046d00083003600e4a2200014427800e54f520027
:1046e0000b003e00e4a22000144278000442e800df
:1046f000044078002eeab7004450800055508000f6
:104700000402420085824a004450880055508800c7
:1047100024002000145488007400370024c0b30023
:10472000644798000002eb00140798005400200032
:10473000145488006d00370024c0b300644798000b
:104740001400200014079800e4a22000144278000e
:10475000e34f52006400360044c0b30004407800c8
:104760002eeab70004242400f500200044508800fd
:10477000555088005d003700e4a220001442780004
:10478000e14f520005003e0024c1b3006447980089
:1047900014002000140798005400370024548000af
:1047a00068026200e00f52000500320044c1b3000d
:1047b0006447980014002000240798004b0037003d
:1047c00024c0b3006447980048003700e4a22000ea
:1047d00014427800e44f520005003e0004c1b300cb
:1047e0006447980014002000140798003f00370029
:1047f000840020001454880014c1b300644798005a
:104800003a003700e4a2200014427800e44f52003e
:1048100005003e0014c1b300644798001400200056
:10482000140798003100370044c1b3006447980072
:1048300014002000240798002c00370044c1b30066
:1048400064479800140020002407980027003700d0
:10485000e4a2200014427800e44f520005003e001c
:1048600004c1b300644798001400200014079800a6
:104870001e00370044c1b3006447980014002000b4
:104880002407980019003700e4a2200014427800a1
:10489000e44f520005003e0014c1b3006447980085
:1048a00014002000140798001000370044c1b30022
:1048b0006447980014002000240798000b0037007c
:1048c000000000000900370000000000070037006a
:1048d0000000000005003700000000000300370062
:1048e0000000000001003700000000006e42900050
:1048f000e04f5200310032001e029000e00f5200e3
:104900002b003200e4a22000144278000442e800a8
:10491000044078002eeab7004450800055508000d3
:104920000402420085824a004450880055508800a5
:10493000a5508000a45380000482520044079800d0
:10494000a5508000a4538000848f520006003100df
:10495000755380006453800004825200ce029000a0
:10496000048242004407980066508000775080001f
:104970004e029000050020000402530085825b0077
:104980006450880075508800d55080004e02900019
:1049900004824200d4508800a4538000a4508800b0
:1049a0008040eb006e409000ba0007000300370023
:1049b00011c0b3006e409000b60007002e029000b8
:1049c000e00f520009003200fe0307000700370025
:1049d0000000000005003700000000000300370061
:1049e0000000000001003700000000001e4fe8003a
:1049f0001e427800e14f5200c1fd36000002eb007c
:104a000044079800390037004e0290007422b90024
:104a100004027800f002420004a320000482420055
:104a200014027800e00f520034003200f28b0200d2
:104a3000000000000002be00040378004e02900057
:104a40007422b90004027800f202420004a320009c
:104a5000048242001402780084025300c42d200016
:104a6000848f52001e003600ce029000c4fe2f003c
:104a700004aab9000402780087022000848343005e
:104a80004e0290000402e8007422b900840278000b
:104a900004a3200004824200040378004e02900028
:104aa0007422b9008402780004a32000048242002a
:104ab000840278000702780013c0b3000601780072
:104ac00011c0b300050078007f0907000002eb0069
:104ad000445388004e0290000402e9004407980005
:104ae0004e0290000402e800440798004e02900035
:104af000e20f5200c4ff3600010037000000000042
:104b00004f0478000080fa00000006002c00fa0034
:104b10003017980041179800521798003e139000e4
:104b2000164278000480fb00964390008783fb00c8
:104b3000c83bdd008083730007027800a643900025
:104b40008783fb00364390000683fb004833dd007b
:104b50000703730086027800340f9800450f980011
:104b60004e1290001403be00560f9800670f980075
:104b70000042eb00645f980064c0b300745f98006b
:104b8000de139000071798000e12900004007800c2
:104b9000726702000000000000027800041798000d
:104ba00076024700c100200004007800ee67020092
:104bb00000000000000278000482ea001417980048
:104bc0005e109000a43d020000000000000278008a
:104bd000241798009e1290002e129000848f52008d
:104be00004003200843a020000000000140020009b
:104bf000250037000000eb00c48702000000000021
:104c00000e82e8004101200004007800e23e02002c
:104c1000000000000e82e80004007800290307006d
:104c20007e0290004422de006f42620025002000d8
:104c30000522dd00744f52009e4278000582fb0081
:104c4000de12900004825200740252005417980041
:104c50000e82e800be10900004007800f301070007
:104c600000027800e00f5200040032000e82e800db
:104c7000de1090000400780001040700843a02006e
:104c80000000000014002000040078000080fa00fa
:104c9000000006002a00fa00006f9800116f9800cb
:104ca00083f707000e6a90000482fb006102620035
:104cb00004427800e04f520005003200856aa800e7
:104cc0008e6a9000e4cfb30004c26200046f9800c3
:104cd00084aaa90084caa90084eaa900852aa90097
:104ce000854aa900850aa900000000006c3a02006c
:104cf0000000000000027800e00f5200fbff3200cd
:104d00000e6a90000482fb0066026200e00f52000f
:104d1000030032000002eb00040f78007600370039
:104d200095538000a4508000848f520003003a0005
:104d30000002eb00040f78006100370095538000fb
:104d4000a4508000848f52001b00360095538000d1
:104d5000a4508000048f5200d45080009e0f520057
:104d600002003100d0508000000f780064518000b4
:104d70009e0f52000300310064518000040f780040
:104d8000854aa80085a8200095427800a65080009a
:104d90001e02780085417800060178008040eb0013
:104da00060032000c8080700a45080001e024200d3
:104db000a45088004200370075538000a450800042
:104dc0000482520034179800be1290009453800061
:104dd0008482420064538000048f5200d4508000cb
:104de0009e0f520002003100d5508000050f780060
:104df000645180009e0f520003003100605180001a
:104e0000000f7800854aa8003e1290009e0f5200c5
:104e1000020036001e027800341798003e129000ff
:104e200085a8200095427800a65080008541780032
:104e3000060178008040eb0060032000a208070014
:104e40003e1290001e021200341798003e1290008d
:104e5000e00f52000d0032003e12900085a82000a5
:104e6000954278006753800070538000a650800000
:104e7000060350006603b000854178000701780002
:104e80008040eb00060078008f080700a4508000e7
:104e90001e024200a4508800a55080007453800078
:104ea000848f520006003900a550800066538000b0
:104eb000745380000402530004824200a45088000e
:104ec000255480000480200004826200e00f52001c
:104ed00009003200d45080009e0f520006003200bc
:104ee000645180009e0f5200030032000e6a900051
:104ef0000404a000046f98001e027800e00f520026
:104f000005003a000e6a90000482fb006302620012
:104f1000e00f520021003200d45080001e025200e7
:104f2000d45088001e027800e00f520003003200c7
:104f30000e6a90000434a000046f98001e6a90006e
:104f40000482fb006102620004427800e04f5200dc
:104f5000070032000042eb00044078002eeab70060
:104f600044422f000500200044508800555088001e
:104f7000e48b0200000000000003be0044508000eb
:104f8000555080000602420087824a00d4538800b0
:104f9000e5538800848aa8003a0037001e6a900012
:104fa0000482fb0062026200e00f52001400320033
:104fb00024548000674262000442e80067426200b5
:104fc0000482fb00670262002654800085ff2f00e8
:104fd00085026300048272002454880064508000bb
:104fe0007550800061025200e0825a0064508800cf
:104ff0007550880014002000040f7800210037004d
:105000002454800070026200e00f52001d00320044
:105010001e6a90000482fb0061026200e00f5200f1
:105020000f003a00e4a2200014427800e04f520042
:105030000b003200e4a22000144278000442e90090
:10504000044078002eeab70044508000555080009c
:105050008502d1000482d300445088005550880056
:10506000e48b0200000000000003be0044508000fa
:10507000555080000602420087824a00d4538800bf
:10508000e5538800c450800024079800b450800085
:1050900034079800645080007550800044079800e1
:1050a0005507980084508000955080006407980050
:1050b000750798000e0a900004e0a10004f0a1001a
:1050c000040f98000e0a90000400a1000410a10033
:1050d0000420a1000430a100040f98000e6a900083
:1050e000145798000002eb00340f980066508000bf
:1050f000775080001e027800050020000602420062
:1051000087824a0064508800755088000e6a9000bb
:105110000482fb0062026200e00f52001a003200bb
:105120000e6a90000482fb0070026200e00f5200e1
:1051300003003a006022b8006407980075079800e1
:105140005451800062026200e00f520007003200fa
:105150004e029000de02900061025200e0825a008e
:1051600044079800550798000700370064508000f6
:105170007550800061024200e0824a00645088005d
:10518000755088002a2aa8000e6a90000482fb004d
:105190006102620004427800e04f520001003200d8
:1051a0002a0aa800b5538000c4538000848f52009f
:1051b00009003900855380007453800084825200b6
:1051c000c6538000b453800004025300048242009e
:1051d000140f980005003700c5538000b4538000b9
:1051e000048252000402e900140f9800b63a02004b
:1051f0000000000000027800140798009e02900052
:10520000f4032000848f520003003e000002eb00f4
:1052100014079800030037001e0290000404b10038
:10522000140798009e0a90001e029000848f52007e
:10523000020036001e029000140f9800640247001e
:10524000040078009f0107009e027800748f4200de
:105250000e0a90000440a0000450a1000460a000c9
:105260000470a100040f98000e6a90000482fb00f5
:1052700062026200e00f5200150032001e0078004a
:10528000640f400024c0b300045f980044c0b30022
:10529000145f980024802100540f98000e0a90009b
:1052a0004422de006f4262000442e8006f42620066
:1052b0000482fb006f0262004422dd000e0b9000ae
:1052c000f5f02f008502630004827200040f98003d
:1052d000e6ad2000164378008683fb00f6ad200083
:1052e000164378000683fb004833dd000703730094
:1052f0000602780006ae2000164378008683fb0085
:1053000016ae2000164378000683fb004833dd000c
:105310000703730086027800640f9800750f9800e9
:10532000f45080000551800004179800151798006c
:105330000042eb004467980064c0b30054679800d3
:105340009e027800351798003e1290000400780005
:105350007267020000000000000278003417980015
:105360007c024700c100200004007800ee670200c4
:1053700000000000000278000482ea00240f980078
:10538000e0002000f03c0200000000001e01780058
:1053900061c0b300e0a120001287020000000000fd
:1053a0006402470041012000040078002c3f020005
:1053b000000000000e6a90000482fb00620262009e
:1053c000e00f520005003200780247004100200043
:1053d000040078002c3f02000000000020022000a2
:1053e0000a3d0200000000001e007800a43d0200fb
:1053f000000000000002780014079800200320003d
:10540000f03c0200000000000e82e80021002000b5
:10541000040078002c3f020000000000703c0200f5
:10542000000000000080fa00000006000a00fa00f8
:1054300030079800410798003e0290001402900047
:10544000e00f520002003a000002eb001a013700a0
:10545000e4cfb30014479800ce029000254290009c
:105460000483fb00354290000482fb004822dd00eb
:1054700006027200840278004e0290009443780085
:105480000783fb00144290000482fb004822dd00e9
:1054900006027200848242003e02900014027800ec
:1054a000848242003e0290001402900004826a004e
:1054b000240798000042eb00044f78003b003700bf
:1054c0001e4078004ef5070014548000ed0f520086
:1054d0003000320014548000e40f520008003a00fb
:1054e000355480003e02900014029000848f5200d8
:1054f0002a003a001e427800144798002a0037001c
:10550000355480002e029000848f520025003a000e
:1055100067f507003e02900094029000c45080009e
:10552000848f520020003a003e02900094027800de
:10553000b4508000848f52001b003a004e0390004c
:10554000964378000780fb00964390008783fb001a
:10555000c83bdd008083730007027800a6439000fb
:105560008783fb00364390000683fb004833dd0051
:105570000703730086027800f65080000751800010
:10558000860f5200878f5a0007003a00140020004f
:10559000c9003700000000000300370000000000d1
:1055a00001003700000000001e4fe8001e42780096
:1055b000e14f5200c2ff36001e429000e24f42000f
:1055c000170032001e4090000df5070038f5070067
:1055d0001e429000e24f4200110032002e02900065
:1055e00034548800a2002000ce009000e0a12000ea
:1055f000d80b0200000000003e0290001402780068
:10560000b45088003e02900014029000c4508800fc
:1056100064538000a450880014002000a6003700c6
:105620003e029000e4029000042020000482620008
:10563000e00f520002003a000002eb009e0037002b
:1056400044538000e00f5200020032000002eb00e1
:10565000990037000002eb00140798004b00370058
:105660001e0290007422b90004027800f002420089
:1056700004a320000482420014027800e00f5200cc
:10568000460032001e0290007422b9000402780025
:10569000f002420004a32000048242009402780039
:1056a0003e02900014029000848f52002f003a00b6
:1056b0001e0290007422b90004027800ea0242003f
:1056c00004a3200004824200940278003e0290006d
:1056d00014027800848f520026003a001e029000c7
:1056e0007422b9008402780004a3200004824200de
:1056f0001403be004e009000104278000481fb00ad
:10570000904090008180fb00c808dd00828070001e
:1057100001027800a04090008180fb0030409000a2
:105720000080fb004800dd0001007000800278006e
:10573000840f5300858f5b0010003a00f28b02004b
:10574000000000000002be00040378001e0290006a
:105750007422b9008402780024a42000048242004c
:10576000060a78000002eb0053003700000000003a
:1057700003003700000000000100370000000000b7
:105780001e0290000402e800140798001e02900018
:10579000e20f5200b2ff36000100370000000000a7
:1057a0000042eb00044f78003f0037001e407800b5
:1057b00093f407002454800068026200e00f520056
:1057c00035003200baf40700c55080003e02900058
:1057d00014029000848f520031003a001e029000a3
:1057e0007422b9008402780004a3200004824200dd
:1057f000a2002000ce00900004007800d80b020028
:10580000000000003e029000140378001e02900089
:105810007422b90084027800a4a32000048242000c
:10582000060a78003e029000b40290002402900024
:105830001e0390007433b90086037800c6a32000cd
:1058400006834300048bbe003e02900014039000c8
:105850001e0290007422b9008402780004a4200083
:1058600004824200060a7800f28b02000000000069
:105870000002be00040378001e0290007422b900ea
:105880008402780024a4200004824200060a7800e2
:105890000002eb00080037000000000001003700a4
:1058a000000000001e4fe8001e427800e14f520049
:1058b000beff36000002eb00040078000080fa0012
:1058c000000006000200fa00000f78001e027800b7
:1058d00014027800040078007267020000000000e3
:1058e000000278009e027800840a78001e02780088
:1058f00014029000040078007267020000000000ab
:10590000000278009e027800940298001e0278003f
:10591000b4029000240290000400be008e670200d2
:10592000000000000002be001e037800240398005f
:10593000350398001e027800d402900044029000c3
:105940000400be008e670200000000000002be00de
:105950001e03780044039800550398001e02780047
:1059600074029000040078007267020000000000da
:10597000000278009e027800f40298001e0278006f
:10598000040a900004007800726702000000000022
:10599000000278009e027800840a98001e027800b7
:1059a000140a9000040078007267020000000000f2
:1059b000000278009e027800940a98000080fa00a5
:1059c000000006000000fa00881f780038f4070085
:1059d000c45080003454880064538000945388007d
:1059e00064538000a453880074538000b45388002b
:1059f00074538000c45388002454800068026200fd
:105a0000e00f520002003200440020000100370085
:105a1000d400200014548800840aa900842aa90014
:105a2000844aa900848aa90084aaa90084caa9007a
:105a300084eaa900850aa900852aa900854aa90047
:105a4000856aa900858aa8002a0aa9002a2aa9002d
:105a50002a6aa9002a8aa90064538000a4508800f9
:105a6000c8a02000b8620200000000000002780018
:105a7000040c7800c8a02000b862020000000000fa
:105a800000027800140498000082eb004451880062
:105a900014002000d45088004f0478000080fa00e1
:105aa000000006000400fa00881f7800c0002000f3
:105ab000c487020000000000d03e02000000000089
:105ac00000427800044f78001e4278008482fb0078
:105ad000040f20000482620042a2de00044278002b
:105ae000744f52001e427800e04f520002003a000c
:105af000842120005e003700710020000000eb00d0
:105b0000e23e02000000000046003700d03e0200e6
:105b10000000000000427800144798001e429000e8
:105b2000e04f5200480032001e429000e14f520008
:105b30003b0032001e429000e24f520023003a0028
:105b40001e427800e24f5200410036000002eb0096
:105b500014079800d03e02000000000000427800c8
:105b6000144798001e429000e44f52000b003a0088
:105b70000e82e8000404e800d03e020000000000ad
:105b800000427800044c78000e84e800d03e020009
:105b90000000000000427800044c78009e02900053
:105ba00074212000848f52002b0036009e0290004a
:105bb000445b2000848f520002003600445b2000ca
:105bc0002b0037001e029000290037001e4278008b
:105bd000e14f520022003600d03e020000000000db
:105be00000427800144798001e4290009e427800c0
:105bf00084cf52001c0039001e4290000482fb003a
:105c0000840078000000eb00e23e0200000000008b
:105c10009e4278001e42900004cf520001003700df
:105c2000000000009e4278000582fb000402ea00aa
:105c30004f22de00044278001e4fe900e04f520080
:105c4000b2ff3a00090037000000000007003700eb
:105c500000000000050037000000000003003700ce
:105c60000000000001003700000000008421200037
:105c7000040078004f0478000080fa00000006005d
:105c80002200fa00700f9800011798007e0a900019
:105c9000d44a9000055798007e0a90004403900073
:105ca000d403900046079800570798007e0a90009a
:105cb00024039000b4039000160f9800270f98005b
:105cc000840aa900842aa900844aa90024548000d7
:105cd00070026200e00f520009003a00e48b0200fb
:105ce000000000000003be008496280095002000fc
:105cf0000602420087824a00d4538800e553880098
:105d000014548000e40f520003003200e50f5200eb
:105d10002c003200780037000e5290000482fb0005
:105d200064026200e00f52000200320025ff07000b
:105d30002e0437000e5290000482fb0070026200b5
:105d4000e00f5200090032004e029000de02900087
:105d500064508800755088008040eb0040c0b3005c
:105d6000ccfb070017ff0700200437000e529000fd
:105d70000482fb0062026200e00f52000f0032005a
:105d80001e0a9000ae0a900061024200e0824a00c2
:105d9000845088009550880042ff07000002780078
:105da0006451880011c0b30020c1b300b9fb0700e3
:105db00064002000145488000c04370001ff070021
:105dc0000a0437000e5290000482fb006402620055
:105dd000e00f5200f2033a000e5290000482fb00e2
:105de00070026200e00f520017003200665080001f
:105df000775080004e029000de029000840f530026
:105e0000858f5b0010003200665080007750800064
:105e1000160f9800270f98004e029000de029000a7
:105e2000645088007550880011c0b30040c0b300b2
:105e300098fb07001e0b9000ae0b90006650880088
:105e400077508800e90337000e5290000482fb006f
:105e500062026200e00f5200d30332001e0a90007b
:105e6000ae0a900061024200e0824a00845088003d
:105e7000955088007e0a900074029000d4508800eb
:105e800008ff070000027800645188000e5290005d
:105e90000482fb0070026200e00f5200100032002a
:105ea00011c0b30000c1b3007afb070074002000ea
:105eb00014548800e48b0200000000000003be00c0
:105ec00084962800950020000602420087824a003e
:105ed000d4538800e5538800848aa900c30337009f
:105ee00011c0b30020c1b3006afb070064002000aa
:105ef00014548800bd0337008e1390006707980084
:105f00000e5290000482fb0061026200044278009d
:105f1000e04f5200030032006e0290000402e800dd
:105f2000640798000e5290000482fb006202620037
:105f3000e00f5200030032006e0290000402e800fd
:105f400064079800b5538000c4538000848f5200ca
:105f50000900390085538000745380008482520008
:105f6000c6538000b45380000402530004824200f0
:105f70003407980005003700c5538000b4538000f3
:105f8000048252000402e900340798008450800023
:105f9000955080001e0b9000ae0b90000402530041
:105fa00085825b00340f9800450f98003e0a9000f0
:105fb000540f98000002eb00740798006e029000e6
:105fc000e00f5200350032003e029000e00f520018
:105fd000480032003e0a9000ce0a9000e00f5200c6
:105fe000e08f5a000a0035003e0290006123b8009d
:105ff0003e0a9000ce0a9000840f5300858f5b000c
:1060000003003600140020007407980014003700c5
:106010006e0290006123b8003e0a9000ce0a900004
:106020000602420087824a00e00f5200e08f5a00c9
:106030000b003400be0290006e02900004825200f9
:106040006123b9003e0a9000ce0a9000840f5300ed
:10605000858f5b0002003500140020007407980053
:106060003e0290006123b8003e0a9000ce0a9000e4
:10607000840f5300858f5b001e003400de0a900001
:106080006e02900004824200e00f520019003400ba
:106090001400200074079800160037003e0a900094
:1060a000ce0a9000e00f5200e08f5a0003003a0041
:1060b00014002000740798000e0037003e0a90007c
:1060c000ce0a9000e00f5200e08f5a000900350020
:1060d0003e0290006123b8003e0a9000ce0a900074
:1060e000840f5300858f5b000200360014002000ef
:1060f000740798007e029000e00f520009003a00f9
:106100000e5290000482fb0064026200e00f520015
:1061100027033a0011c0b30000c1b300ddfa070045
:10612000320337000e5290000482fb0066026200c8
:10613000e00f52000200320022fe07002b0337005e
:106140000e5290000482fb0070026200e00f5200c9
:1061500019033200145480006123b800a4ff2f00fb
:10616000f5ff2f000602420087824a0066002000e9
:1061700007002000860f5200878f5a005b013e0007
:1061800004600100060037001e0037001d003700c4
:106190001c0037001b0037001a0037004801370089
:1061a00066508000775080004e029000de02900022
:1061b000840f5300858f5b00100032006650800012
:1061c00077508000160f9800270f98004e0290001d
:1061d000de029000645088007550880011c0b30042
:1061e00040c0b300abfa07001e0b9000ae0b90004e
:1061f0006650880077508800fc0237007400200049
:106200001454880095538000a450800004825200ea
:10621000240798002e029000e00f520006003d0077
:10622000755380006453800004825200ae029000d7
:106230000482420024079800665080007750800056
:106240002e02900005002000041f430005974b001c
:106250004e039000de0390001e02be0004025300b5
:1062600085825b00048fbe001e02be00e00f52005c
:10627000e08f5a0014003400545180006102620023
:10628000e00f5200060032001e03be001400200082
:1062900005002000840f5300858f5b00040032004e
:1062a0008040eb0000c1b3007afa0700cf0237004c
:1062b0004e029000de02900061025200e0825a001d
:1062c000440798005507980066508000775080007a
:1062d000a5508000a453800004825200cfa2de00ab
:1062e000041f530005975b00a5508000a453800055
:1062f000848f520006003100755380006453800083
:1063000004825200050020001e1f12001e971a0072
:106310004e029000de0290001e1f52001e975a008f
:106320001e02be00e00f5200e08f5a005000340001
:1063300075538000645380000482520005002000e1
:10634000be0f5200ae8f5a00490039002a6aa900d8
:106350002a8aa900850aa900a75380002707980068
:10636000a55380001e02780004824200a4538800d6
:10637000a55080002e029000848f52001100390039
:10638000a5508000a4538000848f52002300310068
:106390006650800077508000a5538000a450800094
:1063a00004825200050020000602420087824a0053
:1063b0006450880075508800a4538000a450880061
:1063c00016003700a550800076538000645380008b
:1063d000040253000482420024079800a553800061
:1063e0002e029000848f52000c0036006650800010
:1063f00077508000a55380002e0290000482520046
:10640000050020000602420087824a00645088008e
:1064100075508800a4538000a4508800a5538000c4
:1064200074538000848f520006003900a553800009
:1064300066538000745380000402530004824200bb
:10644000a4538800a550800074538000848f5200ac
:1064500030003900a55080006653800074538000de
:106460000402530004824200a4508800290037002f
:10647000a5538000a4508000848f52002500320074
:106480005451800068026200e00f52002000320088
:106490005451800070026200e00f52001b00320075
:1064a0006650800077508000a5508000a453800083
:1064b00004825200cfa2de000402530085825b00fa
:1064c0006450880075508800a5508000a453800057
:1064d000848f52000a00310066508000775080009f
:1064e000755380006453800004825200cfa2de0006
:1064f0000402530085825b00645088007550880058
:10650000a4538000a4508800854aa8002a8aa800c5
:106510002a6aa800a553800094538000848f5200fb
:106520001d003a002554800004802000048262008f
:10653000e00f52000b003a00e48b02000000000064
:106540000003be0084962800950020000602420049
:1065500087824a00d4538800e5538800848aa900c2
:106560000d00370066508000775080004e0290008a
:10657000de029000840f5300858f5b0006003a0016
:106580005451800061026200e00f520002003200ac
:10659000848aa900856aa9007e0a9000740390008d
:1065a000ce03900064508000755080000402780093
:1065b0000482530004024300640f9800d45080000a
:1065c000e00f520004003a006e0a9000e00f520003
:1065d00001003200852aa8006e0a9000d45088007d
:1065e00014548000e80f520018003a0066508000f2
:1065f000775080004e029000de029000840f53001e
:10660000858f5b003b003a005451800061026200bc
:10661000e00f520039003200e48b0200000000005d
:106620000003be00444b2c0045002000060242003f
:1066300087824a00d4538800e5538800848aa800e2
:106640009400200014548800310037001454800056
:10665000e90f52000e003a000e5290000482fb0037
:1066600061026200e00f520026003a004e039000e3
:10667000de03900066508800775088008040eb0071
:1066800040c1b30083f90700cefc0700d7013700f3
:1066900014548000ea0f52001c003a00665080003b
:1066a000775080004e029000de029000840f53006d
:1066b000858f5b00c2013a00c2fc0700cb013700a6
:1066c000645080007550800061034200e0834a00fe
:1066d0004e029000de029000840f5300858f5b0015
:1066e000b9013a00b7fc0700c00137000000000004
:1066f0000700370000000000050037000000000020
:106700000300370000000000010037000000000017
:106710000e5290008482fb0004022000048262007a
:10672000e00f5200aa013a0014548000eb0f52000f
:10673000a901320014548000ea0f5200a80132006f
:1067400014548000ec0f5200a70132000e1290008a
:10675000e00f5200220132005e0a9000e00f52006a
:1067600080003c007e0a9000640290004422de001b
:106770006f4262000482fb004222dd008402780046
:106780005e0a90000482520004007800c487020070
:10679000000000008e1290005e0a90000482420009
:1067a000041798008e1290003e029000848f5200d1
:1067b00002003600be039000071798008650800044
:1067c000975080000e129000050020000602420043
:1067d00087824a008450880095508800b553800015
:1067e0000e1290008482420084538000848f5200f5
:1067f0002000360085538000b4538000048252008c
:106800000402e8002407980085a82000954278003b
:10681000b65380002e0290008041eb000081eb0017
:106820008540780006007800270207008e1290004d
:106830002e0290000482520085a820009542780024
:10684000765380008041eb000081eb0085407800aa
:10685000060078001c020700755380000e1390009c
:106860002e0290000402530004824200b4538800b8
:106870000d00370085a8200095427800b6538000af
:106880000e1290008041eb000081eb008540780003
:10689000060078000c020700b55380000e1290002d
:1068a00004824200b453880044518000e10f42004a
:1068b000cb00320044518000840278000e12900018
:1068c0000482520044518800e55080004451800009
:1068d00004824200240798002e029000e00f52002c
:1068e00003003d000082eb0044518800bc003700eb
:1068f00044518000e00f5200b9003c0086508000f7
:10690000975080002e0290000500200006024200f1
:1069100087824a008450880095508800b5538000d3
:106920002e02900004824200b4538800b5538000c8
:1069300084538000848f520007003600b5538000d6
:106940008653800074538000040253000482ea00de
:1069500004824200b45388000082eb004451880056
:106960009f0037005e0a9000e00f52009c00340048
:106970008e1290005e0a9000848242003e029000d7
:10698000848f520004003600be0290005e0a900020
:1069900004825200041798007e0a9000640290005e
:1069a0004422de006f4262000482fb004222dd00ce
:1069b00004007800c487020000000000b553800086
:1069c0005e0a9000848242000e129000848242008f
:1069d00084538000848f520033003600855380003a
:1069e000b4538000848252005e0a90000402ea00e0
:1069f000048242000402e800240798002e0290005e
:106a0000e00f52001700350085a82000954278005d
:106a1000b65380005e0a9000040343002e029000eb
:106a20008041eb000081eb00854078000600780093
:106a3000a50107008e1290002e02900004825200e1
:106a400085a8200095427800765380008041eb00b5
:106a50000081eb0085407800060078009a0107006d
:106a60001c00370085a8200095427800b6538000ae
:106a70005e0a900004034300875380007453800033
:106a8000048253000482ea00040343000e129000c3
:106a90008041eb000081eb00854078000600780023
:106aa000890107000b00370085a820009542780077
:106ab000b65380005e0a9000040343000e1290005b
:106ac0008041eb000081eb008540780006007800f3
:106ad0007d01070044518000e10f420005003a00ab
:106ae0005e0a9000445188000e129000e450880025
:106af0003b00370044518000840278005e0a900019
:106b0000848f52001c003600de0a90000e129000a6
:106b1000848242004451800004037800e4508000e5
:106b200004024300848f520006003e00de0a9000fb
:106b30000e1290008482420044518000848f5200e3
:106b4000030031008e129000e550880007003700e6
:106b50004451800084027800e45080008482420026
:106b60005e0a900004825200e45088005e0a9000a1
:106b7000445188001a003700de0a90000e1290007f
:106b8000848242004451800004037800e450800075
:106b900004024300848f52001100360044518000eb
:106ba00084027800e4508000848242005e0a9000f3
:106bb000848f52000a003900e55080005e0b90007f
:106bc0000e1290000403430044518000040353005c
:106bd000e45080000402530004824200e450880024
:106be0006e029000e00f52001c003200145480002e
:106bf000e70f520002003200b4538000c4538800f3
:106c0000255480000408200004826200e00f520036
:106c10000500320011c0b30000c1b3001df8070029
:106c2000a3ef07000d00370084eaa8002554800078
:106c30000404200004826200e00f520007003a00c2
:106c400084caa800f28b0200000000000002be000f
:106c50000402780078024200045488000e5290002a
:106c60000482fb006102620004427800e04f52009f
:106c70005e00320084508000955080006103420025
:106c8000e0834a006e0290006120b8001e0a900066
:106c9000ae0a90000002420081824a00840f530035
:106ca000858f5b0051003a00845080009550800031
:106cb00061024200e0824a008450880095508800ba
:106cc000145480006123b800a4ff2f00f5ff2f00ab
:106cd0000602420087824a0036002000070020009a
:106ce000860f5200878f5a0028003e000460010082
:106cf0000300370008003700100037001e0037007f
:106d0000c40020001454880011c0b30010c1b300a7
:106d1000e0f7070035003700b40020001454880065
:106d2000f28b0200000000000002be0004027800a6
:106d30000403b0000454880015003700665080003a
:106d4000775080004e029000de029000840f5300c6
:106d5000858f5b0005003a008040eb0000c1b30066
:106d6000ccf7070017fb070020003700a400200025
:106d700014548800060037008040eb0000c1b300c7
:106d8000c4f707000ffb07001800370000000000e1
:106d900011c0b30000c1b300bef7070013003700f5
:106da0000000000011003700000000000f00370055
:106db000000000000d003700000000000b0037004d
:106dc0000000000009003700000000000700370045
:106dd000000000000500370000000000030037003d
:106de0000000000001003700000000000080fa00f1
:106df000000006000e00fa00604798004107980066
:106e000052079800434f98006e429000e14f5200a5
:106e1000020036000002eb00a80037006e40900030
:106e2000f7ee07004e029000e00f520002003a0019
:106e300014002000440798008553800064538000ac
:106e4000048252000402e90024079800ce02900058
:106e50005e029000848242002e029000848f5200d5
:106e6000020036000002eb009400370010ef07002c
:106e70004e4a90000482fb0063026200e00f520061
:106e800003003a004e4a90003440b300444f98004b
:106e90005e02900014079800ce0290005e029000ff
:106ea00004824200ae02900004825200240798003f
:106eb0004e4a90000482fb0062026200e00f520022
:106ec000100032004e4a90000482fb006102620012
:106ed00004427800e04f5200060032002e0290007b
:106ee0000402d1009e029000048242001407980020
:106ef000040037009e0290002e029000048242009f
:106f000014079800655380001e029000048242001e
:106f10000402e80024079800b4538000040f7800ae
:106f200044518000e10f42000d00320044518000c6
:106f300084027800e4508000048242001e0f420068
:106f4000845380009e0f520005003100855380005d
:106f500074538000048252000482ea001e0f420033
:106f6000c45380009e0f520010003100c5538000b2
:106f70002e029000848f5200230031004e4a900070
:106f80000482fb0064026200e00f52000200320043
:106f90000002eb00490037002e029000c453880025
:106fa0002e029000b453880017003700c4538000ad
:106fb0009e0f520010003600755380002e02900084
:106fc000848f5200100031004e4a90000482fb0072
:106fd00064026200e00f5200020032000002eb0087
:106fe000360037002e029000c45388002e02900015
:106ff000b4538800040037002e029000c453880068
:107000002e029000b4538800c45380009e0f52009b
:107010001b0036004e4a90000482fb0064026200ae
:10702000e00f520016003200745380001e0212005e
:1070300086a82000164378007753800085a820009a
:1070400095427800864178000701780085407800f5
:107050002e0090001c000700b5538000c453800030
:10706000848f520006003100b553800074538000b5
:107070002e0390000402530004824200b45388009f
:107080002e0290007453880064538000a45088003e
:1070900064538000a4538800645380009453880094
:1070a00014548000e70f520003003a0011c0b300ef
:1070b00000c1b300f7f607001400200004007800b8
:1070c0000080fa00000006000a00fa00000f7800b5
:1070d00021479800220798006347980044079800ca
:1070e0006e4290000482fb00e00f52001d0032004f
:1070f000e10f52003e003a002e4290000482fb0055
:10710000e00f52000a003200e10f520035003a0051
:10711000ae0290001e0278004e01900085007800bb
:1071200004007800d80b0200000000000c003700bb
:107130001e027800e10f4200030032001e007800ba
:10714000f03c0200000000002e029000ce009000f3
:10715000040078002c3f0200000000000000000046
:10716000230037002e4290000482fb00e00f520003
:107170000e003200e10f52001c003a002e02900077
:10718000e10f4200030032002e0090000a3d020091
:10719000000000001e027800ce009000040078007d
:1071a000e23e0200000000000c0037004e0190009b
:1071b000ae0090001e007800143e020000000000a7
:1071c000000000009a3e020000000000000278006b
:1071d000e00f5200fbff3200000000000000000042
:1071e000030037000000000001003700000000002d
:1071f0000080fa00000006000200fa00d922a80070
:10720000c662a900ca62a900d7c2a800d3c2a90059
:107210000042eb0004407800d2ebb7000002eb0024
:1072200004128800b4132000141288000002eb003e
:107230002412880004002800041288007c03070040
:10724000e4e92000b45e88000002eb00a45e880040
:10725000d80ba800d82ba900d84ba9008000eb00c0
:107260000000eb00ab050700e1e920004000200032
:10727000a8050700e1ff250060002000a505070024
:107280000100260060012000a20507001100260071
:10729000800120009f050700b4b020001442780050
:1072a000e04f520015003a00c4b0200014427800ac
:1072b000e44f520011003a00d5b02000954278000a
:1072c00034cab30084cf52000c003a00e4b020006e
:1072d00014427800e04f520008003a00f4b0200059
:1072e00014427800e04f520004003a0004b120003c
:1072f00014427800e04f520013003200b5b0200075
:1073000095427800c4b020001442780084c2720014
:10731000d4b020001442780084c27200e4b020008f
:107320001442780084c27200f4b020001442780045
:1073300084c2720004b120001442780004c27200ba
:10734000e04f520028003a004006200026050700c2
:1073500000027800040f78000e02780014427800d2
:10736000044078000bebb7000e0278000402e8003e
:1073700014427800044078000cebb700200620008f
:107380001905070000027800040f78000e0278004b
:1073900014427800044078000debb7000e0278002c
:1073a0000402e80014427800044078000eebb700b5
:1073b000000620000c05070000027800040f78008a
:1073c0000e02780014427800044078000febb700fa
:1073d0000e0278000402e8001442780004407800ad
:1073e00010ebb700270037008e027800b4b0200001
:1073f00014427800844a78000e0278008402e80083
:10740000c4b0200014427800844a78001e0278003c
:1074100084007800400620003e0507008e027800b8
:10742000d4b0200014427800844a78000e0278001c
:107430008402e800e4b0200014427800844a780016
:107440001e02780084007800200620003105070025
:107450008e027800f4b0200014427800844a78004c
:107460000e0278008402e80004b120001442780083
:10747000844a78001e02780084007800000620000c
:1074800024050700115e200040c0b300f00507008e
:1074900011002000e00120006a0507000080fa00ca
:1074a000000006000000fa00a0012000ce04070042
:1074b00000027800051020000502620004f0a70019
:1074c0000402ea000402ea004f22de000400780011
:1074d0000080fa00000006000000fa00e001200031
:1074e000c1040700000278006202620004f0a700f5
:1074f0000402ea000402e9004f22de0004007800e2
:107500000080fa00000006000200fa0084bd20009e
:107510001442780061426200e04f520010003a00cd
:10752000d80ba800b45e8000048fe900b55e80002f
:10753000e4e92000848f520002003a00e4ff2500b5
:10754000040f780001102000e00120003d05070035
:107550009e00780060002000ee0407000100370064
:10756000000000000080fa00000006000200fa009f
:10757000800020009c04070000027800040f7800bf
:10758000a45e80009e027800848f520005003600c1
:10759000a45e80009e025200141625000482420060
:1075a00003003700a45e80001e0252000482e9003e
:1075b000040078000080fa00000006001a00fa00bb
:1075c000881f7800300f9800410f9800c0012000fc
:1075d000850407000002780005042000050262000f
:1075e000e00f520042003a00d85e8000f28b0200a9
:1075f000000000000002be00040278008402540073
:10760000841e2000848f520037003600a5ff07003b
:1076100000027800e00f520007003200f28b0200f7
:10762000000000000002be0004027800d413b00085
:10763000d45e88002c003700541680004322de0000
:10764000614262000404a200614262000482fb0005
:10765000610262004322dd005616800075ff2f0094
:10766000850263000482720054168800f28b0200c7
:10767000000000000002be0004047800b8620200ae
:1076800000000000000278000400780001002000e3
:1076900002002000030020006408200005002000f4
:1076a0006033b8002a090200000000000203be0097
:1076b0000002be000400be000601be00f4ff2f0061
:1076c000050020006033b800700a020000000000ce
:1076d0000203be000002be0004027800040244005f
:1076e000440fb000d45e88000002eb005500370064
:1076f00084bd20001442780061426200e04f5200d5
:107700000a003a0080ff0700c0012000360407008d
:10771000000278000504200005026200e00f52001c
:1077200002003a000002eb0046003700b45e800021
:10773000a45e8800a45e800084007800a008200079
:10774000740407000e0278006201200084007800b3
:1077500040c0b300980207002e0a90000400780091
:10776000726702000000000000027800240f9800f9
:107770009e027800f4ff2500848f520015003e0021
:107780000e0278001442780061426200e04f52001d
:1077900010003a007e429000e04f52000d003a0087
:1077a000be0290000408200004826200e00f520034
:1077b00008003a002e02900070026200e00f5200b2
:1077c00004003a009e029000245f2000848f520043
:1077d00002003600000000000000fe001e027800db
:1077e000b45e88003e0a9000ee024700620020006e
:1077f0008500780004007800d80b0200000000002b
:10780000ce0a900000c2eb00844a78005e529000dd
:10781000e84f520009003a004e529000e04f5200eb
:10782000030032004e529000e64f520003003a002f
:107830004e529000ce0a9000844a7800d80ba900de
:1078400014002000040078004f0478000080fa0043
:10785000000006000800fa00100798004147980051
:10786000320798004e429000e04f520002003a006a
:10787000840020000100370084602000040f78009d
:107880008000eb0080082000220407003e029000e8
:107890006e02420084007800200020001d040700d2
:1078a0001e029000620020008400780020c0b30017
:1078b0001602070062002000b1b0200020c0b30013
:1078c000120207000e0278002200200084007800d7
:1078d00020c0b3000d0207000080fa00000006007f
:1078e0000200fa00c0012000bf0307000002780078
:1078f0000580200005026200e00f52001b003200ec
:1079000001802000c0012000800407002004200026
:10791000b503070000027800040f7800a0012000e2
:10792000b103070000027800054020000502620054
:10793000e00f5200050032005101200040042000f9
:10794000f40307001e00a0000500370021012000fd
:1079500040042000ef030700e4ff2f001e0f620029
:107960009e00780020042000ea030700a001200008
:107970009d03070000027800051020000502620048
:10798000e00f52000300320021002000e00120003f
:107990002c0407000080fa00000006000400fa0032
:1079a00010079800a55e80001e029000048242002d
:1079b000760f4200f4ff25009e027800848f52006b
:1079c00002003600e4e92a001e0f42009e00780003
:1079d000a0082000cf0307000080fa000000060086
:1079e0000400fa0010079800800820007e030700ba
:1079f00000027800040f78009e00900080082000ac
:107a0000c40307001e027800040078000080fa001a
:107a1000000006000400fa0010079800a0082000eb
:107a20007103070000027800040f78009e009000a8
:107a3000a0082000b70307001e02780004007800a9
:107a40000080fa00000006000600fa001007980007
:107a500021079800a55e80001e029000048242006b
:107a6000760f4200f4ff25009e027800848f5200ba
:107a700002003600e4e92a001e0f420084bd200007
:107a80001442780062426200e04f5200040032006b
:107a900001002800e0062000ea030700010037008b
:107aa00000000000e00120004f0307000002780002
:107ab0000502200005026200e00f5200f9ff3a00c3
:107ac0009e007800a000200092030700ae00900006
:107ad000c00020008f030700c1012000e00120004a
:107ae0000a04070001022000e0012000d50307007e
:107af00000000000e00120003b03070000027800c6
:107b00000502200005026200e00f5200f9ff3a0072
:107b100084bd20001442780062426200e04f5200af
:107b20000300320001002800e0062000f7030700f0
:107b3000000120002c0307000002780004007800f8
:107b40000080fa00000006000200fa00000f780032
:107b500084bd20001442780062426200e04f52006f
:107b60000400320001002800e0062000b5030700f1
:107b70000100370000000000e00120001a030700a8
:107b8000000278000502200005026200e00f5200aa
:107b9000f9ff3a00a0082000130307000002780054
:107ba00084007800a00020005a0307009e0078009f
:107bb000c000200057030700c1012000e0012000a1
:107bc000d203070001022000e00120009d0307000e
:107bd00000000000e001200003030700000278001d
:107be0000502200005026200e00f5200f9ff3a0092
:107bf00084bd20001442780062426200e04f5200cf
:107c00000300320001002800e0062000bf03070047
:107c100000012000f4020700000278000400780050
:107c20000080fa00000006000800fa001007980023
:107c300021079800320798001e029000e10f4200d1
:107c40000a003a0080082000e702070000027800de
:107c5000140798009e0290003e02900004824200a9
:107c600084007800800820002a0307002e0290007c
:107c7000e10f420010003a00a0082000da020700dd
:107c80000002780024079800ae0290003e029000a7
:107c9000048f4200f4ff25009e027800848f52007a
:107ca00002003600e4e92a001e0f42009e00780020
:107cb000a00820001703070084bd200014427800ac
:107cc00062426200e04f52000400320001002800ce
:107cd000e00620005b030700010037000000000001
:107ce000e0012000c0020700000278000502200029
:107cf00005026200e00f5200f9ff3a00ae0090006a
:107d0000a0002000030307009e009000e000200078
:107d100000030700be009000c0002000fd02070025
:107d200001032000e0012000460307000080fa0064
:107d3000000006000200fa00e0012000aa0207008d
:107d400000027800050220000502620004f0a7008e
:107d50000402ea00040fe9001e0278004f22de0050
:107d6000040f78001e027800e00f52000800320075
:107d700084bd20001442780062426200e04f52004d
:107d80000300320001002800e00620005f03070026
:107d90001e027800040078000080fa00000006004f
:107da0000200fa00120020008e00780040c0b300ec
:107db000010107001e427800044078000080fa00ac
:107dc000000006000600fa0010079800210798003e
:107dd0001e029000e00f5200050032002e019000bc
:107de0009e00900040c0b300f30007000e00370073
:107df000a00820007c02070000027800ae0290007c
:107e0000050f4200f4ff25009e027800848f520087
:107e100002003600e4e92a001e0f42009e007800ae
:107e2000a0082000bb0207002e029000040078008a
:107e30000080fa00000006000200fa00004f7800ff
:107e4000120020008e00780020c0b300af000700b1
:107e50000080fa00000006000400fa00000f78001d
:107e6000110798001e0190009e00780020c0b3000a
:107e7000a60007000080fa00000006000000fa00db
:107e800011002000e0012000200307000000000096
:107e9000a001200054020700000278000500220023
:107ea00005026200e00f5200f9ff3a0000000000f6
:107eb000e00120004c020700000278002582280023
:107ec00005026200e00f5200f9ff3a00d82ba8002b
:107ed000d84ba900c001200043020700000278002f
:107ee000e00f520001003d007003070001802000f8
:107ef0000040eb005603070001002c00e0062000c4
:107f0000020307000080fa00000006000000fa00eb
:107f10000100220010c1b3004d0307000080fa00e9
:107f2000000006000000fa00d82ba90001002c0078
:107f3000e0062000c30207000040eb002503070015
:107f4000000278000580200005026200e00f520068
:107f500003003200010021000040eb003c03070059
:107f60008000eb0010c1b3003903070000000000df
:107f7000a00120001c02070000027800052021005b
:107f800005026200e00f5200f9ff320011002000ec
:107f9000e0012000ab0207000080fa0000000600ac
:107fa0000400fa0020479800e00620000e020700b7
:107fb00000027800f50f2f0005026200040f780020
:107fc0000e0278000403e8000e0278000402e800c4
:107fd00014427800844278002e4290006f42620082
:107fe00004c27200044b78001e02780084007800fe
:107ff000e0062000470207000080fa0000000600ab
:108000000200fa00e0062000f701070000027800f5
:10801000040f78000e0278000402e8001442780091
:108020006f426200044078000080fa000000060001
:108030000000fa00d7e2a900d3e2a9002000200046
:10804000d88d020000000000db22a800d922a90080
:10805000d7e2a8000042eb0004407800d2ebb70062
:108060008002200001002000148e020000000000a9
:10807000d922a80041232100600120002502070029
:1080800060012000d801070000027800452321008c
:10809000850f5200f7ff3a0001012000e0062000a2
:1080a000680207000042eb0004407800d2ebb70002
:1080b00000000000a0012000cb01070000027800b2
:1080c00005a021008502620004a02100848f5200d7
:1080d000f8ff3a003000200001002000148e02005a
:1080e0000000000060012000bf01070000027800ce
:1080f000e00f5200dfff3a0010002000d88d020090
:10810000000000000080fa00000006000a00fa00eb
:10811000404798003107980042079800b404800057
:108120004d22de00614262000482fb0014079800c9
:1081300097a0a90024c3b300044f78004e429000da
:108140000482fb0062026200e00f52000200320073
:10815000a4c2b300044f78004e4290000482fb009a
:1081600064026200e00f520002003200e4c2b30079
:10817000044f78004e019000be0090001e40780031
:10818000540107001e029000044278006142620020
:108190000482fb00610262004d22dd00b604800013
:1081a000f5ff2d008502630004827200b40488008c
:1081b0000080fa00000006000a00fa00404798001c
:1081c00031079800420798004e029000e00f5200dd
:1081d00026003200b40480004d22de0061426200bd
:1081e0000482fb001407980097a0a90004c3b30001
:1081f000044f78004e4290000482fb00620262004d
:10820000e00f52000200320084c2b300044f780035
:108210004e4290000482fb0064026200e00f5200b4
:1082200002003200c4c2b300044f78004e01900037
:10823000be0090001e407800e20007001e02900081
:1082400004427800614262000482fb006102620025
:108250004d22dd00b6048000f5ff2d00850263008d
:1082600004827200b404880001003700000000009e
:108270000080fa00000006000600fa00404798005f
:10828000b40480004d22de00614262000482fb00e3
:10829000040f780097a0a900d7c2a9004e42900011
:1082a0000482fb0044128800041280006202620013
:1082b000e00f5200fcff3a000412800061026200ed
:1082c000e00f5200f8ff32004412800004427800b0
:1082d00024479800d7c2a8001e0278000442780004
:1082e000614262000482fb00610262004d22dd00f7
:1082f000b6048000f5ff2d00850263000482720041
:10830000b40488000080fa00000006000800fa00ab
:108310004047980031079800b40480004d22de00e9
:10832000614262000482fb00040f780097a0a9005c
:10833000d7c2a9004e4290000482fb00441288007c
:108340000412800062026200e00f5200fcff3a005b
:108350000412800061026200e00f5200f8ff320058
:108360008e82e8004412800004427800844a78003b
:1083700066024700144278000482fb004412880021
:108380000412800062026200e00f5200fcff3a001b
:108390000412800061026200e00f5200f8ff320018
:1083a0008e82e8004412800004427800844a7800fb
:1083b000660247000402e800144278000482fb00d1
:1083c000441288000412800062026200e00f520032
:1083d000fcff3a000412800061026200e00f5200cc
:1083e000f8ff32000e82e8008402e80044128000a8
:1083f00004427800844a7800d7c2a8001e027800a0
:1084000004427800614262000482fb006102620063
:108410004d22dd00b6048000f5ff2d0085026300cb
:1084200004827200b40488001e02900004007800e8
:108430000080fa00000006000c00fa006047980077
:108440004207980053079800b40480004d22de00d4
:10845000614262000482fb00040f780097a0a9002b
:10846000d7c2a9006e4290000482fb00441288002b
:108470000e82e800e30242000042eb00844a7800ea
:108480000412800062026200e00f5200fcff3a001a
:108490000412800061026200e00f5200f8ff320017
:1084a0008e82e8004412800004427800844a7800fa
:1084b00068024700144278000482fb0044128800de
:1084c0000412800062026200e00f5200fcff3a00da
:1084d0000412800061026200e00f5200f8ff3200d7
:1084e0008e82e8004412800004427800844a7800ba
:1084f000680247000402e800144278000482fb008e
:10850000441288000412800062026200e00f5200f0
:10851000fcff3a000412800061026200e00f52008a
:10852000f8ff32000e82e8008402e8004412800066
:1085300004427800844a7800680247000482e80018
:10854000144278000482fb00441288000412800068
:1085500062026200e00f5200fcff3a000412800049
:1085600061026200e00f5200f8ff32000e82e80064
:108570008482e8004412800004427800844a780033
:10858000d7c2a8001e02780004427800614262004f
:108590000482fb00610262004d22dd00b60480000f
:1085a000f5ff2d008502630004827200b404880088
:1085b0001e029000ae0290000400be000080fa008f
:1085c000000006000a00fa004047980031079800b2
:1085d00042079800b40480004d22de006142620030
:1085e0000482fb00040f780097a0a900d7c2a9005d
:1085f0004e4290000482fb00441288000412800066
:1086000062026200e00f5200fcff3a000412800098
:1086100061026200e00f5200f8ff32004412800055
:108620000442780024479800110037000002eb0054
:10863000441288000412800062026200e00f5200bf
:10864000fcff3a000412800061026200e00f520059
:10865000f8ff32004412800004427800be0290000d
:10866000844a78003e0290000402e8003407980033
:108670004e02900004f0a7000402ea000402ea009f
:108680004f22de0004427800ce0290008502e9000d
:1086900045079800e04f5200e4ff3a00d7c2a80017
:1086a0001e02780004427800614262000482fb00ee
:1086b000610262004d22dd00b6048000f5ff2d004e
:1086c0008502630004827200b40488000080fa000e
:1086d000000006000a00fa004047980031079800a1
:1086e00042079800b40480004d22de00614262001f
:1086f0000482fb00040f780097a0a900d7c2a9004c
:108700004e4290000482fb00441288000412800054
:1087100062026200e00f5200fcff3a000412800087
:1087200061026200e00f5200f8ff32004412800044
:108730000442780024479800120037003e0290005f
:10874000144278000482fb00441288003e0290002c
:108750000402e800340798000412800062026200fc
:10876000e00f5200fcff3a00041280006102620038
:10877000e00f5200f8ff32004412800004427800fb
:10878000244798004e02900004f0a7000402ea007b
:108790000402ea004f22de0004427800ce0290007c
:1087a0008502e90045079800e04f5200e3ff3a00d8
:1087b000d7c2a8001e02780004427800614262001d
:1087c0000482fb00610262004d22dd00b6048000dd
:1087d000f5ff2d008502630004827200b404880056
:1087e0000080fa00000006000a00fa004007980026
:1087f0004e0290008442780004ceb30004cf6200a1
:1088000004c6b3009e42780084cf52002a003e0086
:1088100024bd2000144278009e42780084cf52008c
:108820001c0032001e427800e04f520003003a0064
:1088300000ccb30090fe07001400370004c2b30060
:108840009e42780084cf520003003a0020ccb3004f
:1088500089fe07000d00370004c4b3009e42780073
:1088600084cf520003003a0040ccb30082fe0700e0
:108870000600370004c6b3009e42780084cf520041
:1088800002003a0060ccb3007bfe07001e40780077
:10889000d2ebb7004e029000044278007f426200a3
:1088a0008000eb000440780098fe0700000278008a
:1088b00014079800130037004e02900005002000b6
:1088c0000401be0000c2b300dbfe07000002be00d0
:1088d00024079800350798008e82e800640247005c
:1088e0000402e80014427800844a78000e82e8000e
:1088f0008402e800640247000482e8001442780021
:10890000844a78001e029000040078000080fa007b
:10891000000006000a00fa0030079800410798009e
:108920003e0290008442780004ceb30004cf62007f
:1089300004c6b3009e42780084cf52002b003e0054
:1089400024bd2000144278009e42780084cf52005b
:108950001c0032001e427800e04f520003003a0033
:1089600000ccb30044fe07001400370004c2b3007b
:108970009e42780084cf520003003a0020ccb3001e
:108980003dfe07000d00370004c4b3009e4278008e
:1089900084cf520003003a0040ccb30036fe0700fb
:1089a0000600370004c6b3009e42780084cf520010
:1089b00002003a0060ccb3002ffe07001e40780092
:1089c000d2ebb7004e0390003e02900004427800c4
:1089d000ff42620004c4b30004c272008600780043
:1089e0000440780049fe0700140037008e82e8003a
:1089f0003e02900004427800844a78000e82e8002b
:108a00008402e8006802470014427800844a780033
:108a10000e82e8008482e800680247000402e80051
:108a200014427800844a78001e029000ae02900042
:108a30000401be0020c2b3007ffe07000080fa00e0
:108a4000000006000600fa001007980021079800b1
:108a50001e0290008442780004ceb30004cf62006e
:108a600024bd2000144278009e42780084cf52003a
:108a70001c0032001e427800e04f520003003a0012
:108a800000ccb300fcfd07001400370004c2b300a3
:108a90009e42780084cf520003003a0020ccb300fd
:108aa000f5fd07000d00370004c4b3009e427800b6
:108ab00084cf520003003a0040ccb300eefd070023
:108ac0000600370004c6b3009e42780084cf5200ef
:108ad00002003a0060ccb300e7fd07001e407800ba
:108ae000d2ebb7001e02900004427800ff42620001
:108af00004c8b30004c27200ae00900004407800c5
:108b000002fe07000080fa00000006000600fa00de
:108b100010079800210798001e02900084427800f8
:108b200004ceb30004cf620024bd200014427800bc
:108b30009e42780084cf52001c0032001e42780012
:108b4000e04f520003003a0000ccb300cafd07001a
:108b50001400370004c2b3009e42780084cf520054
:108b600003003a0020ccb300c3fd07000d0037001e
:108b700004c4b3009e42780084cf520003003a0040
:108b800040ccb300bcfd07000600370004c6b300ac
:108b90009e42780084cf520002003a0060ccb300bd
:108ba000b5fd07001e407800d2ebb7001e02900012
:108bb00004427800ff42620004cab30004c272009b
:108bc000ae00900004407800d0fd07000080fa005d
:108bd000000006000400fa00204798002e42900092
:108be0008482fb000410200004827200840078005c
:108bf0004005200047ff070011002000200520004d
:108c000044ff070000000000a0062000f6fe070059
:108c1000000278006102620004427800e04f5200d6
:108c2000f9ff3a008000eb002005200039ff070023
:108c300080062000ecfe070000027800040f780098
:108c40001e027800040078000080fa000000060090
:108c50000400fa00004f7800110798001e427800c7
:108c60008482fb00041020000482720084007800db
:108c70004005200027ff07009e00900060062000ae
:108c800024ff070000000000a0062000d6fe070019
:108c9000000278006102620004427800e04f520056
:108ca000f9ff3a000080fa00000006000600fa0012
:108cb00020072000ccfe070000027800040f780097
:108cc0001e027800e00f520003003d000100280062
:108cd000200720008dff0700a0012000c2fe070032
:108ce0000002780014079800640247001200200078
:108cf00084007800d0c1b30032fe0700ce4290005d
:108d000004c8b30004c26a004447980064024700e4
:108d10001200200084007800d0c5b3006dfe07006b
:108d2000a0012000b0fe0700000278009e02900023
:108d300085026a000410200004826200e00f5200e5
:108d40000300320001802000c00120003dff070029
:108d50001e027800e00f520003003d0001002800d1
:108d60002007200037ff07000080fa0000000600ff
:108d70000400fa002047980014608000e00f5200c1
:108d80000c003a0014002000146088000042eb0040
:108d9000044f78000400370000c2eb000440780064
:108da00024ebb7001e4fe8001e427800e04f52004f
:108db000f9ff320044b2200014427800e14f420033
:108dc0000800320044b220001442780004407800c9
:108dd000505502000000000000c2eb000440780083
:108de00024ebb70014002000345988000042eb0047
:108df0000440780028ebb700288ba800282ba80097
:108e00000080fa00000006000200fa00004f78001f
:108e100044b2200014427800e14f420008003200c2
:108e200044b22000144278000440780050550200fb
:108e30000000000000c2eb000440780024ebb70003
:108e40000002eb00345988000080fa0000000600a0
:108e50000200fa00004f780034598000e00f520001
:108e600003003a001400200034598800280ba900a0
:108e70000080fa00000006000200fa00004f7800af
:108e80003459800004f0a7000402ea000402ea005a
:108e90004f22de00040078000080fa000000060087
:108ea0000200fa00004f78004459800061426200dd
:108eb0000482fb00040078000080fa000000060035
:108ec0000200fa00004f78004459800062026200fc
:108ed000e00f520003003200282ba90014002000ec
:108ee000010037000002eb00040078000080fa0067
:108ef000000006000200fa00004f7800445980008c
:108f00004322de00614262000482fb00040078001c
:108f10000080fa00000006000000fa00b559800049
:108f2000f40f200084826200e4ad20001442780037
:108f3000604262000542720004407800deeab70039
:108f4000b4598000c822de00f4ad2000144278003d
:108f5000604262000542720004407800dfeab70018
:108f6000c5598000f40f20008482620004ae200006
:108f700014427800604262000542720004407800aa
:108f8000e0eab700c4598000c822de0014ae200019
:108f9000144278006042620005427200044078008a
:108fa000e1eab7000080fa00000006000200fa00c3
:108fb0000042eb00044f78003e0237003459800035
:108fc00005002000c600200007002000860f520088
:108fd000878f5a0036023e00046001001b023700f2
:108fe0000b003700190037005300370071003700bd
:108ff0009000370093013700c3013700d8013700d4
:10900000c1013700d6013700bf013700d401370056
:1090100034042000430420000041eb006000b8004d
:10902000b8510200000000000042780004407800bf
:1090300024ebb70044b2200014427800e14f420014
:10904000040232002400200034598800c4032000a8
:109050000500200074598800855988000042eb0003
:10906000044078004aebb700280ba900284ba90060
:10907000523a02000000000000027800e00f5200a7
:10908000f601320044b22000144278000440780017
:10909000be5502000000000000027800b51220005a
:1090a000850f5200ef013600445980004422de0053
:1090b000614262000404a200614262000482fb007b
:1090c000610262004422dd0046598000f5fe2f0057
:1090d00085026300048272004459880044b2200073
:1090e000144278000482fb007822b90084027800e0
:1090f0000490200004824200a2002000f10f200012
:1091000004007800e60b0200000000008000eb0085
:1091100010c0b3006b030700e48b020000000000e6
:109120000002be00545988006559880034002000b0
:1091300034598800de01370044b220001442780020
:109140000440780078570200000000000002780018
:10915000950f2000850f52000f003e00e48b0200a7
:10916000000000000003be005459800065598000d3
:109170000403530085835b0074842e0015002000d7
:10918000840f5300858f5b00b80136002400200057
:1091900034598800c6013700286ba800ca010700af
:1091a00000427800e24f5200b2013a004400200031
:1091b0003459880044b220001442780004407800fa
:1091c000be550200000000000002780015102000cb
:1091d000850f5200a901360044b2200014427800e5
:1091e0000482fb007822b9008402780004902000f9
:1091f00004824200a2002000f10f20000400780049
:10920000e60b0200000000008000eb0030c0b3005d
:109210002c030700e48b0200000000000002be00e7
:10922000545988006559880054002000345988003a
:109230009f01370044b220001442780004407800b7
:10924000785702000000000000027800950f20000f
:10925000850f52000f003e00e48b0200000000006a
:109260000003be0054598000655980000403530078
:1092700085835b0074842e0015002000840f53004a
:10928000858f5b007f013600240020003459880060
:10929000870137008c010700004278000482fb0040
:1092a000e50f520003003200e60f5200e1003200e9
:1092b0007f01370044b22000144278000440780057
:1092c000505502000000000000c2eb00044078008e
:1092d00024ebb700e48b0200000000000002be0097
:1092e000545988006559880064002000345988006a
:1092f000282ba800280ba800545a800061026200a5
:10930000e00f520022003200b5598000f40f200017
:1093100084826200e4ad2000144278006042620062
:109320000542720004407800deeab700b4598000bc
:10933000c822de00f4ad20001442780060426200d2
:109340000542720004407800dfeab700c55980008a
:10935000f40f20008482620004ae200014427800e2
:10936000604262000542720004407800e0eab70003
:10937000c4598000c822de0014ae200014427800d8
:10938000604262000542720004407800e1eab700e2
:10939000545a800064026200e00f52002200320042
:1093a000f5598000f40f20008482620024ae200072
:1093b0001442780060426200054272000440780066
:1093c000e2eab700f4598000c822de0034ae200083
:1093d0001442780060426200054272000440780046
:1093e000e3eab700055a8000f40f2000848262008f
:1093f00044ae2000144278006042620005427200d0
:1094000004407800e4eab700045a8000c822de0075
:1094100054ae20001442780060426200054272009f
:1094200004407800e5eab700545a80006202620006
:10943000e00f520022003200d5598000f40f2000c6
:109440008482620064ae20001442780060426200b0
:109450000542720004407800e6eab700d459800063
:10946000c822de0074ae2000144278006042620020
:109470000542720004407800e7eab700e559800031
:10948000f40f20008482620084ae20001442780031
:10949000604262000542720004407800e8eab700ca
:1094a000e4598000c822de0094ae20001442780007
:1094b000604262000542720004407800e9eab700a9
:1094c000545a800068026200e00f5200200032000f
:1094d000145a8000255a8000f60f2000860362008f
:1094e000a6ae200016437800604363000743730074
:1094f00006407800eaeab700c823de00b6ae2000d6
:109500001643780060436300074373000640780009
:10951000ebeab700f60f200086836200c6ae20009b
:1095200016437800604363000743730006407800e9
:10953000eceab700c82ade00d4ae2000144278005e
:10954000604262000542720004407800edeab70014
:10955000e4ae2000144278006042620004407800cb
:10956000eeeab700f4ae20001442780060426200d8
:1095700004407800efeab70004af200014427800fe
:109580006042620004407800f0eab70014af2000a7
:10959000144278006042620004407800f1eab700ab
:1095a000545a800070026200e00f52002000320026
:1095b000345a8000455a8000f60f2000860362006e
:1095c000e6ae200016437800604363000743730053
:1095d00006407800eeeab700c823de00f6ae2000b1
:1095e0001643780060436300074373000640780029
:1095f000efeab700f60f20008683620006af200076
:109600001643780060436300074373000640780008
:10961000f0eab700c82ade0014af20001442780038
:10962000604262000542720004407800f1eab7002f
:109630000300370024002000345988000000000097
:109640009b003700e48b0200000000000003be0016
:1096500054598000655980000403530085835b00e2
:1096600034422f0005002000840f5300858f5b00db
:10967000860036007659800087598000140020004b
:1096800005002000840f5300858f5b000f0036001b
:10969000565980006759800044422f000500200081
:1096a0000602420087824a005459880065598800a2
:1096b000745980008559800061025200e0825a008e
:1096c00074598800855988007900370034042000d7
:1096d000430420000041eb006000b800b8510200d4
:1096e00000000000004278000440780024ebb7003e
:1096f00044b2200014427800e14f4200650032007d
:10970000740020003459880044b2200014427800cc
:1097100004407800be5502000000000000027800fe
:1097200015102000850f52005c003600110020004b
:1097300030c0b300e3010700284ba900e48b02000e
:10974000000000000002be005459880065598800de
:10975000345980000402e80034598800540037006e
:1097600044b2200014427800044078007857020088
:109770000000000000027800950f2000850f5200c5
:1097800015003e00e48b0200000000000003be0054
:1097900054598000655980000403530085835b00a1
:1097a00074842e0015002000840f5300858f5b0009
:1097b0003c003600345980000402e8003459880027
:1097c00034598000ec0f520038003600240020008d
:1097d00034598800360037003b000700004278000b
:1097e0000482fb00e50f520003003200e60f520036
:1097f000120032002e00370044b2200014427800dc
:1098000004407800505502000000000000c2eb0048
:109810000440780024ebb700e48b02000000000055
:109820000002be0054598800655988006400200079
:1098300034598800282ba80003003700240020009a
:1098400034598800000000001900370000000000b3
:10985000170037000000000015003700000000006e
:109860001300370000000000110037000000000066
:109870000f003700000000000d003700000000005e
:109880000b00370000000000090037000000000056
:10989000070037000000000005003700000000004e
:1098a0000300370000000000010037000000000046
:1098b0001e4fe8001e427800e04f5200bffd32000c
:1098c0000080fa00000006000c00fa000042eb00e5
:1098d000644798006402470004007800a85702001b
:1098e000000000004e429000e24f52004c013a004e
:1098f000c0012000a8550200000000000042eb005b
:10990000044f78000f00370064024700040078001d
:10991000a8570200000000009e4078000182fb0072
:10992000c502200084824200f4ad2000048242007f
:10993000944278004e42900084cf52004e013a008b
:109940001e4fe8001e427800e54f5200eeff360041
:109950004459800064026200e00f520008003a009f
:1099600000012000a8550200000000004100200076
:1099700060b32000dc570200000000004a0ba80082
:10998000000f2000a8550200000000000002eb00bc
:10999000140798006402470004007800a8570200ea
:1099a0000000000000027800e00f520003003a00bf
:1099b0001400200014079800190137004e4290004f
:1099c0000482fb0035032000850f5200c4003200e2
:1099d00035032000850f520007003c00e30f5200c2
:1099e0003e003200e60f52006a003200e10f5200e2
:1099f0001d003200f100370065032000850f520082
:109a000099003200f50f2000850f5200b10032009e
:109a100055032000850f5200e8003a006402470019
:109a200004007800a8570200000000004e42900099
:109a3000e14f520012013a0066024700040078002c
:109a4000a857020000000000445980006402620030
:109a5000e00f5200ec0032006e429000e24f5200e4
:109a6000eb003a001101370064024700040078005f
:109a7000a8570200000000004e429000e44f520040
:109a800001013a004459800064026200e00f520074
:109a90000c0032000042eb00044f78000500370054
:109aa0006402470004007800a8570200000000008c
:109ab0001e4fe8001e427800e34f5200f8ff3600c8
:109ac000d400370041002000e0b32000dc57020042
:109ad000000000004a4ba800ce0037006502470096
:109ae00004007800a8570200000000005e429000c9
:109af000e34f5200e60036004459800064026200e1
:109b0000e00f52000c0032000042eb00044f7800de
:109b1000050037006402470004007800a8570200df
:109b2000000000001e4fe8001e427800e34f520084
:109b3000f8ff36000500370041002000a0b32000e8
:109b4000dc570200000000004a2ba8005e42900093
:109b500064425200544798000400370064024700f2
:109b600004007800a8570200000000005e42900048
:109b70008482fb008502ea00cf2ade00854278005d
:109b80000442e90054479800e0cf5200f3ff3a0046
:109b9000a00037006502470004007800a8570200c3
:109ba000000000005e429000e34f5200ba00360011
:109bb0004459800064026200e00f520008003a003d
:109bc0004100200020b42000dc570200000000000b
:109bd0004a6ba8005e4290006442520054479800cd
:109be0005e429000e34f520012003600445980005c
:109bf00064026200e00f520010003a0041002000b1
:109c000060b42000dc570200000000004a8ba8006e
:109c10005e429000644252005447980008003700aa
:109c20006402470004007800a8570200000000000a
:109c300003003700000000000100370000000000b2
:109c40005e4290008482fb008502ea00cf2ade009b
:109c5000854278000442e90054479800e0cf520062
:109c6000efff3a006b003700640247000400780001
:109c7000a8570200000000004e429000e44f52003e
:109c800087003a006802470063024200040078003f
:109c9000a857020000000000680247000482e800a4
:109ca00004007800a8570200000000006802470086
:109cb0000402e80004007800a85702000000000039
:109cc0006802470004007800a85702000000000066
:109cd0005000370014002000140798004d00370092
:109ce0006402470004007800a8570200000000004a
:109cf0004e429000e44f52006b003a0044598000fd
:109d000064026200e00f52000c0032000042eb00df
:109d1000044f780005003700640247000400780013
:109d2000a8570200000000001e4fe8001e42780005
:109d3000e34f5200f8ff360036003700e4b220004f
:109d40006302420004007800a857020000000000ef
:109d5000e4b220000482e80004007800a857020062
:109d600000000000e4b220000402e80004007800d3
:109d7000a857020000000000e4b2200004007800b0
:109d8000a857020000000000765980008759800023
:109d90007459800085598000cb28dd004522de0003
:109da00004827000c52ade000402530085825b0035
:109db00074598800855988001600370065024700ed
:109dc00004007800a85702000000000004003700db
:109dd0006402470004007800a85702000000000059
:109de0005e4290008482fb008502ea00cf2ade00fa
:109df000854278000442e90054479800e0cf5200c1
:109e0000f3ff3a00030037000000000001003700b4
:109e1000000000001e029000e00f5200ddfe320044
:109e20006e429000e24f520006003a004e0290004f
:109e3000de02900094598800a5598800284ba8009c
:109e40000900370096598000a75980004e02900003
:109e5000de029000840f5300858f5b000200320009
:109e60000042eb0064479800285802000000000000
:109e70006e42900010003700000000000b00370019
:109e80000000000009003700000000000700370054
:109e9000000000000500370000000000030037004c
:109ea00000000000010037000000000028580200f8
:109eb000000000000042eb00044078000080fa003f
:109ec000000006000a00fa00604798004107980069
:109ed00010c0b300f45502000000000010c0b30031
:109ee000f45502000000000060c0b300f455020009
:109ef000000000000040eb00f455020000000000ec
:109f000020c1b300f45502000000000030c2b300cd
:109f1000f45502000000000040c3b300f4550200f5
:109f20000000000060c5b300f4550200000000000e
:109f30000040eb00f4550200000000000040eb0080
:109f4000f4550200000000004459800070026200d5
:109f5000e00f5200020032000042eb000100370027
:109f600004c8b30004407800f4550200000000006b
:109f70000040eb00f4550200000000006e4290002b
:109f8000e34f520008003a004e029000e00f5200ea
:109f9000050032004100200060b32000245602007a
:109fa000000000000c0037000040eb00f4550200f8
:109fb000000000000040eb00f4550200000000002b
:109fc0000040eb00f4550200000000000040eb00f0
:109fd000f4550200000000000042eb00044f78003e
:109fe000040037000040eb00f455020000000000c0
:109ff0001e4fe8001e427800eb4f5200f9ff36007a
:10a0000061002000b0b020002456020000000000d3
:10a010000042eb00044f7800040037000040eb00e2
:10a02000f4550200000000001e4fe80094ccb3007d
:10a030009e42780084cf5200f8ff360030c6b3004d
:10a04000f45502000000000020c8b300f4550200df
:10a050000000000030c5b300f4550200000000000d
:10a0600030c6b300f45502000000000050c3b30036
:10a07000f45502000000000010c0b300f4550200c7
:10a08000000000006e409000f45502000000000047
:10a090006e429000e14f520001003a00284ba900a7
:10a0a0006e429000e34f520020003a004e029000b2
:10a0b000e00f52001d003a0060c3b300f4550200e7
:10a0c0000000000040c0b300f45502000000000092
:10a0d00024b3200063024200144278000440780058
:10a0e000f45502000000000024b320000482e800c0
:10a0f0001442780004407800f4550200000000008b
:10a1000024b320000402e8001442780004407800e0
:10a11000f45502000000000024b32000144278002f
:10a1200004407800f45502000000000070c3b30042
:10a13000f45502000000000040c0b300f4550200d6
:10a140000000000010c0b300f45502000000000041
:10a1500030c0b300f45502000000000060c0b3003e
:10a16000f455020000000000c0c0b300f455020026
:10a17000000000006e429000e34f520003003a00de
:10a180004e029000e00f5200080032006e42900034
:10a19000e14f52000f003a00b4598000c5598000c9
:10a1a000e00f5200e08f5a000a00320020c3b300d3
:10a1b000f45502000000000040c0b300f455020056
:10a1c000000000004100200060b32000245602007f
:10a1d0000000000000c0eb00f45502000000000089
:10a1e000030037000040eb00f455020000000000bf
:10a1f000154e8000b4122000848f5200f9ff360003
:10a20000e6ad2000164378008683fb00f6ad200003
:10a21000164378000683fb004833dd000703730014
:10a220000602780006ae2000164378008683fb0005
:10a2300016ae2000164378000683fb004833dd008d
:10a24000070373008602780014079800250798001a
:10a250004e029000e00f520014003a00e4ad2000de
:10a26000144278006042620004407800deeab700e1
:10a27000f4ad20001442780060426200044078008f
:10a28000dfeab70004ae20001442780060426200aa
:10a2900004407800e0eab70014ae200014427800d1
:10a2a0006042620004407800e1eab7007e56020096
:10a2b000000000001e029000ae029000f60f200089
:10a2c00086036200e6ad2000164378006043630019
:10a2d0000743730006407800deeab700c823de00bb
:10a2e000f6ad200016437800604363000743730017
:10a2f00006407800dfeab700f60f20008683620090
:10a3000006ae2000164378006043630007437300e5
:10a3100006407800e0eab700c82ade0014ae20004c
:10a3200014427800604262000542720004407800e6
:10a33000e1eab7000080fa00000006000200fa001f
:10a340000042eb00044f7800030037001e40780005
:10a35000d30107001e4fe8001e427800e74f52006d
:10a36000faff3600ca29a8000080fa0000000600a3
:10a370000e00fa002007980031079800024f98005d
:10a380005307980064079800049020001407980071
:10a390000042eb00044f78007b0037001e02900063
:10a3a00064029000e00f520073003a001e02900019
:10a3b0005e009000600298005e029000e00f520084
:10a3c0000f003a006560800004002200848f520074
:10a3d00004003e0065608000f4ff2000848f52007e
:10a3e00002003e0004002100646088006460800078
:10a3f0009e029000e40298000402e8006460880075
:10a400000e4a9000e04f5200050032002e029000ec
:10a41000be029000e00f5200e08f5a000a003a009e
:10a420001e029000a2002000f10f2000040078001e
:10a43000e60b0200000000001e0290005500200004
:10a4400075029800450037000e4a90000482fb0018
:10a450006123b9000082eb008082eb00060242001b
:10a4600087824a003600200007002000860f520035
:10a47000878f5a0038003e00046001000300370057
:10a480000200370018003700270037001e02900036
:10a490002e039000be039000068abe000e4a900074
:10a4a0000414a2000482fb000402e9004f22de0033
:10a4b000044278009e0290000482fb006102620068
:10a4c0004822dd00a50b9000f6ef2f000683630005
:10a4d00004027300a40a98001e02900015002000d8
:10a4e000750298001d0037001e0290002e03900098
:10a4f000be039000068abe009e0290000042eb0060
:10a50000c45298001e039000d403200005002000d0
:10a51000040b9800150b98001e02900025002000e7
:10a52000750298000d0037002e029000840278001a
:10a530001e029000a2002000850078000400780030
:10a54000d80b0200000000001e0290005500200001
:10a550007502980001003700000000001e02900004
:10a56000ee039000570298001e407800c0e9b70043
:10a570001e427800080037001e0290007802420058
:10a58000140798001e4fe8001e427800e74f520063
:10a5900082ff360000c2eb00044078000080fa0021
:10a5a000000006000600fa00881f78000042eb0059
:10a5b000044f7800220137009e4278000582fb009c
:10a5c0007822b90004027800ee02420004902000d4
:10a5d0000482420014027800e50f52000c013200a0
:10a5e0009e4278000582fb007822b90004027800c0
:10a5f000ee0242000490200004824200140278001f
:10a60000e40f5200040132009e4278000582fb00f4
:10a610007822b90004027800ee0242000490200083
:10a620000482420014027800050020003600200059
:10a6300007002000860f5200878f5a00f8003e0066
:10a640000460010036003700020037006c0037005c
:10a65000880037000c5a0200000000000002780059
:10a66000e00f5200f00032009e4278000582fb00ad
:10a670007822b90084027800e4902000048242002d
:10a680008002eb00050a78009e4278000582fb00fc
:10a690007822b90004027800f402420004902000fd
:10a6a00004824200140278004822de006142620007
:10a6b000e04f52000d0032009e4278000582fb0000
:10a6c0007822b900840278000490200004824200bd
:10a6d0001402be000402780011c0b3000400780028
:10a6e000585a020000000000d40037009e42780053
:10a6f0000582fb007822b9008402780004902000d3
:10a70000048242001402be000402780011c0b300ab
:10a7100004007800585a020000000000c70037000b
:10a720000e82e800040078008a5a0200000000004f
:10a7300000027800e00f5200bd003200265a0200ed
:10a740000000000000027800e00f520023003200f9
:10a750001e4278000483fb001e029000ae029000af
:10a760007833b90086037800069020000683430002
:10a77000048bbe009e4278000582fb007822b9005f
:10a7800084027800e490200004824200250020002a
:10a79000050a78009e4278000582fb007822b90005
:10a7a0008402780044912000848242000042eb0041
:10a7b000844a78009e4278000582fb007822b90026
:10a7c000840278000491200004834200d403200016
:10a7d00005002000048bbe00980037009e427800e0
:10a7e0000582fb007822b90084027800e490200002
:10a7f0000482420015002000050a78008f0037000f
:10a800001e4278000484fb00f28b0200000000006e
:10a810000002be00040378007842b9008402780088
:10a820006491200004824200060a78009e4278006b
:10a830000582fb007822b900840278000490200091
:10a8400004824200040078009a7c020000000000ac
:10a850009e4278000582fb007822b90084027800cd
:10a86000e49020000482420035002000050a7800b0
:10a87000720037009e4278000582fb007822b90002
:10a8800004027800e40242000490200004834200a5
:10a890009e4278000582fb007822b900840278008d
:10a8a00004902000048242008600780004007800b2
:10a8b0005c7d02000000000000027800e00f520002
:10a8c0004a003a00f28b0200000000000002be00c5
:10a8d000040378009e4278000582fb007822b900cc
:10a8e00004027800f6024200049020000482420034
:10a8f00014027800040353009e4278000582fb0096
:10a900007822b90004027800f0024200049020008e
:10a91000048242001402be0004027800840f530037
:10a92000450036009e4278000582fb007822b9007f
:10a9300004027800f40242000490200004824200e5
:10a9400014427800e54f52001f003e001e4278007e
:10a950008483fb00783ab90004027800f4024200d4
:10a960000490200004824200144278000443e8006e
:10a97000783ab900840278004491200004824200b1
:10a98000064a78009e4278000583fb009e427800cc
:10a990000582fb007822b90004027800f002420030
:10a9a00004902000048242001402be00040242000f
:10a9b00085824a007833b90086037800069120002a
:10a9c00006834300048bbe009e4278000582fb0094
:10a9d0007822b90084027800e490200004824200ca
:10a9e00025002000050a7800140037009e427800f8
:10a9f0000582fb007822b90084027800e4902000f0
:10aa00000482420055002000050a78000b00370040
:10aa100000000000090037000000000007003700b8
:10aa200000000000050037000000000003003700b0
:10aa30000000000001003700000000001e4fe80089
:10aa40001e427800e74f5200dbfe36004f047800cc
:10aa50000080fa00000006000200fa00004f7800b3
:10aa60009e4278000582fb007822b900040278003b
:10aa7000ee0242000490200004824200140278009a
:10aa800065026a0004f0a7000402ea000402e9007b
:10aa90004f22de00040078000080fa00000006006b
:10aaa0000200fa00004f78001e427800e74f520083
:10aab00019003e009e4278000582fb007822b90012
:10aac00084027800c4902000048242008002eb00df
:10aad000050a78009e4278000582fb007822b900c2
:10aae0008402780004902000048342006022b800b1
:10aaf000048bbe009e4278000582fb007822b900dc
:10ab000084027800e4902000048242004500200086
:10ab1000050a780001003700000000000080fa00fc
:10ab2000000006000200fa00000f7800a5022000d5
:10ab30001e82420004007800f03c02000000000089
:10ab40001e027800344e88000080fa0000000600e3
:10ab50000200fa00000f78009e027800688242002e
:10ab600004007800c4870200000000001e02780084
:10ab7000444e88000080fa00000006000200fa003f
:10ab8000004f78006c3a02000000000000027800dc
:10ab9000e00f520002003a000002eb000f00370005
:10aba000a4c02000144278009e4f520006003200dc
:10abb0001e4078000aecb7000002eb00144e88003b
:10abc0000000eb00d7ff07001e407800c0e9b70087
:10abd000144e8000055c20000482520004007800be
:10abe0000080fa00000006000200fa00004f780022
:10abf000354e8000f45b2000848f52000200360046
:10ac00000002eb000d0037001e4078001c3f0200e0
:10ac100000000000344e80000402e800344e88003a
:10ac2000354e8000144e8000848f520002003600a2
:10ac3000344e8000144e8800140020000400780078
:10ac40000080fa00000006000600fa0010079800d5
:10ac500021079800344e8000055c2000048f5200cc
:10ac60002e0290009e027800848f52000200310074
:10ac70001e02780024079800354e80002e029000b6
:10ac800004824200344e8800354e8000144e80000d
:10ac9000848f520002003600344e8000144e88002b
:10aca000ae0090001e0090002c3f0200000000004b
:10acb0002e029000040078000080fa0000000600d8
:10acc0000200fa00000f78001e02780004007800ed
:10acd000160c0200000000000002780084007800da
:10ace0001e007800d8ff0700000278001e02420014
:10acf000040078000080fa00000006001c00fa0042
:10ad0000049c2000144278000482fb007822b900e1
:10ad10008402780004902000048f4200144e8000ca
:10ad200068024200140798001e0278006402900036
:10ad30000400780072670200000000000002780042
:10ad4000340798001e027800540290000400780036
:10ad500072670200000000000002780044079800bb
:10ad60001e009000726702000000000000027800e0
:10ad7000540798000002eb0064079800e6ad20003d
:10ad8000164378008683fb00f6ad2000164378005a
:10ad90000683fb004833dd000703730006027800da
:10ada00006ae2000164378008683fb0016ae200016
:10adb000164378000683fb004833dd000703730069
:10adc0008602780074079800050f98001e0278002c
:10add0001403be00160f9800270f98000042eb00e6
:10ade0006457980014c1b300745798009e039000f4
:10adf000470f98004e0a9000040078007267020026
:10ae00000000000000027800440f98006e02470026
:10ae1000c100200004007800ee670200000000007e
:10ae2000000278000482ea0064079800e000200035
:10ae3000f03c0200000000001e0278001e0190009d
:10ae400011c1b30004007800128702000000000066
:10ae50006602470081002000040078002c3f0200b9
:10ae600000000000200220000a3d02000000000057
:10ae700000027800240798001e009000a43d020004
:10ae80000000000000027800540f98005e0a900055
:10ae9000e00f520002003a000082eb00540f9800cd
:10aea0002e0090000a3d02000000000080022000f9
:10aeb000f03c0200000000007a0247002100200060
:10aec000040078002c3f020000000000703c0200eb
:10aed000000000000002eb00144e880000c2eb00ee
:10aee000044078000aecb7000080fa000000060079
:10aef0000200fa00004f78001e407800c0e9b70059
:10af0000b4c02000144278009e4f5200020032006c
:10af10000002eb000b003700a49c200014427800d4
:10af200061426200e04f520003003200ca09a900ea
:10af30000000eb0006ff0700254e8000444e800015
:10af400004825200040078000080fa00000006002d
:10af50000200fa00000f7800454e8000244e800069
:10af6000848f520006003100b5c020009542780061
:10af7000049c20001442780084cf5200020032006a
:10af80000002eb0009003700d03e02000000000084
:10af9000004278009e027800844a7800444e800087
:10afa0000402e800444e88001400200004007800e9
:10afb0000080fa00000006000600fa001007980062
:10afc00021079800454e8000244e8000848f520057
:10afd00006003100b5c0200095427800049c200096
:10afe0001442780084cf5200020032000002eb00cd
:10aff00014003700254e8000444e8000048f52001c
:10b000002e0290009e027800848f520002003100d0
:10b010001e02780024079800ae0090001e009000e9
:10b02000e23e0200000000000002780024079800c1
:10b03000454e80002e02900004824200444e88005b
:10b040002e029000040078000080fa000000060044
:10b050000000fa00a49c20001442780062426200c2
:10b06000e04f520008003a00843a0200000000005d
:10b070000002eb00244e880000c2eb000440780080
:10b080000becb700ca29a8000080fa0000000600f7
:10b090002000fa00500f9800610f9800720f98007e
:10b0a0000002eb00244e88000e82e80081002000a0
:10b0b00004007800e23e0200000000001e02900042
:10b0c00004007800726702000000000000027800af
:10b0d000140798002e0290000400780072670200a6
:10b0e0000000000000027800240798003e02900053
:10b0f000040078007267020000000000000278007f
:10b1000068025200340798004e029000e00f52008f
:10b11000390032005e0b9000164278000480fb007c
:10b12000964390008783fb00c83bdd00808373005b
:10b1300007027800a64390008783fb003643900007
:10b140000683fb004833dd000703730086027800a6
:10b1500054079800650798006e0a90001402be001c
:10b1600074079800050f98000042eb0024579800e0
:10b1700014c1b300345798007e089000200f980047
:10b180002e0a9000040078007267020000000000a0
:10b1900000027800240f98006a024700c1002000d6
:10b1a00004007800ee670200000000000002780052
:10b1b0000482ea00340f98000000eb00c48702000c
:10b1c000000000007e089000a43d02000000000086
:10b1d00000027800440f9800be0a90004e0a9000ca
:10b1e000848f520004003200843a02000000000004
:10b1f0000002eb00150037000e82e8006e09900097
:10b20000de08900004007800130007000042780078
:10b21000044f78001e427800e14f420004003a00db
:10b22000843a0200000000000002eb000700370033
:10b230001e4078000becb7003e029000244e8800c0
:10b24000ca09a800ca29a900140020000400780037
:10b250000080fa00000006000a00fa0020079800ab
:10b2600031079800420798003e029000944278000f
:10b270000580fb00944290008582fb00c82add0017
:10b280008082720005037800a44290008582fb0052
:10b29000344290000482fb004822dd000502720067
:10b2a00084037800decabf008080fb00dfcabf00d5
:10b2b0000080fb004800dd00010070000002780003
:10b2c000e0cabf008080fb00e1cabf000080fb0035
:10b2d0004800dd000100700080027800840f5300f8
:10b2e000858f5b0002003a0000c2eb004700370088
:10b2f00000c2eb0014479800049020001407980047
:10b300000042eb00044f7800280037001e02900036
:10b31000e40290002e02900014029000848f5200ec
:10b320001e003a001e029000d40290002e029000ef
:10b3300014027800848f520016003a001e0290001a
:10b340001403be003e009000104278000481fb0010
:10b35000904090008180fb00c808dd008280700072
:10b3600001027800a04090008180fb0030409000f6
:10b370000080fb004800dd000100700080027800c2
:10b38000840f5300858f5b0002003a001e42780054
:10b390001e0037009e427800154798001e0290005c
:10b3a00078024200140798001e4fe8001e42780001
:10b3b000e74f5200d5ff36001e429000e14f420099
:10b3c000110032001e4290000482fb007822b90076
:10b3d0008402780004902000048242001407980040
:10b3e0001e029000a2002000be0090000400780021
:10b3f000d80b0200000000002e029000940278009a
:10b400001e029000550298001e42900004407800f1
:10b410000080fa00000006000000fa0044ba200094
:10b420001442780061426200e04f52000200320094
:10b430000002eb0002003700a40ba800140020005b
:10b44000040078000080fa00000006000000fa0006
:10b45000a4be200014427800e14f420008003200f0
:10b46000a4be200014427800044078005055020029
:10b470000000000000c2eb0004407800eaebb700d7
:10b4800074002000645f8800a40ba90044ba200067
:10b49000144278000482fb000402d1006142620081
:10b4a0000482fb00040078000080fa00000006001f
:10b4b0000400fa00000f780021479800a1b920008d
:10b4c0001e007800326402000000000000027800d4
:10b4d000e00f520004003200a42ba80074002000ea
:10b4e000645f8800090037001e007800a05c8800b7
:10b4f0000002eb00b45c88000002eb00645f88008f
:10b500002e40900098ebb700a42ba9000080fa0011
:10b51000000006001c00fa00500f9800645f8000d5
:10b52000050020007600200007002000860f520052
:10b53000878f5a0082033e00046001000700370035
:10b540000c0037001b0037004c0037005c00370050
:10b55000b00037007c0237006d0237000042eb007c
:10b5600004407800a5ebb7000042eb0004407800ef
:10b57000a6ebb700a0ae20009a7c020000000000fd
:10b5800054ba2000144278000442e80004407800d5
:10b59000a5ebb700e48b0200000000000002be0033
:10b5a000445d8800555d880024002000645f8800a9
:10b5b00063033700e1b92000a0ae20005c7d0200eb
:10b5c0000000000000027800e00f520015003a0071
:10b5d000e48b0200000000000003be00445d800018
:10b5e000555d80000403530085835b0044422f00b7
:10b5f00005002000840f5300858f5b004703360051
:10b6000054ba200014427800e24f52000200360083
:10b61000640020000100370014002000645f8800ef
:10b6200047033700a6ae2000164378008683fb0050
:10b63000b6ae2000164378000683fb004833dd00d9
:10b640000703730006027800c6ae20001643780098
:10b650008683fb00d6ae2000164378000683fb00ed
:10b660004833dd000703730086027800d45c88004d
:10b67000e55c880034002000645f8800a4b92000e5
:10b680006123b800540320008001eb0042c0b300e6
:10b690000600be00b8510200000000000042780021
:10b6a00004407800eaebb700a4be20001442780002
:10b6b000e14f42001b03320044002000645f880019
:10b6c000a4be20001442780004407800be55020059
:10b6d0000000000000027800e00f52001303320067
:10b6e000246080000402e8002460880054c0200028
:10b6f0001442780004407800f45502000000000075
:10b7000044c020001442780004407800f455020040
:10b710000000000010c0b300f4550200000000005b
:10b720000040eb00f4550200000000000040eb0078
:10b73000f45502000000000010c0b300f4550200f0
:10b74000000000000040eb00f45502000000000083
:10b750000040eb00f4550200000000000040eb0048
:10b76000f4550200000000000040eb00f455020018
:10b77000000000000040eb00f45502000000000053
:10b780000040eb00f455020000000000a45c8000c3
:10b79000e00f520004003200a45c80000400780036
:10b7a000eb02070003003700b45c8000040078005f
:10b7b000e70207000040eb00f45502000000000023
:10b7c00084b920001442780004407800f455020047
:10b7d000000000000040eb00f455020000000000f3
:10b7e00010c0b300f4550200000000007e560200b5
:10b7f00000000000e48b0200000000000002be0018
:10b80000445d8800555d880054002000645f880016
:10b81000cb023700a4be2000144278000440780018
:10b82000785702000000000000027800e00f52008c
:10b830000f003a00e48b0200000000000003be008d
:10b84000445d8000555d80000403530085835b00e8
:10b8500044422f0005002000840f5300858f5b00b9
:10b86000b402360064002000645f8800b402370030
:10b87000640247000402e80004007800a8570200b0
:10b88000000000006402470004007800a85702008e
:10b8900000000000ae02900024608000848f5200ff
:10b8a000030032002858020000000000a402370004
:10b8b000640247006302420004007800a8570200b7
:10b8c00000000000640247000482e80004007800e1
:10b8d000a857020000000000640247006502420011
:10b8e00004007800a857020000000000640247002e
:10b8f0006402420004007800a85702000000000023
:10b90000640247006702420004007800a857020062
:10b910000000000064024700660242000400780054
:10b92000a8570200000000006402470069024200bc
:10b9300004007800a85702000000000064024700dd
:10b940006802420004007800a857020000000000ce
:10b95000640247006b02420004007800a85702000e
:10b9600000000000640247006a0242000400780000
:10b97000a85702000000000013003700ba020700b9
:10b980000e82e8000402e80004007800a8570200d4
:10b99000000000000e82e80004007800a8570200b2
:10b9a000000000000e82e8000402e80004007800b5
:10b9b000a8570200000000000e82e8000400780092
:10b9c000a857020000000000ce0290000502780097
:10b9d00004f0a7000402ea000402ea004f22de009d
:10b9e000044278008502e90045079800e04f5200c4
:10b9f000e2ff3a005d0037009b020700700247003b
:10ba00000402e80004007800a857020000000000cb
:10ba10007002470004007800a857020000000000f0
:10ba2000700247006302420004007800a857020039
:10ba300000000000700247000482e8000400780063
:10ba4000a857020000000000700247006702420091
:10ba500004007800a85702000000000070024700b0
:10ba60006602420004007800a857020000000000af
:10ba7000700247006502420004007800a8570200e7
:10ba800000000000700247006402420004007800d9
:10ba9000a85702000000000070024700690242003f
:10baa00004007800a8570200000000007002470060
:10bab0006802420004007800a8570200000000005d
:10bac0000e0a9000e10f520018003a001e0a900082
:10bad000e10f520017003a004e0a9000e40f5200a6
:10bae00016003a00a42ba800a0b92000a857020015
:10baf00000000000b0b92000a857020000000000bc
:10bb0000c0b92000a857020000000000d0b92000f2
:10bb1000a857020000000000f10037000e00780076
:10bb2000a8570200000000000500370000000000d8
:10bb30000300370000000000010037000000000093
:10bb4000ce0a90000502780004f0a7000402ea0083
:10bb50000402ea004f22de00044278008502e90078
:10bb6000450f9800e04f5200ecff3a00de029000d3
:10bb70000502780004f0a7000402ea000402ea00cb
:10bb80004f22de00044278008502e9005507980044
:10bb9000e04f520098ff3a005d0037003202070084
:10bba000700247000402e80004007800a857020071
:10bbb000000000007002470004007800a85702004f
:10bbc0000000000070024700630242000400780099
:10bbd000a857020000000000700247000482e8003d
:10bbe00004007800a857020000000000700247001f
:10bbf0006702420004007800a8570200000000001d
:10bc0000700247006602420004007800a857020054
:10bc10000000000070024700650242000400780046
:10bc2000a8570200000000007002470064024200b2
:10bc300004007800a85702000000000070024700ce
:10bc40006902420004007800a857020000000000ca
:10bc5000700247006802420004007800a857020002
:10bc6000000000000e0a9000e10f520018003a0098
:10bc70001e0a9000e10f520017003a004e0a900091
:10bc8000e40f520016003a00a42ba800a0b920002f
:10bc9000a857020000000000b0b92000a857020019
:10bca00000000000c0b92000a857020000000000fa
:10bcb000d0b92000a857020000000000880037001b
:10bcc0000e007800a85702000000000005003700b1
:10bcd00000000000030037000000000001003700f2
:10bce00000000000ce0a90000502780004f0a700d2
:10bcf0000402ea000402ea004f22de000442780057
:10bd00008502e900450f9800e04f5200ecff3a0031
:10bd1000ee0290000502780004f0a7000402ea0099
:10bd20000402ea004f22de00044278008502e900a6
:10bd300065079800e04f520098ff3a005d00370019
:10bd4000c9010700700247000402e80004007800ff
:10bd5000a8570200000000007002470004007800ad
:10bd6000a857020000000000700247006302420072
:10bd700004007800a857020000000000700247008d
:10bd80000482e80004007800a857020000000000c8
:10bd9000700247006702420004007800a8570200c2
:10bda00000000000700247006602420004007800b4
:10bdb000a857020000000000700247006502420020
:10bdc00004007800a857020000000000700247003d
:10bdd0006402420004007800a8570200000000003e
:10bde000700247006902420004007800a857020070
:10bdf0000000000070024700680242000400780062
:10be0000a8570200000000000e0a9000e10f520047
:10be100018003a001e0a9000e10f520017003a0085
:10be20004e0a9000e40f520016003a00a42ba8001e
:10be3000a0b92000a857020000000000b0b92000ff
:10be4000a857020000000000c0b92000a857020057
:10be500000000000d0b92000a85702000000000038
:10be60001f0037000e007800a857020000000000f5
:10be7000050037000000000003003700000000004c
:10be80000100370000000000ce0a90000502780093
:10be900004f0a7000402ea000402ea004f22de00d8
:10bea000044278008502e900450f9800e04f5200f7
:10beb000ecff3a00fe0290000502780004f0a700b3
:10bec0000402ea000402ea004f22de000442780085
:10bed0008502e90075079800e04f520098ff3a008c
:10bee0002858020000000000a4be20001442780080
:10bef00004407800505502000000000000c2eb0032
:10bf000004407800eaebb70074002000645f88000a
:10bf100044ba20001442780062426200e04f5200ae
:10bf200003003a006022b800d45c8800e55c880019
:10bf3000d45c8000e55c80005e0b9000048bbe004a
:10bf400014002000ff00370064ba2000144278007b
:10bf5000e14f5200050036005e0b90006022b800f1
:10bf6000048bbe0014002000f600370064ba2000e5
:10bf7000144278000442e80004407800a6ebb700c1
:10bf8000e6ae2000164378008683fb00f6ae200064
:10bf9000164378000683fb004833dd000703730077
:10bfa0000602780006af2000164378008683fb0067
:10bfb00016af2000164378000683fb004833dd00ef
:10bfc0000703730086027800e00f5200e08f5a00ea
:10bfd000da003200a4ae2000144278008482fb0014
:10bfe000b4ae2000144278000482fb004822dd0039
:10bff0000502720004037800c4ae200014427800e9
:10c000008482fb00d4ae2000144278000482fb003e
:10c010004822dd000502720084037800eecabf00ea
:10c020008080fb00efcabf000080fb004800dd00fd
:10c030000100700000027800f0cabf008080fb00a1
:10c04000f1cabf000080fb004800dd000100700065
:10c050008002780004026b0085826b00f60f2000de
:10c0600086036200a6ae200016437800604363009a
:10c070000743730006407800eaeab700c823de00f1
:10c08000b6ae200016437800604363000743730098
:10c0900006407800ebeab700f60f200086836200c6
:10c0a000c6ae200016437800604363000743730068
:10c0b00006407800eceab700c82ade00d4ae2000c3
:10c0c0001442780060426200054272000440780029
:10c0d000edeab700e4ae2000144278008482fb0051
:10c0e000f4ae2000144278000482fb004822dd00f8
:10c0f000050272000403780004af200014427800a7
:10c100008482fb0014af2000144278000482fb00fc
:10c110004822dd000502720084037800eacabf00ed
:10c120008080fb00ebcabf000080fb004800dd0000
:10c130000100700000027800eccabf008080fb00a4
:10c14000edcabf000080fb004800dd000100700068
:10c150008002780004026b0085826b00f60f2000dd
:10c1600086036200e6ae2000164378006043630059
:10c170000743730006407800eeeab700c823de00ec
:10c18000f6ae200016437800604363000743730057
:10c1900006407800efeab700f60f200086836200c1
:10c1a00006af200016437800604363000743730026
:10c1b00006407800f0eab700c82ade0014af20007d
:10c1c0001442780060426200054272000440780028
:10c1d000f1eab700a4ae2000144278008482fb008c
:10c1e000b4ae2000144278000482fb004822dd0037
:10c1f0000502720004037800c4ae200014427800e7
:10c200008482fb00d4ae2000144278000482fb003c
:10c210004822dd000502720084037800eecabf00e8
:10c220008080fb00efcabf000080fb004800dd00fb
:10c230000100700000027800f0cabf008080fb009f
:10c24000f1cabf000080fb004800dd000100700063
:10c250008002780004026b0085826b00f60f2000dc
:10c2600086036200a6ae2000164378006043630098
:10c270000743730006407800eaeab700c823de00ef
:10c28000b6ae200016437800604363000743730096
:10c2900006407800ebeab700f60f200086836200c4
:10c2a000c6ae200016437800604363000743730066
:10c2b00006407800eceab700c82ade00d4ae2000c1
:10c2c0001442780060426200054272000440780027
:10c2d000edeab7000042eb0004407800a5ebb700a0
:10c2e000a4be200014427800e14f42000800320052
:10c2f000a4be20001442780004407800505502008b
:10c300000000000000c2eb0004407800eaebb70038
:10c3100014002000645f880009003700000000005e
:10c320000700370000000000050037000000000093
:10c33000030037000000000001003700000000008b
:10c340000002eb00040078000080fa000000060004
:10c350000600fa00200798002e029000040f7800d3
:10c3600001003700000000001e02780094427800af
:10c37000254798001e0fe8002e429000e04f520023
:10c3800010003200ae429000e4c2b30084cf5200ed
:10c390000c003200ae429000f4c2b30084cf5200d1
:10c3a00008003200ae429000c4c2b30084cf5200f5
:10c3b00004003200ae429000e4c3b30084cf5200c8
:10c3c000e9ff3a001e027800844278002e029000b5
:10c3d0000442780004c252000442e9003447980045
:10c3e0003e409000f4550200000000003e429000e4
:10c3f0000482fb00840078002e0090002456020086
:10c4000000000000000278000402e800ae02900084
:10c4100004824200240798002e429000e04f520010
:10c420000c003200ae429000f4c2b30084cf520040
:10c4300008003200ae429000c4c2b30084cf520064
:10c4400004003200ae429000e4c3b30084cf520037
:10c45000c4ff3a000040eb00f45502000000000069
:10c460000080fa00000006000200fa000e007800ca
:10c47000a85702000000000000027800e00f520000
:10c48000150032001e4278008482fb00040c20005c
:10c4900084826200040c2000848f520004003a0061
:10c4a0000e007800a8570200000000000d003700c1
:10c4b0001e427800e04f5200090032001e42780010
:10c4c0000482fb00840078000000eb00dc570200cf
:10c4d00000000000e5ff3700000000000100370009
:10c4e000000000000080fa00000006000a00fa00c8
:10c4f0003007980041079800745f8000855f8000d6
:10c5000014079800250798003e029000ce02900084
:10c51000e00f5200e08f5a0004003a00140020009f
:10c520000500200034079800450798003e0290005f
:10c53000ce029000745f8800855f88000042eb00a7
:10c54000044f780002003700090007001e4fe80082
:10c550001e427800ef4f5200fbff36001e02900093
:10c56000ae0290000400be000080fa000000060049
:10c570000200fa000042eb00044f78002b00370065
:10c58000745f8000855f80008500d1000480d30047
:10c59000765f8000875f8000140020000500200087
:10c5a000060178000703780084037800050278000c
:10c5b000070161000402630005002000c022dd00c5
:10c5c000040020000403be006112b80004037300dd
:10c5d0008583730060031300e0831b0014002000b8
:10c5e00005002d0006017800070378008403780019
:10c5f00005027800070161000402630005002000c5
:10c60000c022dd00040020000403be006112b80057
:10c610000403730085837300060268008782680044
:10c62000745f8800855f88001e4fe8001e42780016
:10c63000ee4f5200d2ff3600745f8000855f8000ad
:10c6400004027800040078000080fa000000060070
:10c650001a00fa00881f7800041980004407980027
:10c66000141980005407980024198000640798006a
:10c67000240880007407980014088000040f9800b4
:10c680000002eb000419880004f029002419880036
:10c69000f403200014198800440e280004198800af
:10c6a00004002800240888000082eb001408880099
:10c6b0000042eb00044f78006022b8002407980085
:10c6c000350798000002eb0014079800a8ff070048
:10c6d0000002780005002000340f9800450f9800f4
:10c6e00001003700000000000060fe0000000000b4
:10c6f000250480000400220004826200e00f520042
:10c70000fbff320004088000140f98000002eb00c9
:10c710000408880085a0a90095ff070000027800a2
:10c72000240f98001e0a9000050020002e039000a0
:10c73000be0390000602420087824a002407980048
:10c74000350798002e039000be039000f43f2200ae
:10c75000450f2000840f5300858f5b000b003600cf
:10c760003e0c900082ff07000002780004026c007b
:10c77000340f98004e0c90007dff070000027800f7
:10c7800004026c00440f9800240037009e029000c1
:10c790001e0a9000848f520002003a000000000040
:10c7a000d1ff37009e0290001e0a90008482520042
:10c7b0002e0a900004824200050020000400be0002
:10c7c0004aff07001e0a9000140798003e0a9000d6
:10c7d000ce0a90000402420085824a00340f98007d
:10c7e000450f980062ff070000027800050820004e
:10c7f00005026200e00f5200030032003e0a900082
:10c800000400a000340f98001e4fe8001e4278007c
:10c81000e04f5200b3ff3a00000000000002eb00be
:10c82000041988006e029000241988005e029000ae
:10c83000141988004e029000041988007e029000ae
:10c84000240888000e0a9000140888003e0a900010
:10c85000ce0a90000400be004f0478000080fa0069
:10c86000000006000c00fa004007980051079800ed
:10c870000042eb00044f78000042eb0014479800a0
:10c880006022b80024079800350798007000370030
:10c890001e429000e34f52007b003e00ae429000eb
:10c8a00004cdb30004c24200244798001e42780021
:10c8b000e04f520005003a002e429000e94f52002e
:10c8c000580036000002eb00a20037001e4278003c
:10c8d000e34f520028003a002e429000e24f4200ff
:10c8e000020032000002eb009a0037002e03900095
:10c8f000be0390005450200025002000840f5300f8
:10c90000858f5b00020036000002eb0091003700cb
:10c910001e4290008483fb006e429000450620007a
:10c9200005a2b90004027800044378005e4290003a
:10c930006a22b9000402780004427800844243006d
:10c940004e42900004c24200de0290008782420004
:10c95000844a78001e4290000442e8001447980080
:10c960000042eb00044f78006022b80024079800d2
:10c9700035079800360037002e429000e24f420003
:10c9800023003a002e039000be0390005450200074
:10c9900025002000840f5300858f5b0002003600c5
:10c9a0000002eb006b0037001e4290008483fb0006
:10c9b0006e4290004506200005a2b90004027800ee
:10c9c000044378005e4290006a22b90004027800b5
:10c9d00004427800844243004e42900004c2420068
:10c9e000de02900087824200844a78001e42900056
:10c9f0000442e800144798000042eb00044f78001e
:10ca00006022b8002407980035079800100037000e
:10ca10002e429000e94f5200020036000002eb0067
:10ca20004c0037001e4fe8002e039000be0390001c
:10ca3000483add00c832de00850272004832dd006f
:10ca400024079800350798002e429000444798002c
:10ca50004e02900094427800254798002e429000a4
:10ca60000482fb000402ea004f22de000442780048
:10ca7000ce0290008502e80045079800e04f520082
:10ca800083ff3a0001003700000000002e429000b2
:10ca9000e04f520017003200ae429000f4c2b300e3
:10caa00084cf5200130032002e429000ed4f52000e
:10cab000100032002e429000ea4f52000d0032006a
:10cac000ae42900004c2b30084cf5200090032008d
:10cad0002e429000e94f520006003200ae42900014
:10cae000a4c3b30084cf5200020032000002eb0066
:10caf000180037002e039000be0390005450200011
:10cb000025002000840f5300858f5b000200360053
:10cb10000002eb000f0037006e4290004506200037
:10cb200005a2b90004027800044378005e42900038
:10cb30006a22b9000402780004427800844243006b
:10cb40004e42900004c24200de029000b4429800bf
:10cb500014002000040078000080fa0000000600a5
:10cb60000c00fa0040079800510798000002eb0003
:10cb7000240798004e029000e00f52002d00320072
:10cb80000042eb00044f7800047122001407980063
:10cb900024003700ce0290001e0290001100090010
:10cba0008482d80000027800340798003e0290008a
:10cbb000e00f520003003a002e029000e00f5200f6
:10cbc000110032003e029000044278000443b0009d
:10cbd000de029000844a78005e0290000402e800c1
:10cbe00054079800be0290001e02900004aab900eb
:10cbf00004027800ce02900004825200440798009c
:10cc000014002000240798009e029000a400200039
:10cc1000110009008482d8000002780014079800ef
:10cc20001e4fe8001e427800e44f5200d9ff360044
:10cc300006003700de02900004c3b300844a780087
:10cc40005e0290000402e80054079800de029000a3
:10cc50000042eb00844a78000080fa0000000600e1
:10cc60000200fa00000f78009e42900064c4b300f6
:10cc700084cf5200040036009e42900004ceb300e0
:10cc800004c24200144798009e42780064c4b30076
:10cc900084cf5200040036009e42780004ceb300d8
:10cca00004c24200044f78009e42900094c3b30037
:10ccb00084cf5200050036009e42900094ccb30011
:10ccc00004c2420014479800040037009e429000be
:10ccd00004cdb30004c24200144798009e4278007d
:10cce00094c3b30084cf5200050036009e42780002
:10ccf00094ccb30004c24200044f78000400370013
:10cd00009e42780004cdb30004c24200044f780074
:10cd10001e4290000482fb004422dd008442780021
:10cd20001e42780004c27200044078000080fa00bd
:10cd3000000006000200fa00004f78009e427800d2
:10cd40000582fb004422de00044f78001e4278007a
:10cd5000e94f52000300360075c3b3001ec2420003
:10cd60000200370005c3b3001ec242000440780031
:10cd70000080fa00000006000200fa00004f780070
:10cd80001e4278006f4f62001e427800e94f520049
:10cd90000300360075c3b3001ec242000200370014
:10cda00005c3b3001ec24200044078000080fa00b0
:10cdb000000006000600fa001007980021079800fe
:10cdc0001e029000144f78002e02900094427800ca
:10cdd000154798002d00370004c6b3009e42780026
:10cde00084cf520006003600a4c7b3009e427800ec
:10cdf00084cf520002003e0004ceb3001e4f42001a
:10ce00009e42900004c6b30084cf52000800360052
:10ce10009e429000a4c7b30084cf520004003e009d
:10ce20009e42900004ceb30004c242001447980012
:10ce30001e4290009e42780084cf520002003600cd
:10ce400014c0b300240037001e4290009e427800b8
:10ce500084cf52000200310000c2eb001e003700f8
:10ce60001e0290000402e800140798002e029000b1
:10ce70000402e800240798001e029000144f780076
:10ce80002e02900094427800154798001e427800c8
:10ce9000e04f5200030032001e429000e04f52006b
:10cea000cdff3a001e4290009e42780084cf52008f
:10ceb0000200360014c0b300070037001e42900085
:10cec0009e42780084cf52000200310000c2eb0085
:10ced000010037000042eb00044078000080fa00b7
:10cee000000006000600fa00200798002e029000bd
:10cef000140798003e429000044f78002e429000a4
:10cf0000344798001e427800244798001e02900083
:10cf1000040078000080fa00000006000400fa0017
:10cf2000008fbe000e0378000e0278009442780055
:10cf30000e0278003442900004c26a00044b78006c
:10cf40000e0378000e027800b44290000e027800c2
:10cf50001442780004c26a00344398000e0378003b
:10cf60000e027800944278000e027800344290005d
:10cf700004c26a00044b78000e0378000e027800a9
:10cf8000944290000e0278002442900004c26a008d
:10cf9000144398000e0378000e027800a44290001b
:10cfa0000e0278001442900004c26a0024439800e4
:10cfb0000e0378000e027800944290000e02780072
:10cfc0002442900004c26a00144398001e02be006e
:10cfd0000400be000080fa00000006000c00fa0009
:10cfe00040079800510798005e0290000402d100ab
:10cff000040f78004e029000140798006022b800d9
:10d0000024079800350798000c0037002e03900085
:10d01000be0390001e02900014027800050020005c
:10d020000602420087824a002407980035079800cc
:10d030001e0290000482e800140798001e02780087
:10d0400004f0a7000402ea000402ea004f22de0016
:10d05000044278001e0fe900e04f5200ebff3a0057
:10d060005e0290006102620004427800e04f5200cc
:10d070000a0032002e039000be0390001e029000b2
:10d08000144278000482fb000500200006024200e2
:10d0900087824a0024079800350798002e029000e6
:10d0a0006123b8003e029000050020000602420005
:10d0b00087824a002407980035079800ae02900046
:10d0c0003e02900004824200240798002e02900045
:10d0d0000482ea00040078000080fa0000000600e4
:10d0e0000600fa00200798002e029000040f780036
:10d0f00010003700ae42900004c6b30084cf520047
:10d100000b003400ae429000a4c7b30084cf52009d
:10d1100007003c001e027800144278008442780028
:10d1200004ceb30004c242009e027800844a780014
:10d130001e0fe8001e0278009442780025479800f0
:10d140002e429000e04f5200eaff3a002e0290007b
:10d15000040078000080fa00000006000400fa00d5
:10d16000100798001e029000ef0242000042eb0000
:10d17000844a78001e02900004007800d8ff07005f
:10d180000042eb00044f7800140037009e42780004
:10d190000582fb009e029000048242001442780047
:10d1a000e04f52000c003a00070037009e42780022
:10d1b0000582fb009e0290008482420004c2b300fc
:10d1c000844a78001e4fe8001e427800ee4f52005d
:10d1d000f6ff3600040037001e4fe8001e427800bc
:10d1e000ee4f5200e9ff36000080fa000000060012
:10d1f0000800fa001007980021079800624798007d
:10d20000130037001e029000144f78001e02900099
:10d210000402e800140798001e427800e04f520014
:10d2200002003a000002eb00150037006e42900049
:10d230009e42780084cf520005003a001e02900002
:10d240000402e900140798001e0290000c00370049
:10d250002e02900004f0a7000402ea000402ea0093
:10d260004f22de0004427800ae0290008502e90001
:10d2700025079800e04f5200e2ff3a000002eb0061
:10d28000040078000080fa00000006000c00fa009c
:10d290004007980051079800ce0290000042eb0032
:10d2a000844a78005e0290000402e900ce029000f9
:10d2b0000482420024079800ae0290000042eb0076
:10d2c000844a78000002eb001407980068025700b7
:10d2d000040f78001d0037002e02900014427800e1
:10d2e000e04f5200030032005e02900014079800e5
:10d2f000210037001e8fe9001e027800940278009a
:10d3000035079800de0290001e02900084825200d1
:10d310004e0390001e0290000402430005017800b5
:10d32000be00900004007800f40b02000000000032
:10d330003e009000160c0200000000000002780081
:10d340009e02900004824200140798004eba970093
:10d3500004f0a7000402ea000402ea004f22de0003
:10d3600004427800ceba97008502e90045bf9f00cd
:10d37000e04f5200d8ff3a001e02900004007800ef
:10d380000080fa00000006000000fa00d8760200d3
:10d390000000000000027800040078000080fa001d
:10d3a000000006000000fa00e27602000000000023
:10d3b00000027800040078000080fa0000000600f7
:10d3c0000a00fa0040479800310798004207980089
:10d3d0000042eb00244798000e82e800be01900056
:10d3e0000e017800ce0090004e409000de790200e1
:10d3f0000000000000027800e00f520002003a0036
:10d400002e4290000c0037001e027800be029000f1
:10d4100004824200340798001e027800ce02900079
:10d4200004825200440798004e029000e00f520020
:10d43000e9ff3a002e429000044078000080fa0094
:10d44000000006007a02fa00842720000e02420043
:10d45000004a7800252120008e8242000042eb0025
:10d46000844a78000e82e800852720008e824200e0
:10d47000720020008400780015407800d0ff07007b
:10d4800000427800252120008e824200844a7800e4
:10d49000242120000e02420014427800e04f520086
:10d4a00017003200242120000e02420014427800ae
:10d4b0008482fb00342120000e024200851f780088
:10d4c000a5292900851f780004007800240c02009b
:10d4d00000000000e4875700342120000e024200c3
:10d4e000852720008e8242000401780011c0b3001d
:10d4f00015407800b27a020000000000600037009a
:10d500002e029000e00f520014003200ae02900094
:10d51000342120000e024200851f7800252e2900ac
:10d52000851f780004007800240c02000000000031
:10d53000e4875700342120000e0242008527200096
:10d540008e8242000401780011c0b30015407800bb
:10d55000b27a020000000000490037003e0290004d
:10d56000c822dd004822de00050272003407980060
:10d570000e82e800852720008e8242008400780019
:10d5800015407800b20007000042780025212000f5
:10d590008e824200844a7800242120000e0242003c
:10d5a00014427800e04f520035003a008510200008
:10d5b0008e8242000e82e800862720000e03430080
:10d5c00005017800840078001640780032000700da
:10d5d000e42020000e024200144278000482fb0086
:10d5e000670f4200871020008e8343002421200013
:10d5f0000e024200052120008e8242008627200074
:10d600000e03430087017800050178009e00780032
:10d6100016407800387a020000000000000278000e
:10d62000e00f520016003a00242120000e024200b2
:10d63000144278008482fb00342120000e02420054
:10d64000851f7800d5322900851f780004007800f6
:10d65000240c020000000000e48757003421200061
:10d660000e024200852720008e82420004017800cd
:10d6700011c0b30015407800b27a0200000000002b
:10d68000242120000e024200144278000440780059
:10d690000080fa00000006000800fa002047980009
:10d6a00021079800320798000042eb00044f7800f1
:10d6b0002e029000744290000482fb006123b900a6
:10d6c0000082eb008082eb000602420087824a0063
:10d6d000f600200007002000860f5200878f5a00b6
:10d6e0002d003e00046001000f0037000e003700df
:10d6f0001400370013003700190037001f003700ef
:10d7000025003700240037002300370022003700af
:10d7100021003700200037001f0037001e003700af
:10d720000f003700150037003e019000ae0090005a
:10d730002e4090007e00070000427800044f7800e1
:10d74000180037003e019000ae0090002e4090007f
:10d750007b01070000427800044f78001100370079
:10d760003e019000ae0090002e409000d6000700d1
:10d7700000427800044f78000a0037003e01900014
:10d78000ae0090002e409000ca01070000427800d1
:10d79000044f78000300370014c0b300044f780032
:10d7a000000000001e427800e04f52000c003200e2
:10d7b0002e029000f442900004c8b30004c272002c
:10d7c000be029000f44298003e0290009e42780013
:10d7d000054a9800be02900024c0b300e4429a00bb
:10d7e0002e02900064429000be029000e442980035
:10d7f0003e029000ae029000351a780025127800a3
:10d8000025039000260298003e0290006442920098
:10d810000482fb000402e800840278003e029000cb
:10d82000250298003e02900024029000c822dd00ec
:10d830004822de0005027200be029000a402980099
:10d840000042eb00044078000080fa00000006006f
:10d850006c00fa0000ef9800513798000042eb008e
:10d86000044f78005e329000240290000402e90028
:10d87000140798009e02900004102000848f52002c
:10d880000c00360084c0b300044f780052362900e3
:10d8900011c0b3000ee89000b27a02000000000050
:10d8a0005e3190009e0090000ee890000302070099
:10d8b0001b0037005e329000670242001e0190009c
:10d8c000840078000ee89000bdfe0700004278005a
:10d8d000044f78001e427800e04f520010003200e2
:10d8e0001e4278008482fb0064024700851f780096
:10d8f00095392900851f780004007800240c020067
:10d9000000000000e487570064024700040178002b
:10d9100011c0b3000ee89000b27a020000000000cf
:10d920001e427800044078000080fa0000000600e3
:10d930000c00fa00604798004107980052079800d1
:10d940004e029000044a90000482fb004822dd0051
:10d95000140798004e029000144a90000482fb00c5
:10d960009e02900004827200140798004e029000fc
:10d97000244a90000482fb004822dd00240798001e
:10d980004e029000344a90000482fb00ae029000e8
:10d9900004827200240798002e029000e00f5200cb
:10d9a00043003200ae02900004042000848f520035
:10d9b0003f003e004e029000744390004e029000e3
:10d9c000e44290002e0290009e01900006417800f3
:10d9d000ee4090000540780004770200000000004f
:10d9e00000027800e10f52002e003a005e02900023
:10d9f00069024200ce029000f5439000ce029000f2
:10da000065439000840278002e0290009e019000f1
:10da100007417800ee40900006407800dc77020075
:10da20000000000000427800044f78001e42780099
:10da3000e04f520018003a004e02900074429000ed
:10da4000de029000f44298002e0290004322de0095
:10da500004427800de029000844a98002e02900072
:10da600067026200e00f5200050032005e02900083
:10da7000044a90000442e800de029000844a9800c4
:10da80005e029000044a900004c2e800de029000aa
:10da9000e4429a000800370044c0b300044f780005
:10daa0000500370024c0b300044f7800020037009f
:10dab00034c0b300044f78001e4278000440780060
:10dac0000080fa00000006001200fa00404f9800a3
:10dad00071079800020f98000042eb00044f780095
:10dae00014002000340798007e029000044a900041
:10daf0000482fb004822dd00440798007e0290006b
:10db0000144a90000482fb00ce029000048272004e
:10db1000440798007e02900074429000ef4f52003c
:10db20002b003a007e029000244a90000482fb0001
:10db30004822dd00340798007e029000344a9000ad
:10db40000482fb00be029000048272003407980039
:10db50003e029000e00f520004003200be0290002e
:10db600004042000848f52000300360034c0b30048
:10db7000044f7800300037003e0290004322de0060
:10db8000244798003e02900067026200e00f5200b6
:10db9000030032002e4290000442e800244798001f
:10dba0007e029000c44a90002e42900084cf520022
:10dbb0000300320034c0b300044f78001e00370069
:10dbc0007e0290006d024200240798001a00370080
:10dbd0007e029000244a9000e04f520007003a0075
:10dbe0007e029000344a9000e04f520003003a0059
:10dbf0000042eb00244f98000d0037007e02900099
:10dc0000244a9000e14f420007003a007e02900053
:10dc1000344a9000e04f520003003a0014c0b300b1
:10dc2000244f98000200370034c0b300044f78003e
:10dc30006a024700240798001e427800e04f520015
:10dc40003b003a007e029000744390007e029000f8
:10dc5000e44290003e029000ce0190000641780020
:10dc6000ce489000054078000477020000000000d4
:10dc700000027800e10f52002b003a007e02900073
:10dc8000f44390007e02900064439000ae02900046
:10dc90003e029000ce01900007417800ce489000ef
:10dca000064078005e790200000000000042780023
:10dcb000044f78001e427800e04f520017003a00ef
:10dcc00014c0b300144798000d0037001e429000a6
:10dcd0008482fb001e4290000482fb007e039000c1
:10dce0006602420066427a000e0b900085024300f5
:10dcf000e44298001e4290000442e8001447980055
:10dd00001e429000e54f5200f0ff36008e0a900050
:10dd100054c0b300e4429a000500370044c0b30089
:10dd2000044f78000200370024c0b300044f78008d
:10dd30001e427800044078000080fa0000000600cf
:10dd40000c00fa00604798004107980052079800bd
:10dd50004e029000044a90000482fb004822dd003d
:10dd6000140798004e029000144a90000482fb00b1
:10dd70009e02900004827200140798004e029000e8
:10dd8000244a90000482fb004822dd00240798000a
:10dd90004e029000344a90000482fb00ae029000d4
:10dda00004827200240798002e029000e00f5200b7
:10ddb0003a003200ae02900004022000848f52002c
:10ddc00036003e004e029000744390004e029000d8
:10ddd000e44290002e0290009e01900006417800df
:10dde000ee4090000540780004770200000000003b
:10ddf00000027800e10f520025003a005e02900018
:10de000069024200ce029000f5439000ce029000dd
:10de100065439000840278002e0290009e019000dd
:10de200007417800ee40900006407800dc77020061
:10de30000000000000427800044f78001e42780085
:10de4000e04f52000f003a004e02900074429000e2
:10de5000de029000f44298002e0290000442780006
:10de600004424200de029000844a98005e02900064
:10de7000044a900004c2e800de029000e4429a00e6
:10de80000800370044c0b300044f78000500370095
:10de900024c0b300044f78000200370034c0b30040
:10dea000044f78001e427800044078000080fa0099
:10deb000000006000e00fa00004f9800510798007d
:10dec000620798000042eb00044f780044c0b300a2
:10ded0002447980014002000240798005e02900058
:10dee000044a90000482fb004822dd0034079800b9
:10def0005e029000144a90000482fb00be02900073
:10df000004827200340798005e0290007442900010
:10df1000f04f520022003a005e029000244a900026
:10df20000482fb004822dd00240798005e02900076
:10df3000344a90000482fb00ae029000048272001a
:10df4000240798002e029000e00f520004003200d7
:10df5000ae02900004042000848f520003003600bb
:10df600034c0b300044f78000d0037002e0290003b
:10df700004024200840278005e029000444a90004d
:10df80000482fb00848f52000300320034c0b300cf
:10df9000044f78000200370074c0b3002447980093
:10dfa0001e427800e04f520040003a005e029000ae
:10dfb000744390005e029000e44290002e029000b4
:10dfc000be019000064178008e4890000540780020
:10dfd000047702000000000000027800e10f520008
:10dfe00030003a005e029000e60242002e429000ad
:10dff0000482fb0004824200de029000f5439000a0
:10e00000de02900065439000840278002e029000aa
:10e01000be019000074178008e48900006407800cd
:10e020005e7902000000000000427800044f780092
:10e030001e427800e04f520017003a0014c0b300af
:10e04000144798000d0037001e4290008482fb00a8
:10e050001e4290000482fb005e03900066024200b4
:10e0600066427a006e03900085024300e442980005
:10e070001e4290000442e800144798001e4290009f
:10e08000e54f5200f0ff3600ee02900054c0b3009e
:10e09000e4429a000500370044c0b300044f780002
:10e0a0000200370024c0b300044f78001e427800fd
:10e0b000044078000080fa00000006000a00fa0020
:10e0c0004047980031079800420798000002eb0093
:10e0d000040f78000002eb00040f78000600370000
:10e0e0000e82e80012002000840078004e4090006c
:10e0f000b3fc07001e0fe8003e0290009e0278006d
:10e10000848f5200f6ff39000080fa0000000600fc
:10e110000e00fa0040079800510798006207980027
:10e120006022b80024079800350798006e0290001e
:10e130004322de00044f78006e0290006702620006
:10e14000e00f5200010032001e4fe8000042eb00d9
:10e1500014479800340037001e4290000482fb00f0
:10e16000de029000848242000042eb00844a780084
:10e170000042eb0024479800250037001e42900023
:10e180000482fb00de029000048342001e429000e5
:10e190000482fb00de0290000482420014427800f8
:10e1a000844278002e029000ce0390000482430047
:10e1b000144278008483fb002e4290000482fb000e
:10e1c000043add000442780004c27200044b780077
:10e1d0002e029000be02900061024200e0824a00de
:10e1e00024079800350798006e0290006123b8005c
:10e1f0002e029000be029000840f5300858f5b00ba
:10e200000d0036002e4290000442e800244798009a
:10e210002e429000e74f5200d8ff36001e42900079
:10e220000442e800144798001e4290009e4f52009e
:10e23000c9ff390001003700000000000080fa002b
:10e24000000006000c00fa00300798004107980013
:10e25000520798000042eb00044f78000042eb00a8
:10e26000144798000042eb00244798002b00370029
:10e2700014c0b300444798000042eb0034479800b4
:10e28000220037001e4290000482fb00ce02900064
:10e29000048342009e4278000582fb00be0290008b
:10e2a00004824200944278004e42900004c2620010
:10e2b0008482fb003e4290000482fb0004aade0040
:10e2c00004427800044b78001e4290000442e800ab
:10e2d000144798004e429000044242004447980080
:10e2e0002e4290000442e800244798002e429000fd
:10e2f0008482fb005e029000848f52000d0031008a
:10e300003e4290000442e800344798003e429000ac
:10e31000e74f5200dbff36001e4fe8002e42900010
:10e320008482fb005e029000848f5200d0ff39008f
:10e3300001003700000000000080fa000000060025
:10e340000c00fa0020079800310798004207980057
:10e35000530798000042eb00144798000042eb007e
:10e36000244798000042eb00044f78002300370058
:10e370002e4290000482fb00be0290008482420084
:10e380001e4290000482fb00040242002e03900013
:10e3900004024300140278004822de0004427800a0
:10e3a000844a78002e4290000442e80024479800f6
:10e3b0002e4290000482fb00be0290008482420044
:10e3c0001e4290000482fb00040242002e039000d3
:10e3d000040243001402780004427800844a780062
:10e3e0002e4290000442e800244798001e4290000c
:10e3f0000442e800144798001e4fe8001e427800cf
:10e400000483fb00070020004e029000de02900013
:10e41000840f5300858f5b00d5ff39000080fa0020
:10e42000000006000c00fa00200798003107980051
:10e4300042079800530798000042eb0014479800e9
:10e440000042eb00244798000042eb00044f7800a4
:10e45000660037002e4290000482fb00be0290004e
:10e46000048042001e4290000482fb004222dd0034
:10e47000ae029000048242001403be0004f02f009c
:10e4800005002000860078000703780084037800e8
:10e490000502780087806000040263000500200008
:10e4a000c022dd00040020000403be00610ab800a1
:10e4b0000403730085837300c838dd004832de0032
:10e4c00004827000c83ade000442780004487800f4
:10e4d0002e4290000442e800244798002e4290000b
:10e4e0000482fb00be029000048342001e429000a2
:10e4f0000482fb004222dd00ae0290000482420052
:10e500001402be0004427800044b78002e429000b2
:10e510000442e800244798002e4290000482fb0049
:10e52000be029000048342001e4290000482fb0061
:10e530004222dd00ae029000048242001402be00be
:10e54000482ade000500200004427800044b7800d1
:10e550002e4290000442e800244798002e4290008a
:10e560000482fb00be029000048042001e42900024
:10e570000482fb004222dd00ae02900004824200d1
:10e580001403be0004002000f50f20008600780070
:10e590000703780084037800050278008780600014
:10e5a0000402630005002000c022dd0004002000fa
:10e5b0000403be00610ab80004037300858373007e
:10e5c000403ade000500200004427800044878004c
:10e5d0002e4290000442e800244798001e4290001a
:10e5e0000442e800144798001e4fe8001e427800dd
:10e5f0000483fb00070020004e029000de02900022
:10e60000840f5300858f5b0092ff39000080fa0071
:10e61000000006001000fa0040079800510798001b
:10e6200062079800730798000042eb0014479800b7
:10e630000042eb00244798000042eb00044f7800b2
:10e64000610037001e4290000482fb004222dd0080
:10e65000ce02900084824200640247004200200003
:10e660008500780004007800d80b0200000000004c
:10e670002e4290000482fb00de02900004804200e3
:10e680002e039000be03900004f02f000500200030
:10e69000860078000703780084037800050278007c
:10e6a000878060000402630005002000c022dd00b6
:10e6b000040020000403be00610ab80004037300d4
:10e6c00085837300c838dd004832de0004827000a4
:10e6d000c83ade0004427800044878002e429000d8
:10e6e0000442e800244798002e4290000482fb0078
:10e6f000de029000048342002e029000be029000d1
:10e7000004427800044b78002e4290000442e80056
:10e71000244798002e4290000482fb00de02900005
:10e72000048342002e029000be029000482ade00c0
:10e730000500200004427800044b78002e4290002f
:10e740000442e800244798002e4290000482fb0017
:10e75000de029000048042002e039000be03900071
:10e7600004002000f50f20008600780007037800e1
:10e77000840378000502780087806000040263004b
:10e7800005002000c022dd00040020000403be00bc
:10e79000610ab8000403730085837300403ade0009
:10e7a0000500200004427800044878002e429000c2
:10e7b0000442e800244798001e4290000442e8000a
:10e7c000144798001e4fe8001e4278000483fb00a7
:10e7d000070020006e029000fe029000840f53009c
:10e7e000858f5b0097ff39000080fa00000006006b
:10e7f0000c00fa00200798003107980042079800a3
:10e80000530798000042eb00144798000042eb00c9
:10e81000244798000042eb00044f780011003700b5
:10e820002e4290000482fb00be02900084824200cf
:10e830001e4290000482fb002e039000040243005d
:10e8400014427800844a78002e4290000442e80086
:10e85000244798001e4290000442e80014479800a4
:10e860001e4fe8001e4278000483fb0007002000d2
:10e870004e029000de0290000402420085824a00af
:10e88000840f5300858f5b00e5ff39000080fa009c
:10e89000000006000c00fa002007980031079800dd
:10e8a00042079800530798000042eb001447980075
:10e8b0000042eb00244798000042eb00044f780030
:10e8c000280037002e4290000482fb000402420020
:10e8d000be029000848242001e4290000482fb002f
:10e8e0002e03900004024300144278000482fb00cf
:10e8f0004822dd00840a78002e4290000482fb004a
:10e9000004024200be029000848242002e42900027
:10e910000482fb00040242003e0390000402430014
:10e92000140378001e4290000482fb000402e800f9
:10e93000ae03900004824300144278000482fb007e
:10e9400004027300840a78002e4290000442e8001a
:10e95000244798001e42900004c2e8001447980023
:10e960001e4fe8001e4278000483fb0007002000d1
:10e970004e029000de029000840f5300858f5b00f2
:10e98000d0ff39000080fa00000006000c00fa00f9
:10e990002007980031079800420798005307980015
:10e9a0000042eb00144798000042eb002447980017
:10e9b0000042eb00044f7800610037002e429000c7
:10e9c0000482fb004222dd00be029000048342006c
:10e9d0001e4290000482fb00ae02900004824200be
:10e9e000144278000482fb004822dd00cfa2de0042
:10e9f000048bbe001e4290000442e80014479800b9
:10ea00002e4290000482fb004222dd00be029000f4
:10ea1000048042002e4290000482fb004222dd006e
:10ea2000be029000048242001403be001e42900009
:10ea30000482fb00ae02900004824200144278007f
:10ea40000482fb000500200004027300858273002d
:10ea50000488be001e4290000442e800144798005b
:10ea60002e4290000482fb004222dd00be02900094
:10ea7000048042002e4290000482fb004222dd000e
:10ea8000be029000048242001403be001e429000a9
:10ea90000482fb00ae02900004824200144278001f
:10eaa0000482fb0005002000c822dd0004002000d5
:10eab00004027300858273000488be001e42900029
:10eac0000442e800144798002e4290000482fb00a4
:10ead0004222dd00be029000048042002e429000df
:10eae0000482fb004222dd00be029000048242004c
:10eaf0001403be001e4290000482fb00ae02900090
:10eb000004824200144278000482fb0005002000c9
:10eb1000c022dd000400200004027300858273001f
:10eb20000488be001e4290000442e800144798008a
:10eb30002e4290000442e800244798001e4fe8004f
:10eb40001e4278000483fb00070020004e02900064
:10eb5000de029000840f5300858f5b0097ff390021
:10eb60000080fa00000006001000fa00400798003c
:10eb70005107980062079800730798000042eb0065
:10eb8000144798000042eb00244798000042eb0035
:10eb9000044f7800530037006022b8002407980023
:10eba000350798001e4290000482fb00ce029000c0
:10ebb00004824200144278000482fb004822dd00f7
:10ebc000cfa2de0024079800350798001e4290006f
:10ebd0000442e800144798001e4290000482fb00a3
:10ebe000ce02900004824200144278000483fb00ad
:10ebf000070020002e029000be0290000402730065
:10ec00008582730024079800350798001e42900003
:10ec10000442e800144798001e4290000482fb0062
:10ec2000ce02900004824200144278000482fb006d
:10ec300005002000c823dd00060020002e02900001
:10ec4000be029000040273008582730024079800be
:10ec5000350798001e4290000442e80014479800cf
:10ec60001e4290000482fb00ce029000048242000b
:10ec7000144278000482fb0005002000c023dd0060
:10ec8000060020002e029000be02900004027300d5
:10ec90008582730024079800350798001e42900073
:10eca0000442e800144798002e4290000482fb00c2
:10ecb0004222dd00de02900004824200e4024700ae
:10ecc000420020008500780004007800d80b020084
:10ecd000000000002e4290000442e8002447980003
:10ece0001e4fe8001e4278000483fb00070020004e
:10ecf0006e029000fe029000840f5300858f5b002f
:10ed0000a5ff39000080fa00000006000c00fa00a0
:10ed10002007980031079800420798005307980091
:10ed20000042eb00144798000042eb002447980093
:10ed30000042eb00044f7800110037002e42900093
:10ed40000482fb00be029000848242001e429000ba
:10ed50000482fb002e03900004024300144278005a
:10ed6000844a78002e4290000442e800244798002c
:10ed70001e4290000442e800144798001e4fe8002d
:10ed80001e4278000483fb00070020004e02900022
:10ed9000de0290000402420085824a00840f530084
:10eda000858f5b00e5ff39000080fa000000060057
:10edb0000000fa0014002000040078000080fa002f
:10edc000000006000000fa00140020000400780093
:10edd0000080fa00000006000200fa00004f7800f0
:10ede000114798001e427800e14f520002003a009d
:10edf00014002000010037000002eb00040078003e
:10ee00000080fa00000006000a00fa00204798007f
:10ee1000314798004247980033079800440798000c
:10ee20004e4290000482fb006123b9000082eb0097
:10ee30008082eb000602420087824a00f600200032
:10ee400007002000860f5200878f5a0053003e00b3
:10ee5000046001000f00370019003700230037005d
:10ee60002d00370037003700410037004b003700d6
:10ee70004a00370049003700480037004700370094
:10ee80004600370045003700440037002d003700aa
:10ee900037003700be0290004e029000048242000c
:10eea000f00f5200030036000002eb00040f780060
:10eeb0003d00370014002000040f78003a003700ae
:10eec000be0290004e02900004824200f00f5200f9
:10eed000030036000002eb00040f78003200370018
:10eee00014002000040f78002f003700be029000ad
:10eef0004e02900004824200ea0f520003003600e6
:10ef00000002eb00040f78002700370014002000f7
:10ef1000040f780024003700be0290004e029000db
:10ef200004824200ea0f5200030036000002eb00a8
:10ef3000040f78001c00370014002000040f780034
:10ef400019003700be0290004e0290000482420079
:10ef5000f00f5200030036000002eb00040f7800af
:10ef60001100370014002000040f78000e00370055
:10ef7000be0290004e02900004824200ea0f52004e
:10ef8000030036000002eb00040f78000600370093
:10ef900014002000040f7800030037000002eb008b
:10efa000040f7800000000001e02780004007800c2
:10efb0000080fa00000006000e00fa0040479800aa
:10efc00051479800624798004307980054079800fb
:10efd000650798000418800004007800500c0200b7
:10efe000000000005e0c020000000000000278003b
:10eff000670262000508200004aade00040f780002
:10f000000002eb00140798006e4290000482fb009f
:10f010006123b9000082eb008082eb00060242000f
:10f0200087824a003600200007002000860f520029
:10f03000878f5a009d003e000460010003003700e6
:10f04000230037002b0037008a003700ce029000e3
:10f0500064a92000048242005e019000ee0090004e
:10f0600004007800887002000000000064a92000fd
:10f0700014427800e14f520008003a00c402a80090
:10f08000c422a800c442a800c462a800c482a80088
:10f09000c4a2a800c4c2a800c4e2a80064a92000b9
:10f0a00014427800e04f52007f003a00c402a900e9
:10f0b000c422a900c442a900c462a900c482a90054
:10f0c000c4a2a900c4c2a900c4e2a9007700370005
:10f0d000ce02900064aa2000048242005e019000eb
:10f0e000ee0090000400780088700200000000002c
:10f0f0006e0037005e029000050020004e03900075
:10f10000060343008603780066ab200006834300b5
:10f110000401be00ee00900006007800a07102001d
:10f120000000000004188000b4558800b455800029
:10f13000e00f520005003200b55580006409200040
:10f14000848f520001003e00c402a800b555800023
:10f1500064092000848f520007003600b5558000f6
:10f16000c4122000848f520003003e00c402a80095
:10f17000c422a80002003700c422a900c402a900ca
:10f18000b5558000c4122000848f5200080036005c
:10f19000b555800064222000848f520004003e0098
:10f1a000c402a800c422a800c442a800020037007c
:10f1b000c422a900c442a900b555800064222000e1
:10f1c000848f520009003600b5558000c42b200002
:10f1d000848f520005003e00c402a800c422a8008b
:10f1e000c442a800c462a80001003700c462a9009c
:10f1f000b5558000c42b2000848f52000b003600d0
:10f20000b5558000643b2000848f520007003e000b
:10f21000c402a800c422a800c442a800c462a80076
:10f22000c482a800c4a2a80002003700c482a900ba
:10f23000c4a2a900b5558000643b2000848f520011
:10f2400009003600c402a800c422a800c442a800d5
:10f25000c462a800c482a800c4a2a800c4c2a800b6
:10f26000c4e2a80011003700c4c2a900c4e2a9008a
:10f270000e0037005e029000050020004e03900053
:10f280000603430086037800a6ac200006834300f3
:10f290000401be00ee00900006007800a07102009c
:10f2a0000000000001003700000000000042eb00f9
:10f2b000044078000080fa00000006000a00fa000e
:10f2c000004f7800114798002247980023079800c4
:10f2d00034079800450798002e4290000482fb00f6
:10f2e0006123b900b4ff2f00f5ff2f000602420092
:10f2f00087824a00b600200007002000860f5200d7
:10f30000878f5a0023003e00046001000b00370085
:10f31000130037001f0037001e0037001d003700a4
:10f320001c0037001b0037001a0037001900370097
:10f33000180037000100370009003700ae029000c6
:10f3400064a92000048242003e01900084007800fd
:10f350004e00900022710200000000000d003700f6
:10f360003e029000050020002e039000060343009b
:10f370008603780066ab2000068343000401be00cc
:10f38000860078004e0090004a74020000000000e1
:10f39000000000000042eb00044078000080fa000a
:10f3a000000006000200fa00004f78001400200060
:10f3b000040078000080fa00000006000e00fa0049
:10f3c000404798003107980042079800530798007b
:10f3d0006407980014002000040f78000c820200db
:10f3e00000000000748402000000000064bf2000e0
:10f3f000144278003e019000de0090000440780046
:10f40000321c02000000000000027800140798007f
:10f4100064bf200014427800044078001e180200e7
:10f420000000000000027800e00f520006003a00e1
:10f43000ee02900094c0b300844a78000002eb0012
:10f44000040f7800060037009e0290004e029000e4
:10f45000050a7800ee0290000042eb00844a780032
:10f460001e027800040078000080fa000000060008
:10f470000e00fa00404798003107980042079800b4
:10f48000530798006407980014002000040f7800c8
:10f490000c820200000000007484020000000000e2
:10f4a00064bf2000144278003e019000de0090000e
:10f4b000044078003a1a02000000000000027800c0
:10f4c0001407980064bf20001442780004407800bc
:10f4d000281902000000000064bf200014427800d8
:10f4e000044078001e1802000000000000027800ae
:10f4f000e00f520006003a00ee02900094c0b30004
:10f50000844a78000002eb00040f78000600370000
:10f510009e0290004e029000050a7800ee029000d4
:10f520000042eb00844a78001e0278000400780054
:10f530000080fa00000006000200fa00004f780088
:10f5400064bf20001442780004407800e2180200f2
:10f550000000000014002000040078000080fa0081
:10f56000000006000400fa00004f780011479800e0
:10f57000120798001e009000148d02000000000089
:10f580000080fa00000006002600fa00600f9800d4
:10f59000710f98000217980013179800446798009d
:10f5a0004e6290000482fb003407980000c2eb001a
:10f5b0002457980000c2eb003457980000c2eb00bb
:10f5c0004457980000c2eb005457980000c2eb006b
:10f5d0006457980000c2eb00745798000e12900018
:10f5e0009e129000440f9800550f98006e0a9000ec
:10f5f000fe0a900074079800050f98000e0078002e
:10f600000400070000027800040078000080fa007f
:10f61000000006000200fa00000f78000000000061
:10f620006c3a02000000000000027800e00f520077
:10f63000fbff32000000eb00f03c02000000000085
:10f640001e02780015002000050a78001e027800ce
:10f6500005802000150298009e02780064c0b30067
:10f66000c44298009e02780044c0b300d44298007f
:10f670009e0278006882420062002000b1b0200043
:10f6800004007800d80b0200000000009e03780000
:10f69000e6ad2000164378000680fb00f6ad2000a2
:10f6a000164378000683fb004833dd000003730037
:10f6b0000602780006ae2000164378000680fb00a4
:10f6c00016ae2000164378000683fb004833dd00a9
:10f6d0000003730086027800f4039800850b9800fd
:10f6e0001e007800500107009e02780072824200de
:10f6f000c201200061c0b300040078002a3c02006f
:10f70000000000001e027800c10120000400780003
:10f710002c3f020000000000703c020000000000ce
:10f7200014002000040078000080fa0000000600a9
:10f730000000fa0000c2eb0004407800b0ebb70014
:10f7400000c2eb0004407800b1ebb70000c2eb0050
:10f7500004407800b2ebb70000c2eb000440780030
:10f76000b3ebb70000c2eb0004407800b4ebb70085
:10f7700000c2eb0004407800b5ebb7000082eb005c
:10f780008082eb00645d8800755d88000080fa006f
:10f79000000006001c00fa00b45d8000e00f52007b
:10f7a00003003200e10f5200480032005d003700d4
:10f7b0000e027800c101200004007800e23e020041
:10f7c00000000000843a0200000000000e007800f3
:10f7d000150107001e027800e10f520006003a00f2
:10f7e0004e429000e64f520003003a005e42900005
:10f7f000e44f520002003200140020004a0037009b
:10f800003e029000e20f52000c003a004e029000bf
:10f81000de029000845d8800955d8800ee02900015
:10f82000a55d88007e0290008e0a9000645d8800cd
:10f83000755d8800140020003b0037003e029000f8
:10f84000e10f520021003a004e0b9000de0b9000b9
:10f85000decabf008080fb00dfcabf000080fb0063
:10f860004800dd000100700000027800e0cabf001f
:10f870008080fb00e1cabf000080fb004800dd0083
:10f880000100700080027800840f5300858f5b00b8
:10f890000200320014002000230037007e02900096
:10f8a0008e0a9000c45d8800d55d88004e029000ed
:10f8b000de029000e45d8800f55d8800ee029000b5
:10f8c000055e880014002000b45d8800240020003c
:10f8d00034079800e45d8000f55d8000140f980007
:10f8e000250f9800055e8000350f9800c45d8000ec
:10f8f000d55d8000440f9800550f98000e007800e9
:10f9000044ff070000027800e00f520002003a00b6
:10f910000002eb00040037000002eb00b45d880039
:10f920000000000014002000040078000080fa00ad
:10f93000000006001e00fa00600f9800140020006e
:10f940003407980000c2eb002457980000c2eb0077
:10f950003457980000c2eb004457980000c2eb00f7
:10f960005457980000c2eb006457980000c2eb00a7
:10f9700074579800e6ad2000164378008683fb009c
:10f98000f6ad2000164378000683fb004833dd0007
:10f99000070373000602780006ae200016437800c5
:10f9a0008683fb0016ae2000164378000683fb001a
:10f9b0004833dd0007037300860278006e0b900069
:10f9c0001603be0006036a0087836a00e2cabf000e
:10f9d0008080fb00e3cabf000080fb004800dd0020
:10f9e0000100700000027800e4cabf008080fb00c4
:10f9f000e5cabf000080fb004800dd000100700088
:10fa000080027800060078000703780084037800fd
:10fa10000502780007006000040263000500200072
:10fa2000c022dd00040020000403be006102b80013
:10fa30000403730085837300e00f5300e08f5b00c5
:10fa40001500320066ae2000164378008683fb0066
:10fa500076ae2000164378000683fb004833dd00b5
:10fa6000070373000602780086ae20001643780074
:10fa70008683fb0096ae2000164378000683fb00c9
:10fa80004833dd000703730086027800440f9800b6
:10fa9000550f9800040037006e0a90001403be0052
:10faa000460f9800570f98000e007800d9fe070007
:10fab0000080fa00000006000400fa00000f780041
:10fac00011079800645d8000755d80001e0378005a
:10fad0001603be00860f5200878f5a00470032007f
:10fae000665d8000775d8000e6cabf008080fb0015
:10faf000e7cabf000080fb004800dd000100700085
:10fb000000027800e8cabf008080fb00e9cabf009d
:10fb10000080fb004800dd000100700080027800da
:10fb2000840f5300858f5b003b003a00e6ad200058
:10fb3000164378008683fb00f6ad2000164378005c
:10fb40000683fb004833dd000703730006027800dc
:10fb500006ae2000164378008683fb0016ae200018
:10fb6000164378000683fb004833dd00070373006b
:10fb7000860278001e0378001603be0006036a00a2
:10fb800087836a00e2cabf008080fb00e3cabf002f
:10fb90000080fb004800dd000100700000027800da
:10fba000e4cabf008080fb00e5cabf000080fb0004
:10fbb0004800dd0001007000800278000600780037
:10fbc00007037800840378000502780007006000ce
:10fbd0000402630005002000c022dd0004002000b4
:10fbe0000403be006102b800040373008583730040
:10fbf000e00f5300e08f5b00070032001e02900010
:10fc000005bb200005000900355a78006400b100ea
:10fc100014002000010037000002eb00040078000f
:10fc20000080fa00000006000200fa00000f7800d1
:10fc30001e02780014027800040078007267020047
:10fc400000000000000278009e027800840a78001c
:10fc50001e0278001402900004007800726702000f
:10fc600000000000000278009e02780094029800d4
:10fc70001e027800340290000400780072670200cf
:10fc800000000000000278009e027800b402980094
:10fc90000080fa00000006000000fa00d782a800e9
:10fca000d382a900e4c2a900e4e2a800e502a90009
:10fcb00034132000141388000002eb002413880082
:10fcc0000002eb000413880061e2a8000080fa0043
:10fcd000000006000400fa00008fbe001e02be00f5
:10fce000645a8800755a88000042eb00044078008e
:10fcf00070ebb7000002eb00040078000080fa000f
:10fd0000000006000000fa0004b72000144278004a
:10fd1000e04f52000f003a00645a8000755a80008c
:10fd20000302200002b520000400be001d000700f1
:10fd3000645a8000755a80000402b0000580b0004b
:10fd4000645a8800755a880004c2b30004407800e1
:10fd500070ebb70004b72000144278008482fb00e7
:10fd6000060220000503530005b52000850243006c
:10fd7000954278000442e9000440780070ebb70037
:10fd800005427800044078000080fa000000060078
:10fd90000000fa000002eb00040078000080fa0086
:10fda000000006000c00fa002007980031079800b8
:10fdb000420798005307980014138000040f78003e
:10fdc000041380004f22de0004427800244798008c
:10fdd00061e2a900341320001413880061e2a80036
:10fde000d782a90034002000441388000413800047
:10fdf00062026200e00f5200fcff3a000413800030
:10fe000061026200e00f5200f8ff320044138000ec
:10fe1000044278003447980064024700144290007e
:10fe20000482fb0044138800041380006202620015
:10fe3000e00f5200fcff3a000413800061026200f0
:10fe4000e00f5200f8ff32004413800004427800b3
:10fe50003447980064024700144278000482fb0093
:10fe6000441388000413800062026200e00f520015
:10fe7000fcff3a000413800061026200e00f5200b0
:10fe8000f8ff3200441380000442780034479800a1
:10fe9000160037000002eb004413880004138000b2
:10fea00062026200e00f5200fcff3a00041380007f
:10feb00061026200e00f5200f8ff3200441380003c
:10fec00004427800344798004e029000e00f520040
:10fed000060032003e429000ce029000844a780034
:10fee0004e0290000402e800440798005e02900071
:10fef00004f0a7000402ea000402ea004f22de0038
:10ff000004427800de0290008502e900550798005f
:10ff1000e04f5200dfff3a00d782a80061e2a9005b
:10ff20001e027800141388002e4290006142620085
:10ff30000482fb004f22dd0006138000f5ff27003e
:10ff40008502630004827200041388000002eb0043
:10ff5000040078000080fa00000006000400fa00a7
:10ff6000008fbe000042eb000440780070ebb70049
:10ff70001e02be00645a8800755a88000002eb0019
:10ff8000040078000080fa00000006000200fa0079
:10ff9000004f780004b72000144278000483fb006f
:10ffa00005b52000850243009e4a78000442e8001f
:10ffb0000440780070ebb70004b7200014427800ca
:10ffc000ff4f520002003600340007000e003700d9
:10ffd000645a8000755a8000044278008482fb00d5
:10ffe00004b72000144278000482fb00048242001f
:10fff00084027800f403200004826200e00f5200c3
:020000040001f9
:1000000001003a00250007000002eb000400780020
:100010000080fa00000006000400fa00000f7800db
:1000200011079800050037001e027800144278007e
:100030001e0fe80004407800d4ff07001e02900065
:1000400004f0a7000402ea000402ea004f22de00e6
:10005000044278009e0290008502e900150798008e
:10006000e04f5200f0ff3a00020007000080fa0063
:10007000000006000000fa0004b7200014427800d7
:10008000e04f520001003200040007000002eb00c4
:10009000040078000080fa00000006000600fa0064
:1000a0001013800010079800041380004f22de0018
:1000b000044278004447980061e2a900341320000c
:1000c0001413880061e2a800d782a9006400200010
:1000d000441388000413800062026200e00f5200a3
:1000e000fcff3a000413800061026200e00f52003e
:1000f000f8ff32004413800004427800544798000f
:10010000d782a800d782a9002400200044138800c9
:100110000413800062026200e00f5200fcff3a000c
:100120000413800061026200e00f5200f8ff320009
:10013000441380000442780054479800c4b420005f
:10014000144290000482fb004413880004138000d2
:1001500062026200e00f5200fcff3a0004138000cc
:1001600061026200e00f5200f8ff32004413800089
:100170000442780054479800c4b420001442780028
:100180000482fb00441388000413800062026200b2
:10019000e00f5200fcff3a0004138000610262008d
:1001a000e00f5200f8ff3200441380000442780050
:1001b000544798000042eb00044f780013003700ca
:1001c0001e4278008482fb0004b5200004824200b5
:1001d000144278000482fb0044138800041380005a
:1001e00062026200e00f5200fcff3a00041380003c
:1001f00061026200e00f5200f8ff320044138000f9
:1002000004427800544798001e4fe80004b72000cd
:10021000144278009e42780084cf5200e8ff3900f3
:10022000d782a80004b72000144278000483fb00a2
:1002300007002000645a8000755a800006024200c0
:1002400087824a00645a8800755a88000042eb0091
:100250000440780070ebb70061e2a9001e02900034
:10026000141388004e429000614262000482fb0039
:100270004f22dd0006138000f5ff27008502630092
:1002800004827200041388000000000005000700cb
:1002900000027800e00f5200fcff3a000080fa00f4
:1002a000000006000400fa0014138000040f780018
:1002b000041380004f22de00044278002447980097
:1002c00061e2a900341320001413880061e2a80041
:1002d000d782a90054002000441388000413800032
:1002e00062026200e00f5200fcff3a00041380003b
:1002f00061026200e00f5200f8ff320044138000f8
:1003000004427800344798000002eb004413880050
:100310000413800062026200e00f5200fcff3a000a
:100320000413800061026200e00f5200f8ff320007
:10033000441380000442780034479800d782a80014
:1003400061e2a9001e027800141388002e4290007a
:10035000614262000482fb004f22dd000613800030
:10036000f5ff2700850263000482720004138800f1
:100370003e429000614262000482fb00040078006b
:100380000080fa00000006000000fa000002eb0006
:10039000145e88000aeba800845e8000e00f520023
:1003a00008003a0028630200000000000002be00be
:1003b0000400be007662020000000000140020006d
:1003c000845e8800fc38020000000000987b020078
:1003d000000000009e51020000000000ca1502004b
:1003e000000000000040eb00b846020000000000e2
:1003f000a4b02000144278000444b200e04f520040
:1004000003003a000040eb00044702000000000037
:100410000080fa00000006000a00fa00a4b02000e4
:10042000144278000444b200e04f52007a003200d7
:10043000523a02000000000000027800040f780029
:10044000745e80009e027800848f52006900320042
:100450001e007800705e88001e027800e00f5200d7
:1004600064003a0026af2000164378008683fb0024
:1004700036af2000164378000683fb004833dd00ca
:10048000070373000602780046af20001643780089
:100490008683fb0056af2000164378000683fb00de
:1004a0004833dd000703730086027800f60f200052
:1004b00086036200e6ad20001643780060436300c7
:1004c0000743730006407800deeab700c823de0069
:1004d000f6ad2000164378006043630007437300c5
:1004e00006407800dfeab700f60f2000868362003e
:1004f00006ae200016437800604363000743730094
:1005000006407800e0eab700c82ade0014ae2000fa
:100510001442780060426200054272000440780094
:10052000e1eab70066af2000164378008683fb003f
:1005300076af2000164378000683fb004833dd00c9
:10054000070373000602780086af20001643780088
:100550008683fb0096af2000164378000683fb00dd
:100560004833dd000703730086027800f60f200091
:100570008603620026ae20001643780060436300c5
:100580000743730006407800e2eab700c823de00a4
:1005900036ae2000164378006043630007437300c3
:1005a00006407800e3eab700f60f20008683620079
:1005b00046ae200016437800604363000743730093
:1005c00006407800e4eab700c82ade0054ae2000f6
:1005d00014427800604262000542720004407800d4
:1005e000e5eab7000aeba8000040eb00b8460200bd
:1005f00000000000d6470200000000000040eb00b1
:10060000504702000000000000027800e00f520096
:10061000010032000aeba900762002000000000071
:10062000d25202000000000001003700000000006c
:10063000285802000000000068024700840078008b
:1006400080bc2000de3a02000000000000027800ba
:10065000e00f52009f0032000e4a90000482fb001f
:10066000e00f520005003200e60f5200efff3a00a3
:10067000ca7b020000000000950037000e83e800ee
:10068000e90247006402470086017800050178000e
:1006900041bc2000040078004886020000000000f1
:1006a00000027800e00f520001003a008800370095
:1006b0001e4a9000e14f52006c003a002e03900059
:1006c000be039000decabf008080fb00dfcabf000f
:1006d0000080fb004800dd0001007000000278008f
:1006e000e0cabf008080fb00e1cabf000080fb00c1
:1006f0004800dd000100700080027800840f530084
:10070000858f5b00530032002e039000be039000e3
:100710000082eb008082eb00840f5300858f5b002a
:100720004c0032002e009000be009000e4ad20008e
:10073000144278008482fb00f4ad2000144278005b
:100740000482fb004822dd000502720004037800e9
:1007500004ae2000144278008482fb0014ae200016
:10076000144278000482fb004822dd00050272007a
:100770008403780022ae2000124178008281fb00c1
:1007800032ae2000124178000281fb004811dd00ea
:10079000030171000202780042ae2000124178008d
:1007a0008281fb0052ae2000124178000281fb00e2
:1007b0004811dd0003017100820278000601780013
:1007c00007037800840378000502780007016100c0
:1007d0000402630005002000c022dd0004002000a8
:1007e0000403be006112b800040373008583730024
:1007f00022ae2000124178008281fb0032ae200040
:10080000124178000281fb004811dd0003017100f4
:100810000202780042ae2000124178008281fb0083
:1008200052ae2000124178000281fb004811dd0029
:1008300003017100820278000482ea008582ea00e6
:100840000402730085827300840f5000858f580066
:1008500005003a001e0290008400780040bc200091
:10086000448d020000000000190037001e4a90006d
:10087000e64f520008003a009e02900064024700d2
:10088000050178008400780040bc20008625020025
:10089000000000000e0037001e4a9000f14f520089
:1008a0000a003a009e0290006402470005017800a9
:1008b0008400780040bc200048580200000000007e
:1008c00000027800e00f520004003a00000000002f
:1008d00057ff370000000000010037000000000053
:1008e0000080fa00000006000000fa002c850200db
:1008f000000000000080fa00000006000200fa007c
:10090000523a02000000000000027800e00f52009e
:100910004c003200f4652700c3b220000041eb0018
:100920006000b800b85102000000000000427800ea
:10093000144798001e429000e14f420043003200ed
:10094000000000001e409000be55020000000000a4
:1009500000027800e00f5200faff3200f1002000a0
:10096000a0af20002456020000000000d0c0b30059
:10097000f455020000000000a0c0b300f4550200ce
:10098000000000000042eb00044f78009e42780017
:100990000582fb00c502200084824200f4ad2000e5
:1009a0000482420014427800044078009a660200f3
:1009b000000000000042780004407800f455020076
:1009c000000000009e4278000582fb00c502200066
:1009d00084824200f4ad2000048242001442780078
:1009e00004407800bc66020000000000004278006d
:1009f00004407800f4550200000000001e4fe8009b
:100a00001e427800e64f52000a003a00844d290049
:100a10000400780060560200000000007e560200cc
:100a2000000000001e409000505502000000000031
:100a300007003700d0c2b300f455020000000000e8
:100a4000d2ff370000000000010037000000000066
:100a50000080fa00000006000200fa00345f800007
:100a6000050020003600200007002000860f5200fd
:100a7000878f5a0084003e000460010003003700a5
:100a8000130037003200370076003700f465270086
:100a9000f36527000041eb006000b800b851020088
:100aa000000000000042780004407800e8ebb70046
:100ab00084be200014427800e14f42006b003200f7
:100ac000345f80000402e800345f88006e00370065
:100ad00084be200014427800044078007857020059
:100ae0000000000000027800e00f520061003200b8
:100af0000e007800a85702000000000028580200ed
:100b0000000000009e42780044c4b30084cf52002d
:100b10005a003a00345f80000402e800345f880025
:100b200084be2000144278000482fb007822b900c1
:100b3000840278000490200004824200a200200079
:100b400041bc200004007800d80b02000000000027
:100b500084be20001442780004407800be55020094
:100b60000000000000027800e00f52004500320053
:100b7000f1002000a0af2000245602000000000079
:100b8000d0c0b300f455020000000000a0c0b300c4
:100b9000f4550200000000000042eb00044f780012
:100ba0001e4278000482fb00c502200084824200bd
:100bb000f4ad200004824200144278000440780022
:100bc0009a660200000000000042780004407800ad
:100bd000f4550200000000001e4278000482fb0071
:100be000c502200084824200f4ad2000048242004d
:100bf0001442780004407800bc6602000000000047
:100c00000042780004407800f45502000000000023
:100c10001e4278000442e800044f78001e4278002b
:100c2000e64f52000b003a00d0c0b300f45502006a
:100c300000000000a0c0b300f45502000000000056
:100c40007e5602000000000014002000345f88007f
:100c50000d003700d0c2b300f455020000000000c0
:100c6000cfff370000000000070037000000000041
:100c700005003700000000000300370000000000fe
:100c800001003700000000000080fa0000000600ac
:100c90001e00fa00300f9800410f9800520f980084
:100ca000630f98000e82e8004101200004007800e4
:100cb000e23e0200000000002e4290008482fb0011
:100cc000040f20008482620004042000848f5200fc
:100cd000020032000002eb004f003700ce0290000d
:100ce000f4f12f0004826200e00f52000200320093
:100cf0000002eb00480037002e4290006f42620075
:100d0000250020000522dd0004407800f4ebb70048
:100d100044bf2000144278000482fb008400780065
:100d20000000eb00243d02000000000000027800fb
:100d3000040f780044bf2000144278000482fb00b6
:100d400004007800ce3c0200000000001e02780083
:100d5000e00f5200020032000002eb002e003700cc
:100d60000e82e80004007800920007003e0a90001e
:100d7000e00f5200040032001e0a9000ae0a9000fc
:100d80003e0b9000048bbe007e0390008e0b900003
:100d90004e0a9000f50f2000050063009442780091
:100da000e0c2620080c27200054a78004830de006e
:100db00094429000e0c2620080c272001542980026
:100dc000f50f200005806300a4429000e0c262009d
:100dd00080c2720025429800483bde00b442900079
:100de000e0c2620086c27200354298003e4a90001e
:100df000de0a9000844a7800ae02900044bf2000d2
:100e0000144278000482fb00848252006e0a900033
:100e1000050a780014002000040078000080fa0021
:100e2000000006001a00fa00200f98006157980091
:100e3000420f980044c1b30004407800f4ebb700bf
:100e400054c4b300044f78000042eb0014479800ec
:100e50004e0a90007402420014079800945f8000cc
:100e60000402e800945f8800945f800024079800e3
:100e70000002eb003407980044c6b300044f98000a
:100e80006e529000144f98000002eb005407980037
:100e9000e6ad2000164378008683fb00f6ad200007
:100ea000164378000683fb004833dd000703730018
:100eb0000602780006ae2000164378008683fb0009
:100ec00016ae2000164378000683fb004833dd0091
:100ed000070373008602780064079800750798007e
:100ee0002e0b9000164278000480fb009643900081
:100ef0008783fb00c83bdd00808373000702780016
:100f0000a64390008783fb00364390000683fb00d6
:100f10004833dd000703730086027800040f980051
:100f2000150f98000e0078002200070041012000f4
:100f30000e007800ee67020000000000000278005a
:100f4000540798004e0a9000f40242002e0a9000c6
:100f500064024200050178008040eb000400780044
:100f60002a3c020000000000410120000e00780031
:100f70002c3f0200000000000002eb00040078009b
:100f80000080fa00000006000200fa00000f78005e
:100f900044bf2000144278000482fb001e0242007d
:100fa00004007800ce3c0200000000000080fa003f
:100fb000000006000200fa00000f78001e02780010
:100fc0001402900004007800726702000000000024
:100fd000000278009e027800940298001e027800b9
:100fe00024029000040078007267020000000000f4
:100ff000000278009e027800a40298001e02780089
:1010000054029000040078007267020000000000a3
:10101000000278009e027800d40298000080fa0056
:10102000000006000200fa00004f78001147980007
:10103000852d20000042eb00844a7800c7e2a90019
:10104000d2a2a900d6a2a9009e42780061c2620085
:101050000482fb004f22dd0056168000f5ff2700ba
:10106000850263000482720054168800c42d20009b
:101070009e429000054a7800000000000000000039
:10108000d682a80000000000000000000000000060
:101090000000000000000000000000000000000050
:1010a0000000000000000000d682a9000080fa00c5
:1010b000000006000200fa000202200001022000e7
:1010c00020b72000e60b0200000000000042eb0009
:1010d0000440780092ebb700d682a900d6a2a900fe
:1010e000852d20000042eb00844a7800d2a2a9009e
:1010f000c7e2a900d282a90080022000d88d020098
:1011000000000000cbe2a900c52d200034c0b300d0
:10111000844a780000000000000000000042eb005c
:10112000044f78000a003700d682a8001000200083
:1011300001002000148e020000000000d682a900e9
:1011400020002000d88d0200000000001e4fe800a3
:101150001e427800e24f5200f3ff360081c3b30015
:101160000040eb00afff070050002000010020000e
:10117000148e02000000000061c0b3000040eb00cc
:10118000a8ff07005000200001002000148e02007c
:1011900000000000c1c0b3000040eb00a1ff070049
:1011a0005000200001002000148e0200000000000a
:1011b00011c0b3000040eb009aff070020002000a0
:1011c000d88d0200000000000080fa000000060038
:1011d0000200fa0021c0b3000040eb0091ff0700bd
:1011e00020002000d88d0200000000000042eb002b
:1011f000044f7800230037001e4278008482fb00f1
:1012000024b720000482420014427800e04f5200cc
:101210000f003a001e42780014479800090037007a
:101220001e4290008482fb0024b72000848242008a
:1012300004c2b300844a78001e4290000442e800d1
:10124000144798001e429000ef4f5200f4ff360002
:101250001e4278008482fb0024b7200004824200f2
:10126000144278008440780010c0b3006dff07007e
:101270005000200001002000148e02000000000039
:101280001e4fe8001e427800ef4f5200daff360092
:1012900001ccb3000040eb0062ff070050002000cb
:1012a00001002000148e02000000000004c1b30001
:1012b000044f7800230037001e4278008482fb0030
:1012c00024b720000482420014427800e04f52000c
:1012d0000f003a001e4278001447980009003700ba
:1012e0001e4290008482fb0024b7200084824200ca
:1012f00004c2b300844a78001e4290000442e80011
:10130000144798001e429000ff4f5200f4ff360031
:101310001e4278008482fb0024b720000482420031
:10132000144278008440780010c0b3003dff0700ed
:101330005000200001002000148e02000000000078
:101340001e4fe8001e427800ff4f5200daff3600c1
:101350000080fa00000006000000fa0011c0b3008f
:101360000040eb002fff070020002000d88d020076
:1013700000000000020220000102200020b720002f
:10138000e60b0200000000000080fa0000000600ea
:020000040000fa
:020000040001f9
:10139000ac0b00001600000000000000e60b00008f
:1013a0000400000000000000020c00000200000029
:1013b0000200000000000000240b000028000000d4
:1013c00000000000ea0b0000040000000200000022
:1013d000ff00070000000000940b00001800000050
:1013e00000000000d20b00000a0000000000000016
:1013f000ee0b000004000000020000009e9ffe00b3
:1014000041000000f20b000004000000000000009a
:10141000720b000022000000000000004c0b0000d6
:101420002600000000000000c20b000010000000b9
:1014300000000000cc090000ca000000000000000d
:10144000080c00000200000002000000fefe000088
:10145000dc0b00000a000000000000000009000092
:10146000cc000000000000000a0c00000200000098
:1014700002000000ffff0000f60b00000400000067
:10148000000000000e0c000002000000020000003e
:1014900000000000960a0000480000000200000062
:1014a0000000010001000000000001000101010036
:1014b0000001000001010100000001000101010024
:1014c00000010000010100000100010000022200f3
:1014d00003330400440555000666070077088800ba
:1014e00009990a00aa02220004440600660888003e
:1014f0000aaa010011033300055507007709990076
:10150000fa0b0000040000000000000000080000ca
:101510000001000000000000fe0b000004000000bd
:10152000020000000000000000000000de0a0000d1
:101530004600000000000000100c00000200000047
:101540000200000002000000020d00000600000082
:1015500000000000b20c00002a00000002000000a1
:1015600030313200333435003637380039414200eb
:1015700043444500460030003132330034353600f4
:1015800037383900616263006465660000286e00c8
:10159000756c6c0029000000120c0000a000000017
:1015a00002000000010000000000000000000a002e
:1015b00000000000000000000064000000000000c7
:1015c00000000000e8030000000000000000100020
:1015d000270000000000000000a0860001000000bd
:1015e0000000000040420f000000000000008000ea
:1015f00096980000000000000000e100f5050000e2
:101600000000000000ca9a003b000000000000003b
:10161000e40b5400020000000000e80076481700c8
:10162000000000000010a500d4e800000000000049
:10163000a0724e0018090000000040007a10f3006c
:101640005a0000000080c600a47e8d000300000048
:1016500000c16f00f2862300000000008a5d780060
:101660004563010000006400a7b3b600e00d000070
:1016700000e889000423c7008a000000080d00006c
:101680000600000000000000dc0c00002600000046
:1016900002000000090d000000090d000900000013
:1016a000000200000b0d0000000b0d000e020100f7
:1016b0000000000000000000000000000602020020
:0c16c00000000000dc0c00000000000036
:020000040000fa
:020000040001f9
:1016cc000000fa00240880000440a0000450a00090
:1016dc00240888000082eb00140888000002eb004c
:1016ec00040888002405800004c0a10004d0a000d8
:1016fc0004e0a100240588008460a9009460a8007f
:10170c0005e1a8000080fa00000006000400fa00c1
:10171c009460a800000000009460a90004be2000a2
:10172c0005088000050a7800e45e8000f55e800004
:10173c00048fbe0004be200014027800e10f4200aa
:10174c0004003a001e02be0061025200e0825a0000
:10175c00048fbe000e02780014427800044078001a
:10176c00e2ebb7000e0278000402e80014427800a5
:10177c0004407800e3ebb7000e0278000482e80026
:10178c001442780004407800e4ebb7000e027800b5
:10179c00630242001442780004407800e5ebb70085
:1017ac002404800068026200e00f5200d8ff3a0067
:1017bc009460a8000080fa00000006000000fa0007
:1017cc00d2ff070004be20001402be000400be00bd
:1017dc000080fa00000006000400fa00cbff0700ae
:1017ec008e02780014be200014427800844a7800df
:1017fc000e0278008402e80024be20001442780017
:10180c00844a78000e0278008482e80034be2000fe
:10181c0014427800844a78000e027800e3024200f9
:10182c0044be200014427800844a78001e02be0098
:10183c000400be000080fa00000006000400fa005c
:10184c00b2ff07008e02780024be200014427800fc
:10185c00844a78000e0278008402e80034be20002e
:10186c0014427800844a78000e0278008482e800e2
:10187c0044be200014427800844a78000e0278009e
:10188c00e302420054be200014427800844a7800df
:10189c001e02be000400be000080fa00000006001c
:1018ac000400fa00008fbe001e02be000003eb0015
:1018bc008003eb00f0012000010020006011b80053
:1018cc0004004000858048000601490087814900da
:1018dc00e4032000050020006033b800700a020009
:1018ec00000000000203be000002be000402be00a5
:1018fc000400be000080fa0000000600849fbe00b9
:10190c000000fa00e45e8000f55e80006102420097
:10191c00e0824a00e45e8800f55e88008460a900dd
:10192c000080fa004f02be00004006000000fa00e2
:10193c00e45f8000e10f520015003200e10f52000d
:10194c0003003900e20f52001c0032003100370056
:10195c0014c0b300036222000041eb006000b80029
:10196c00a01602000000000000427800044078003d
:10197c00faebb700a4bf200014427800e24f4200fb
:10198c001f00320014002000e45f880021003700a3
:10199c00a4bf200014427800044078001e180200f6
:1019ac000000000000027800e00f52001600320028
:1019bc0024002000e45f880016003700a4bf20003c
:1019cc0014427800044078001e1802000000000049
:1019dc0000027800e00f52000d003a00a4bf200076
:1019ec001442780004407800e21802000000000065
:1019fc000002eb00e45f88000000000005003700e7
:101a0c000000000003003700000000000100370058
:101a1c00000000000080fa00000006000200fa003e
:101a2c00000f7800a4bf2000144278000440780016
:101a3c001e1802000000000000027800e00f5200a7
:101a4c000c0032009e027800a4bf200014427800e3
:101a5c008500780004407800181b0200000000008c
:101a6c00a4bf20001442780004407800281902001a
:101a7c00000000000080fa00000006000800fa00d8
:101a8c002007980031079800410020000e007800d4
:101a9c00e23e0200000000001e027800e80f520037
:101aac003e003a00be00900040012000243d0200a0
:101abc000000000000027800e00f520036003a00ef
:101acc000042eb00044f78002e4290006842420026
:101adc00244798002e429000e74f52000a003e0027
:101aec003e4290000442e800344798003e42900089
:101afc00e04f520006003a002e4290000442e800eb
:101b0c002447980003003700000000000100370054
:101b1c00000000006c3a0200000000000002780097
:101b2c00e00f5200fbff3200e0002000f03c02000e
:101b3c00000000003e01900011c0b3002e00900088
:101b4c001287020000000000410020000e00780007
:101b5c002c3f0200000000003e0290006402520084
:101b6c00040178008080eb000080eb00143e020042
:101b7c0000000000000000009a3e0200000000007f
:101b8c0000027800e00f5200fbff3200703c0200b4
:101b9c000000000001003700000000000080fa0087
:101bac00000006000400fa00100798000e00370031
:101bbc0044c0b300044f78000300370090012000ac
